:020000040800F2
:1000000000500020CD0F00087D100008E9410008D5
:100010007D1000087D1000087D1000080000000021
:100020000000000000000000000000007D1000083B
:100030007D100008000000007D1000080950000835
:100040007D1000087D1000087D1000087D1000085C
:100050007D1000087D1000087D1000087D1000084C
:100060007D1000087D1000087D1000087D1000083C
:100070007D1000087D100008612900087D1000082F
:100080007D1000087D1000087D1000087D1000081C
:100090007D1000087D1000087D1000087D1000080C
:1000A0007D1000087D1000087D100008612C0008FC
:1000B0006D2C0008752C0008812C000861170008C1
:1000C000E11A000865170008DD1A00087D10000815
:1000D0007D10000895290008D12900087D1000082E
:1000E0007D1000087D1000087D1000080000000051
:1000F0000000000000000000000000000000000000
:0C01000000000000000000005FF808F1A3
:1001100010B5054C237833B9044810B10448AFF347
:1001200000800121217010BDCC05002000000000DE
:10013000FC1E010808B5064B1BB106480649AFF383
:1001400000800648016811B1054A02B1904708BD18
:1001500000000000FC1E0108D0050020CC05002096
:100160000000000081F0004102E000BF83F0004386
:1001700030B54FEA41044FEA430594EA050F08BF42
:1001800090EA020F1FBF54EA000C55EA020C7FEA06
:10019000645C7FEA655C00F0E2804FEA5454D4EB83
:1001A0005555B8BF6D420CDD2C4480EA020281EA4D
:1001B000030382EA000083EA010180EA020281EA85
:1001C0000303362D88BF30BD11F0004F4FEA0131D7
:1001D0004FF4801C4CEA113102D0404261EB4101E6
:1001E00013F0004F4FEA03334CEA133302D052426C
:1001F00063EB430394EA050F00F0A780A4F1010428
:10020000D5F1200E0DDB02FA0EFC22FA05F2801861
:1002100041F1000103FA0EF2801843FA05F3594147
:100220000EE0A5F120050EF1200E012A03FA0EFCC6
:1002300028BF4CF0020C43FA05F3C01851EBE371F0
:1002400001F0004507D54FF0000EDCF1000C7EEB0D
:1002500000006EEB0101B1F5801F1BD3B1F5001F4B
:100260000CD349085FEA30004FEA3C0C04F101046A
:100270004FEA445212F5800F80F09A80BCF1004F93
:1002800008BF5FEA500C50F1000041EB045141EA15
:10029000050130BD5FEA4C0C404141EB010111F416
:1002A000801FA4F10104E9D191F0000F04BF0146C1
:1002B0000020B1FA81F308BF2033A3F10B03B3F19F
:1002C00020020CDA0C3208DD02F1140CC2F10C022F
:1002D00001FA0CF021FA02F10CE002F11402D8BF8D
:1002E000C2F1200C01FA02F120FA0CFCDCBF41EA59
:1002F0000C019040E41AA2BF01EB0451294330BD28
:100300006FEA04041F3C1CDA0C340EDC04F1140404
:10031000C4F1200220FA04F001FA02F340EA0300DB
:1003200021FA04F345EA030130BDC4F10C04C4F121
:10033000200220FA02F001FA04F340EA0300294601
:1003400030BD21FA04F0294630BD94F0000F83F44B
:10035000801306BF81F480110134013D4EE77FEA2E
:10036000645C18BF7FEA655C29D094EA050F08BF7A
:1003700090EA020F05D054EA000C04BF194610465B
:1003800030BD91EA030F1EBF0021002030BD5FEA9F
:10039000545C05D14000494128BF41F0004130BDC7
:1003A00014F580043CBF01F5801130BD01F000451B
:1003B00045F0FE4141F470014FF0000030BD7FEA8E
:1003C000645C1ABF194610467FEA655C1CBF0B4689
:1003D000024650EA013406BF52EA033591EA030FA0
:1003E00041F4002130BD00BF90F0000F04BF002198
:1003F000704730B54FF4806404F132044FF00005CB
:100400004FF0000150E700BF90F0000F04BF002143
:10041000704730B54FF4806404F1320410F00045A9
:1004200048BF40424FF000013EE700BF42004FEAA4
:10043000E2014FEA31014FEA02701FBF12F07F4321
:1004400093F07F4F81F06051704792F0000F14BF1E
:1004500093F07F4F704730B54FF4607401F0004562
:1004600021F0004120E700BF50EA010208BF7047B9
:1004700030B54FF000050AE050EA010208BF7047AE
:1004800030B511F0004502D5404261EB41014FF417
:10049000806404F132045FEA915C3FF4DCAE4FF01B
:1004A00003025FEADC0C18BF03325FEADC0C18BF02
:1004B000033202EBDC02C2F1200300FA03FC20FA53
:1004C00002F001FA03FE40EA0E0021FA02F11444A0
:1004D000C1E600BF70B54FF0FF0C4CF4E06C1CEAB5
:1004E00011541DBF1CEA135594EA0C0F95EA0C0F2A
:1004F00000F0DEF82C4481EA030621EA4C5123EA9D
:100500004C5350EA013518BF52EA033541F48011CB
:1005100043F4801338D0A0FB02CE4FF00005E1FB7E
:1005200002E506F00042E0FB03E54FF00006E1FBC8
:1005300003569CF0000F18BF4EF0010EA4F1FF040B
:10054000B6F5007F64F5407404D25FEA4E0E6D414B
:1005500046EB060642EAC62141EA55514FEAC5205C
:1005600040EA5E504FEACE2EB4F1FD0C88BFBCF5D8
:10057000E06F1ED8BEF1004F08BF5FEA500E50F189
:10058000000041EB045170BD06F0004646EA01014F
:1005900040EA020081EA0301B4EB5C04C2BFD4EB81
:1005A0000C0541EA045170BD41F480114FF0000E7A
:1005B000013C00F3AB8014F1360FDEBF002001F0E8
:1005C000004170BDC4F10004203C35DA0C341BDC62
:1005D00004F11404C4F1200500FA05F320FA04F034
:1005E00001FA05F240EA020001F0004221F0004168
:1005F00010EBD37021FA04F642EB06015EEA430EDB
:1006000008BF20EAD37070BDC4F10C04C4F120050A
:1006100000FA04F320FA05F001FA04F240EA0200BD
:1006200001F0004110EBD37041F100015EEA430E8E
:1006300008BF20EAD37070BDC4F1200500FA05F2AE
:100640004EEA020E20FA04F301FA05F243EA02032D
:1006500021FA04F001F0004121FA04F220EA02003C
:1006600000EBD3705EEA430E08BF20EAD37070BD82
:1006700094F0000F0FD101F00046400041EB010162
:1006800011F4801F08BF013CF7D041EA060195F044
:10069000000F18BF704703F00046520043EB0303FE
:1006A00013F4801F08BF013DF7D043EA06037047EB
:1006B00094EA0C0F0CEA135518BF95EA0C0F0CD0F6
:1006C00050EA410618BF52EA4306D1D181EA03013C
:1006D00001F000414FF0000070BD50EA410606BF36
:1006E0001046194652EA430619D094EA0C0F02D17B
:1006F00050EA013613D195EA0C0F05D152EA0336C0
:100700001CBF104619460AD181EA030101F00041DD
:1007100041F0FE4141F470014FF0000070BD41F026
:10072000FE4141F4780170BD70B54FF0FF0C4CF400
:10073000E06C1CEA11541DBF1CEA135594EA0C0F1F
:1007400095EA0C0F00F0A7F8A4EB050481EA030E6C
:1007500052EA03354FEA013100F088804FEA033353
:100760004FF0805545EA131343EA12634FEA022221
:1007700045EA111545EA10654FEA00260EF00041E2
:100780009D4208BF964244F1FD0404F5407402D234
:100790005B084FEA3202B61A65EB03055B084FEAC5
:1007A00032024FF480104FF4002CB6EB020E75EBC2
:1007B000030E22BFB61A754640EA0C005B084FEAEA
:1007C0003202B6EB020E75EB030E22BFB61A754667
:1007D00040EA5C005B084FEA3202B6EB020E75EBB2
:1007E000030E22BFB61A754640EA9C005B084FEA2A
:1007F0003202B6EB020E75EB030E22BFB61A754637
:1008000040EADC0055EA060E18D04FEA051545EA25
:1008100016754FEA06164FEAC30343EA52734FEACE
:10082000C2025FEA1C1CC0D111F4801F0BD141EA47
:1008300000014FF000004FF0004CB6E711F4801FAC
:1008400004BF01430020B4F1FD0C88BFBCF5E06F8C
:100850003FF6AFAEB5EB030C04BFB6EB020C5FEA9C
:10086000500C50F1000041EB045170BD0EF0004EF1
:100870004EEA113114EB5C04C2BFD4EB0C0541EA23
:10088000045170BD41F480114FF0000E013C90E620
:1008900045EA060E8DE60CEA135594EA0C0F08BFE4
:1008A00095EA0C0F3FF43BAF94EA0C0F0AD150EAE3
:1008B00001347FF434AF95EA0C0F7FF425AF104676
:1008C00019462CE795EA0C0F06D152EA03353FF49E
:1008D000FDAE1046194622E750EA410618BF52EA1B
:1008E00043067FF4C5AE50EA41047FF40DAF52EAEF
:1008F00043057FF4EBAE12E74FEA4102B2F1E04369
:1009000024BFB3F5001CDCF1FE5C0DD901F0004CF6
:100910004FEAC0024CEA5070B2F1004F40EB830046
:1009200008BF20F00100704711F0804F21D113F172
:100930003872BCBF01F00040704741F480114FEAAB
:100940005252C2F11802C2F1200C10FA0CF320FA34
:1009500002F018BF40F001004FEAC1234FEAD32351
:1009600003FA0CFC40EA0C0023FA02F34FEA4303BB
:10097000CCE77FEA625307D150EA01331EBF4FF044
:10098000FE4040F44000704701F0004040F0FE405F
:1009900040F40000704700BF80F0004002E000BF5C
:1009A00081F0004142001FBF5FEA410392EA030F5A
:1009B0007FEA226C7FEA236C6AD04FEA1262D2EBA4
:1009C0001363C1BFD218414048404140B8BF5B42A9
:1009D000192B88BF704710F0004F40F4000020F042
:1009E0007F4018BF404211F0004F41F4000121F058
:1009F0007F4118BF494292EA030F3FD0A2F10102A2
:100A000041FA03FC10EB0C00C3F1200301FA03F1DF
:100A100000F0004302D5494260EB4000B0F5000F02
:100A200013D3B0F1807F06D340084FEA310102F1C1
:100A30000102FE2A51D2B1F1004F40EBC25008BF73
:100A400020F0010040EA03007047490040EB00003D
:100A500010F4000FA2F10102EDD1B0FA80FCACF16C
:100A6000080CB2EB0C0200FA0CF0AABF00EBC2506B
:100A700052421843BCBFD0401843704792F0000F59
:100A800081F4000106BF80F400000132013BB5E7AC
:100A90004FEA41037FEA226C18BF7FEA236C21D022
:100AA00092EA030F04D092F0000F08BF0846704787
:100AB00090EA010F1CBF0020704712F07F4F04D155
:100AC000400028BF40F00040704712F100723CBF68
:100AD00000F50000704700F0004343F0FE4040F492
:100AE000000070477FEA226216BF08467FEA236350
:100AF0000146420206BF5FEA412390EA010F40F43B
:100B0000800070474FF0000304E000BF10F0004386
:100B100048BF40425FEA000C08BF704743F096436D
:100B200001464FF000001CE050EA010208BF704788
:100B30004FF000030AE000BF50EA010208BF70470F
:100B400011F0004302D5404261EB41015FEA010C24
:100B500002BF84460146002043F0B64308BFA3F11C
:100B60008053A3F50003BCFA8CF2083AA3EBC253FE
:100B700010DB01FA02FC634400FA02FCC2F120021D
:100B8000BCF1004F20FA02F243EB020008BF20F054
:100B90000100704702F1200201FA02FCC2F12002BA
:100BA00050EA4C0021FA02F243EB020008BF20EAAF
:100BB000DC7070474FF0FF0C1CEAD0521EBF1CEADD
:100BC000D15392EA0C0F93EA0C0F6FD01A4480EACB
:100BD000010C400218BF5FEA41211ED04FF00063B4
:100BE00043EA501043EA5111A0FB01310CF00040E0
:100BF000B1F5000F3EBF490041EAD3715B0040EA06
:100C0000010062F17F02FD2A1DD8B3F1004F40EBD5
:100C1000C25008BF20F00100704790F0000F0CF0A8
:100C2000004C08BF49024CEA502040EA51207F3A6C
:100C3000C2BFD2F1FF0340EAC250704740F4000047
:100C40004FF00003013A5DDC12F1190FDCBF00F038
:100C500000407047C2F10002410021FA02F1C2F1E6
:100C6000200200FA02FC5FEA310040F1000053EA82
:100C70004C0308BF20EADC70704792F0000F00F0D0
:100C8000004C02BF400010F4000F013AF9D040EAD6
:100C90000C0093F0000F01F0004C02BF490011F46A
:100CA000000F013BF9D041EA0C018FE70CEAD15368
:100CB00092EA0C0F18BF93EA0C0F0AD030F0004CE8
:100CC00018BF31F0004CD8D180EA010000F000409C
:100CD000704790F0000F17BF90F0004F084691F05A
:100CE000000F91F0004F14D092EA0C0F01D1420294
:100CF0000FD193EA0C0F03D14B0218BF084608D15D
:100D000080EA010000F0004040F0FE4040F40000A6
:100D1000704740F0FE4040F4400070474FF0FF0C39
:100D20001CEAD0521EBF1CEAD15392EA0C0F93EA80
:100D30000C0F69D0A2EB030280EA010C49024FEAD2
:100D4000402037D04FF0805343EA111143EA10138B
:100D50000CF000408B4238BF5B0042F17D024FF443
:100D6000000C8B4224BF5B1A40EA0C00B3EB510F1E
:100D700024BFA3EB510340EA5C00B3EB910F24BF07
:100D8000A3EB910340EA9C00B3EBD10F24BFA3EB8C
:100D9000D10340EADC001B0118BF5FEA1C1CE0D154
:100DA000FD2A3FF650AF8B4240EBC25008BF20F007
:100DB000010070470CF0004C4CEA50207F32C2BF5B
:100DC000D2F1FF0340EAC250704740F400004FF0F8
:100DD0000003013A37E792F0000F00F0004C02BF29
:100DE000400010F4000F013AF9D040EA0C0093F0F3
:100DF000000F01F0004C02BF490011F4000F013B4D
:100E0000F9D041EA0C0195E70CEAD15392EA0C0FB4
:100E100008D142027FF47DAF93EA0C0F7FF470AFEC
:100E2000084676E793EA0C0F04D14B023FF44CAF2F
:100E300008466EE730F0004C18BF31F0004CCAD1C4
:100E400030F000427FF45CAF31F000437FF43CAF00
:100E50005FE700BF4FF0FF3C06E000BF4FF0010C22
:100E600002E000BF4FF0010C4DF804CD4FEA400204
:100E70004FEA41037FEA226C18BF7FEA236C11D04E
:100E800001B052EA530C18BF90EA010F58BFB2EB01
:100E9000030088BFC81738BF6FEAE17018BF40F081
:100EA000010070477FEA226C02D15FEA402C05D135
:100EB0007FEA236CE4D15FEA412CE1D05DF8040BBA
:100EC000704700BF844608466146FFE70FB5FFF74D
:100ED000C9FF002848BF10F1000F0FBD4DF808ED05
:100EE000FFF7F4FF0CBF012000205DF808FB00BFF6
:100EF0004DF808EDFFF7EAFF34BF012000205DF850
:100F000008FB00BF4DF808EDFFF7E0FF94BF01209C
:100F100000205DF808FB00BF4DF808EDFFF7D2FF99
:100F200094BF012000205DF808FB00BF4DF808EDDC
:100F3000FFF7C8FF34BF012000205DF808FB00BFA9
:100F40004FEA4002B2F1FE4F0FD34FF09E03B3EBD6
:100F500012620DD94FEA002343F0004310F0004F16
:100F600023FA02F018BF404270474FF0000070476C
:100F700012F1610F01D1420205D110F0004008BF0B
:100F80006FF0004070474FF00000704742000ED2F3
:100F9000B2F1FE4F0BD34FF09E03B3EB126209D4B4
:100FA0004FEA002343F0004323FA02F070474FF06A
:100FB0000000704712F1610F01D1420202D14FF0DF
:100FC000FF3070474FF00000704700BF1D481E49BA
:100FD000026800608A4200F01F80002100F004B81F
:100FE0001A4B5B584350043119481A4B42189A4225
:100FF000FFF4F6AF184A00F003B8002342F8043BB0
:10100000164B9A42FFF4F9AF09F078FC0CF0CEFCD5
:1010100003F0E4F8FFF7FEBF114E124830601248AB
:10102000016821F070610160410201600F4C1820DD
:1010300020600F490F4808600F48D0F800D0406882
:1010400000470000F04F0020EFBEADDE201F01087A
:1010500000000020CC050020CC0500209C1E0020B4
:10106000181002400900000004000140140C014067
:10107000000C01404434434400F0FF1FFFF7FEBF63
:10108000064B187820B1012806D14FF4805201E0B8
:101090004FF4006202490A80704700BFE805002053
:1010A0000400002007B5232003F0E1FF682075212C
:1010B00001220DF1070300F0EFFB30B19DF80700AE
:1010C000B0F16803594251EB03000EBD13B506227F
:1010D000044643216B46682000F0DEFB9DF80020AB
:1010E0009DF8013043EA022001B2042391FBF3F2A0
:1010F0009DF802009DF80310228041EA002210B200
:1011000090FBF3F19DF805209DF80400618042EA10
:10111000002108B290FBF3F3A3801CBD13B5062297
:1011200004463B216B46682000F0B6FB9DF800208A
:101130009DF801309DF8021043EA02209DF803203B
:10114000208042EA01239DF804009DF80510638089
:1011500041EA0022A2801CBD07B5204A02204FF4BC
:101160000053ADF804308DF8070013681C480421C3
:1011700083428DF8061001D11A4803E01A498B42C8
:1011800003D11A4801A900F059FD6B218022682083
:1011900000F046FC052003F06AFF192100226820B8
:1011A00000F03EFC6B210322682000F039FC37215F
:1011B0000222682000F034FC0D4A1A2168201278BF
:1011C00000F02EFC1B211822682000F029FC68206A
:1011D0001C21102200F024FC0EBD00BF780100206D
:1011E00000127A00000C0140001BB7000010014003
:1011F0000000002030B585B00446FFF753FF0028FB
:1012000041D006210A46682002AB00F045FB9DF85C
:101210000B309DF80D5003F0010105F001004A006C
:1012200042EA80059DF8090000F001031D4307D044
:10123000012D164801D1002318E0022D0CD114E035
:101240000C21682001220DF1070300F025FB9DF819
:10125000071011F00F0203D1052003F07BFF06E019
:10126000042A0A4801D1057001E0012303700748F0
:1012700007490378074A2160002B14BF6E216F21B4
:1012800062602172012005B030BD00BFE80500207A
:10129000811000081D11000838B505460C46FFF7FF
:1012A00001FF28B3134B14481449142C2B606860B9
:1012B000E960134B15D004D8052C16D00A2C0ED19A
:1012C00011E0BC2C08D0B4F5807F03D0622C06D18D
:1012D00002220BE0002209E00120187038BD032231
:1012E00004E0042202E0052200E006221A70012038
:1012F00038BD00BF59110008CD10000819449231C3
:101300000000002070B5414C414E2568414B04223D
:101310000021B54290B01A7059704FF0010403D10A
:101320000522DC709A700224007820B1394B013418
:10133000611E18715971384D3848394E0AF0C6FA95
:10134000202105954FF480700025012C14BF8022C8
:101350002A464FF4806306960B900D914FF4005689
:101360002E4805A90A920C930E96079508940995A4
:101370000F950AF023FB012128480AF04CFB012CB1
:101380004FF46020D4BF002201220290012625489C
:1013900069468DF8042000958DF8056003958DF859
:1013A000104009F031FC04211E483246032309F0A5
:1013B0007CFC3146A1420ADA164B4D1C194813F841
:1013C0001110EAB2032309F070FC2946F2E7154830
:1013D000012109F046FC1348012109F039FC1148AC
:1013E00009F048FC0F4809F04AFC0028FAD10D48E2
:1013F00009F049FC0B4809F04BFC0028FAD10948D8
:10140000012109F049FC10B070BD00BF7801002037
:10141000001BB700E90500204C24014008000240F1
:10142000F005002000240140044B054903EB400077
:10143000427831F8123098B2704700BFE9050020B9
:10144000F00500202DE9F84F9C4C2068838A9BB260
:1014500013F0010239D0018821F400631A04110C41
:10146000018001210AF010FA954A964B117800206C
:101470001870D9B1944803781BB9944A1178FF29A0
:1014800014D10123037092480278022A06D18B49B5
:101490000B68188882B242F4006119808D4B87482E
:1014A0001978006801220AF009FA2FE18948834B74
:1014B0000178002218680AF001FA844A1178FF299D
:1014C00000F02481FF207F4BDEE003F00201C9B26F
:1014D00000293DD0BFF35F8F7D4D2E78012E35461C
:1014E00016D177490B789BB177490B7883B11146B8
:1014F0000AF0CAF9BFF35F8F20683146038B0AF008
:10150000B7F9754A206816704FF480613246FBE0E7
:10151000038BBFF35F8F6E490A78022A09D1684BAB
:101520001A7832B1684B1A781AB100210AF0ACF976
:10153000E5E00978032907D1614B1A7822B16249A5
:101540000B78002B40F0DD804FF480610122DBE05E
:1015500003F00406F6B2002E71D0594BDFF8788103
:101560001A78012688F80060574B002A4DD01A7867
:10157000002A4AD0564D2F78524D022F574F29D965
:101580000AF082F9206895F80090D7F800A00AF0D8
:1015900092F94FFA89FB0AF80B0009EB0600314675
:1015A000287020680AF064F9206888F800603F68B5
:1015B00095F800800AF07FF94FFA88F907F80900DA
:1015C000B04420684FF48061324685F800800AF00C
:1015D00067F92BE031460AF04BF920682E78D7F8EE
:1015E00000800AF068F94FFA86F9731C08F80900C0
:1015F000D9B220684FFA81F83F6829700AF05BF988
:10160000033607F808002E7010E01B78012113B98B
:10161000334A13782BB10AF02BF92A480278511C6F
:1016200003E00AF019F9284801210170234A1168E2
:101630000B8803F4807082B2002AF9D166E003F0CF
:1016400040010F461F4D09B3244B2F78D3F800807B
:101650000AF031F94FFA87F908F80900781CC1B28D
:1016600029701B4D4FB22A780337BA4205D1206842
:101670004FF4806132460AF013F9124B28781A7839
:1016800051B2884242D1501C18703FE01B063DD534
:101690002B785EB2721C27D0124901330A682B7076
:1016A000915D0AF006F90A4895F900200178914207
:1016B0002CD120684FF480613A4625E00C060020CA
:1016C000090600200806002000060020FA05002078
:1016D000FB05002011060020F9050020FC05002074
:1016E000F805002004060020154A297011780AF038
:1016F000E0F81448017811B9134B1A7832B913483D
:1017000000684FF4806100220AF0CAF80E4A104BBC
:10171000117893F900004A1C90420ED10D4B0E49EE
:10172000187800220A7028B1084908684FF44071FF
:101730000AF0B6F8094B00221A70BDE8F88F00BF16
:10174000FA05002009060020FB0500200C060020F9
:1017500008060020F90500200006002010060020E1
:10176000FFF770BEFFF76EBEF0B5484C89B04FF47E
:1017700040651C2307460226204602A9ADF8085002
:101780008DF80A308DF80B6000F058FA40481421AB
:1017900007608DF80E10204603A9ADF80C508DF8A7
:1017A0000F6000F04BFA25610825384CA2685205FD
:1017B00003D40A2003F050FCF7E74FF480660A20B8
:1017C000666103F049FC6F1E0A20266103F044FCA9
:1017D00017F0FF05E9D14FF4006767610A2003F0B5
:1017E0003BFC66610A2003F037FC26610A2003F007
:1017F00033FC022027611C218DF80F002046244C69
:101800004FF440638DF80E1003A9ADF80C3000F0D2
:1018100015FA206809F082FF04A80AF003F820688E
:101820002A464FF440710AF03BF81A484FF48043BF
:101830004BF6FF72049001212068ADF81C30ADF822
:101840001620ADF8145009F0FBFF04A9206809F038
:101850007FFF4FF4A06009F075FA2221012201A850
:101860008DF804108DF805508DF806508DF807207E
:1018700009F072FA212301A82E468DF804308DF864
:10188000055009F069FA09B0F0BD00BF000C014035
:101890000C060020801A060010B54000244CC0B28F
:1018A00020702448244C017000212170234C012019
:1018B0002070234C2360234C2360234B1A70234A4F
:1018C00010702348017023490868838803F400726C
:1018D00091B2A1B9038803F4807291B241B903882F
:1018E00003F4007291B20029F9D1012109F0B4FF8B
:1018F00018484FF440710068012209F0D1FF47F207
:101900003053124A117811B1013BFAD100E053B9BA
:1019100011490A88501C83B20B800E490868FFF7F2
:1019200023FF002010BD0A4B187880F0010010BD85
:1019300011060020FA050020F80500200906002005
:10194000FC05002004060020FB05002010060020F6
:10195000010600200C060020F605002010B540000E
:10196000244CC0B220702448244C0170244901202A
:10197000087000212170234C2360234C2360234BEB
:101980001A70234A1070234801702349086883881D
:1019900003F4007291B2A1B9038803F4807291B28A
:1019A00041B9038803F4007291B20029F9D10121F1
:1019B00009F052FF18484FF440710068012209F005
:1019C0006FFF47F23053124A117811B1013BFAD13F
:1019D00000E053B911490A88501C83B20B800E49AC
:1019E0000868FFF7C1FE002010BD0A4B187880F090
:1019F000010010BD11060020FA0500200906002094
:101A0000F805002004060020FC050020FB0500204E
:101A100010060020010600200C060020F60500201C
:101A200007B502AB03F8012D0122FFF797FF0EBDAA
:101A3000274B37B51868818A8AB20192019B13F44B
:101A4000706F02D0234A01211170019B13F4E06FE3
:101A500031D04FF480610022038B09F021FF0198FF
:101A6000810528D41A4D2868018801F4007293B2C8
:101A70000BBB048804F480718CB29CB1028802F420
:101A8000807399B20029F9D1012109F0F1FE1048C3
:101A90000068028802F4007399B20029F9D1FFF7B7
:101AA00063FE08E0012109F0E3FE28684FF440716D
:101AB000224609F0F5FE06480268938A23F4706115
:101AC0000804030C0449938200220A703EBD00BF43
:101AD0000C0600200106002010060020FFF7A8BF1A
:101AE000FFF7A6BF014B188880B27047F6050020AB
:101AF000F8B5134B05469B890E461446ECB116B15A
:101B000016F8017B00E0FF270D48022109F076F866
:101B10000028F9D00A48394609F06BF80848012135
:101B200009F06CF80028F9D0054809F064F8C0B253
:101B30000DB105F8010B013CE0E70120F8BD00BF45
:101B4000003800402DE9F047012188B04FF4804073
:101B500009F0B8FD374C01214FF4804009F0CAFD6F
:101B600003214FF420401823ADF800008DF8031036
:101B7000204669468DF802304FF0040800F05EF808
:101B80002D4E4FF4804220466946ADF800204FF4B8
:101B900080554FF0100A8DF8028000F04FF869462A
:101BA0002046ADF800508DF802A000F047F830460E
:101BB00008F0C2FF07214FF4007000230222ADF8A5
:101BC0001600ADF81C104FF00109304603A94FF480
:101BD0008277ADF80C30ADF81030ADF81A30ADF8B2
:101BE0001220ADF80E70ADF814901F46ADF818A095
:101BF00008F0D4FF3046494608F0EFFF9F238DF8E8
:101C000004308DF805708DF806708DF807700DEBB7
:101C100008014246656102A8FFF76AFF25619DF849
:101C20000900B0F1EF014A4252EB010008B0BDE8F3
:101C3000F08700BF000C0140003800402DE9F04162
:101C40000F88002347FA03F2D2072DD58A7803F0D4
:101C50000705DC08AD0012F0100F18BF91F803C0A3
:101C600002F00F0618BF46EA0C064FF00F0C0CFAF4
:101C700005FC06FA05F550F82480282A28EA0C0C01
:101C800045EA0C0540F8245006D1012202FA03F27D
:101C9000C46824EA020206E0482A05D1012202FAB9
:101CA00003F2C4682243C2600133102BCAD1BDE8DD
:101CB000F08100002DE9F843044683796278002B17
:101CC00014BF0220002002B101303A49002551F82A
:101CD0002090A8462F462E4619F80620FF2A02F02B
:101CE0000F0002F0F00363D0A17811B1811E012929
:101CF0005BD9E17811B1011F032956D9E17909B106
:101D0000814252D002F02002D1B219B12278002AC9
:101D100008BF002303F01001CAB21AB1617800298C
:101D200008BF0023227932B1A17921B9A0F10802BC
:101D3000012A98BF8023617929B1A2791AB9011FBC
:101D4000032998BF802303F01002D1B211B100F033
:101D5000CBF92AE003F02002D1B221B1F9B200F0B0
:101D60008DF9013721E003F04002D1B281B122891F
:101D7000114B4FEA0010B2F5FA7F1844E9B2A3897B
:101D800002D900F0E3F801E000F0F6F801350CE0CC
:101D90001B060AD5084B5FFA88F103EB0010628935
:101DA000E38900F0FFF808F1010801360E2E93D107
:101DB000BDE8F883ECF600084CF70008074BA1F5E6
:101DC0007A7153F82000838802684B434FF47A708D
:101DD00093FBF0F18BB21380704700BF1406002014
:101DE000024B53F82000026811807047140600204F
:101DF0002DE9F04F044647488E46057889B0691CA6
:101E00000170914611462068724601930C2700F03C
:101E100075FEA268182303A96F4360684FF0020A99
:101E2000ADF80C208DF80E308DF80FA0FFF706FFEF
:101E300004A8394E256894F80CB009F082F9702096
:101E4000019BADF81000012100224FF4807007EBD8
:101E50000608ADF81210ADF81420ADF81630ADF844
:101E600018A0ADF81C00BBF10C0F2BD8DFE80BF06D
:101E7000072A2A2A102A2A2A192A2A2A2200284628
:101E800004A909F057F82846082109F08FF919E04C
:101E9000284604A909F092F82846082109F08EF98D
:101EA00010E0284604A909F0CDF82846082109F0D9
:101EB0008FF907E0284604A909F006F92846082109
:101EC00009F08EF9A17B19B12068012109F057F9B9
:101ED0002068012109F047F9237B0C2B14D8DFE897
:101EE00003F0071313130A1313130D131313100026
:101EF0002268343207E02268383204E022683C323B
:101F000001E022684032BA51A8F80490404609B076
:101F1000BDE8F08F120600202412002008B5044B03
:101F200053F820301BB10B2801D89A68904708BDA0
:101F300014060020044B53F820201AB107289CBF38
:101F400012681180704700BF4406002010B50C468F
:101F50000649B1FBF2F292B20821FFF749FF044BA8
:101F6000044943F82400816010BD00BF00127A00CC
:101F700014060020BD1D000810B50C460649B1FB33
:101F8000F2F292B20121FFF733FF044B044943F808
:101F90002400816010BD00BF40420F0014060020E5
:101FA000E11D000810B50C46054991FBF2F292B212
:101FB0000121FFF71DFF034B43F8240010BD00BFB4
:101FC00040420F00440600200A4A0B481368116083
:101FD000C91A40F68C2291420360084B01DD0020B3
:101FE00006E01A78072A9CBF054820F81210501CFA
:101FF000187070471C070020780600206406002037
:10200000660600207FB5044601A80D46164609F075
:10201000A2F800200123ADF80A00ADF80C0001A9D8
:102020002046ADF80450ADF80660ADF8083009F070
:1020300013F97FBD0F4B142210B502FB00308278DC
:10204000036932B94160012181701868197B02224D
:102050000BE044688160084A091B4478C16022F89B
:102060001410002282701868197BBDE81040FFF739
:10207000C9BF00BF7C060020660600202DE9F341A1
:1020800014220D466A43154F4FEA0018144908EB15
:10209000070401268B188E54E17BA2685D701C61D9
:1020A000606802238DF8061001A98DF80730ADF89D
:1020B0000420FFF7C3FD58F80700217B0022FFF73B
:1020C000A1FF204632464FF6FF7100F039FD204651
:1020D0002946044A00F0F4FCBDE8FC814CF70008F6
:1020E0007C06002035200008F7B5124E0701BC1908
:1020F000A168114B0025E27B1D701C616068022302
:10210000ADF8041001A98DF807308DF80620FFF70F
:1021100095FDB859217B2A46FFF774FF204601221E
:102120004FF6FF7100F00CFD20462946034A00F0EF
:10213000C7FCFEBD4CF700087C060020C91F000844
:10214000014B33F81000704766060020417170475C
:10215000426A806A131A594251EB030070477FB5F7
:10216000044601A80D46164608F0F5FF002001239D
:10217000ADF80A00ADF80C0001A92046ADF80450F6
:10218000ADF80660ADF8083009F066F87FBD437918
:1021900013F001010BD0026AC3699A4205D09CBFBB
:1021A000C0681218D01AC0B27047002070470846A5
:1021B0007047437910B513F0010104460ED0FFF7C4
:1021C000E6FF60B1E3696269E168D05C4A1E934250
:1021D00001D2013300E00023E36110BD084610BDC9
:1021E00043799A070AD5436A8269D154416A0369DF
:1021F0004A1CB2FBF3F103FB112242627047837960
:10220000012B03D1D1F1010138BF0021D0F83401F5
:102210004268836809B1136170475361704707B51D
:10222000034699684822ADF804100223406801A9CA
:102230008DF806208DF80730FFF700FD0EBD000079
:102240002DE9F74391464FF4127242431F463B4B30
:102250000646D41808B93A4802E0012804D13948A2
:1022600020631030C4F83401374D0020D5500322CC
:102270004FF001086271D4F8342184F8388284F870
:102280003C0284F8390284F84662E1624FF48071BE
:10229000E1602161916804F1340304F59C75636188
:1022A00020621023E061A561A0626062A4F842028E
:1022B000A4F84402ADF80410506801A9C4F80890CD
:1022C000A77102258DF806308DF80750FFF7B6FC90
:1022D000206BFFF7A4FF41462046FFF790FF322016
:1022E00002F0C5FE1948D4F8348103681846B0FBE3
:1022F000F9F1B1F5803F03D30128F8D94008F6E79A
:10230000134A4046B3FBF2F5EAB289B200F018FC7A
:10231000404631460F4A00F0D3FB256B012F14BF16
:10232000022200222868297BFFF719FF2846314640
:10233000094A00F0C5FB2046BDE8FE83B412002028
:102340008CF70008ACF700081CF700087C0100209F
:1023500040420F00852500080D24000803460A4668
:1023600090F84602D96A9B79FFF76ABFC268036A90
:10237000511E8B4201D3002300E0013303627047FA
:1023800010B590F83C220446AAB9836A416A994282
:1023900025D080692169C05C01338B42A36228BFCC
:1023A000A26242000A2342F4007084F83D32A4F88D
:1023B0003E02012311E090F93D3273B1B0F83E12B4
:1023C0004A08A0F83E2201F00101FFF718FF94F837
:1023D0003D02431E84F83D3210BD84F83C3210BDEE
:1023E00090F83B3210B583B990F83A3290F8392220
:1023F00093420AD2012101FA03F1B0F840420133BD
:102400002143A0F84012DBB2F2E710BD2C4B10B50F
:102410004FF4127404FB00346079C1074ED594F870
:10242000381219B3236B0021186808F0E3FE94F802
:102430003C1221B1B4F84202421CA4F84222236BA0
:10244000A2791868197B012A0CBF02220022FFF72B
:1024500086FE0020012184F83B1284F8390284F8BA
:102460003A02A4F8400284F8380210BD94F83B22E6
:102470002046012A04BF94F8392284F83A22FFF753
:10248000AFFF94F83B02236B50B90120A27984F886
:102490003B021868197B012A0CBF0222002209E0C6
:1024A000002184F83B12A2791868197B012A14BF15
:1024B00002220022BDE81040FFF751BE10BD00BF50
:1024C000B412002090F83B1200230122012980F869
:1024D000393280F838220BD180F83B32036B827995
:1024E000197B1868012A14BF02220022FFF737BEA9
:1024F0007047427908B5D20703461BD5B0F8402291
:1025000002F4007189B209B9D10705D4B3F84402C5
:10251000421CA3F8442208BDC16AC2F3470211B1AC
:102520001046884708BD4169036ACA54BDE808409F
:10253000FFF71CBF08BD10B590F838320446002BD9
:102540001ED190F839124A1CD3B2092B80F83932C7
:1025500003D1BDE81040FFF743BF0A2B10D190F81C
:102560003B0228B9B4F8401241F00102A4F840221D
:102570002046FFF7BEFF2046BDE81040FFF7A2BF90
:1025800010BD0000064B10B54FF4127404FB00346C
:102590002046FFF7F5FE2046BDE81040FFF7CBBF11
:1025A000B4120020036B13B15A68006C01E0026A98
:1025B000C069101A18BF01207047436B13B190F81F
:1025C00044007047826A406A111A4B4253EB010083
:1025D00070471FB58368002100934379ADF804105C
:1025E00003F0040101F0FF0231B14FF40051ADF8E6
:1025F00006104FF4806201E0ADF80620ADF8082027
:10260000002213F0010118BF0421ADF80C209A0735
:10261000ADF80A1005D5BDF80A3043F00802ADF850
:102620000A20006D694608F0CFFE05B000BD41717B
:10263000FFF7CFBF8160FFF7CCBF026B034610B539
:10264000406942B11A6CD9688C1A013A18BF114618
:10265000005D196410BD196ADA68405C0131B1FB94
:10266000F2F402FB1411196210BD00002DE9F041D3
:102670001E464B4B8CB098428846174604D11046F4
:10268000314600F0C7F807E04649884240F08380B1
:102690001046314600F014F9002587600562C561D7
:1026A00085624562C0F82C80467185710446FFF74B
:1026B00090FF01A809F0A2F9E06C802701904FF487
:1026C0008052F0070A920B95059507950697089595
:1026D00027D5206BD0B1E368039565692021049369
:1026E0000991029509F0F2F8206B01A909F066F949
:1026F000206B012109F08FF9206D4021012208F0A3
:10270000E1FE206B09F09CF920640AE0206D40F2A4
:10271000255108F0E0FE206D40F22551012208F01D
:10272000B7FE01A809F06AF9A06C002580274FF4D4
:102730008052B10701900A920B950595079506976F
:10274000089523D5606BD8B12369102104930391B8
:10275000099509F0BBF8606B01A909F02FF9012276
:10276000606B022109F062F9606B294609F066F995
:10277000606B394645600122206D08F0A3FE05E03C
:10278000206D40F22771012208F082FE206D0121A8
:1027900008F072FE00E0002420460CB0BDE8F08195
:1027A0000038014000440040836A8169426BC918C7
:1027B000D160416A994203D9CB1A5360816204E027
:1027C0000169CB1A536000228262002180F8441014
:1027D000406B012109F01FB910B5426A8469A15408
:1027E000416A02690131B1FBF2F402FB1411426B40
:1027F000416232B11368DB070BD4BDE81040FFF72C
:10280000D3BF006D40F227710122BDE8104008F0EF
:102810003FBE10BD234B13B5234A986023481A606E
:1028200058614FF4807222480C462249DA601A61DE
:10283000214A9961011D18659964D9641A630121BF
:10284000143A4FF480405A6308F030FF02231821F5
:102850004FF40070A2078DF80330ADF800008DF83A
:10286000021003D515486946FFF7E8F948234FF4ED
:1028700080628DF80230E307ADF8002003D50F48E1
:102880006946FFF7DBF90E2001218DF8040001A84D
:102890008DF805108DF806108DF8071008F05CFA19
:1028A00000481CBDE009002034F700082007002084
:1028B0000038014060080020580002400008014034
:1028C000214B224A13B598600C46802040211A60A3
:1028D000D86019611E4A1F491F485A6198610A1D34
:1028E00019654FF4003001219A64DA6408F0EAFEB9
:1028F000042002231821ADF80000A0078DF8033052
:102900008DF8021003D515486946FFF797F908229C
:102910004823E107ADF800208DF8023003D50F48B9
:102920006946FFF78BF9262001218DF80400022269
:1029300001A88DF805108DF806208DF8071008F015
:102940000BFA01481CBD00BF340A002034F7000810
:1029500060090020004400402008002000080140D9
:1029600010B50B4C4FF4005009F06EF80021606B6D
:1029700009F051F8626AA36A9A4204D02046BDE881
:102980001040FFF711BF012084F8440010BD00BFC4
:10299000E00900200D4B186D028802F080018AB218
:1029A0009AB19A6A596A8A420AD09969895C013255
:1029B00081801969B2FBF1F001FB10229A62704725
:1029C00040F22771002208F063BD7047E009002043
:1029D0001C4B10B51A6D1488A4B204F0200188B203
:1029E00090B1D96A19B1938898B288470CE092885F
:1029F000D9695869D2B24254D869DA68411CB1FB2E
:102A0000F2F002FB1011D96104F08004A4B2C4B149
:102A10000C4B9A6A586A82420BD09869196D805C97
:102A2000013288801969B2FBF1F001FB10229A6231
:102A300010BD186D40F227710022BDE8104008F06B
:102A400027BD10BD340A002030B500240E4D55F8C6
:102A50002450854202D00134E4B2F7E700200B4D48
:102A600035F810508D4202D0451CE8B2F7E704EB70
:102A70008000C0B20F2805D8054C04EB001083601D
:102A80000171027330BD00BF2CF800083CF800084B
:102A9000441700200C2912D8DFE801F007111111AA
:102AA000091111110B1111110D00022104E0042173
:102AB00002E0082100E01021012208F06EBB7047FF
:102AC00038B504460D461346217B00682A46FFF7B9
:102AD000BBFF2068217BBDE83840FFF7DBBF07B5AF
:102AE0008DF80400012000238DF806008DF8070002
:102AF00001A88DF8053008F02FF90EBD7FB504460A
:102B000001A80D46164608F013FB0B4B0B485E431D
:102B100001680023B1FBF6F2013D561E204601A9D3
:102B2000ADF80850ADF80460ADF80A30ADF80630E5
:102B300008F0B6F97FBD00BF40420F007C010020C5
:102B400010B504460068FFF7D9FF2068012108F09E
:102B50000AFB607BBDE81040FFF7C1BF00230C4AB1
:102B600052F82320824202D00133DBB2F7E7002281
:102B7000084830F81200884202D0501CC2B2F7E771
:102B800003EB82030449DAB201EB0210704700BF85
:102B90002CF800083CF800084417002070B50446E3
:102BA00000262E4B9D5D95B90221204608F0FDFBC5
:102BB00001284FD12046022108F002FC2946204678
:102BC000FFF7CCFF0546204608F0E2FB3DE0042D70
:102BD00012D12046294608F0E8FB01283AD12046C8
:102BE000294608F0EDFB29462046FFF7B7FF0546CA
:102BF000204608F0D0FB28E0082D12D120462946B7
:102C000008F0D3FB012825D12046294608F0D8FB3F
:102C100029462046FFF7A2FF0546204608F0BEFBE6
:102C200013E00C2D16D11021204608F0BEFB012820
:102C300010D12046102108F0C3FB29462046FFF79B
:102C40008DFF0546204608F0ACFBAA6801460AB194
:102C5000287B90470236082EA3D170BD3CF80008AF
:102C60000148FFF79BBF00BF002C01404FF08040A0
:102C7000FFF794BF0148FFF791BF00BF0004004079
:102C80000148FFF78BBF00BF000800400248002149
:102C90004FF480720AF082BF4417002010B5FDF790
:102CA00035FF0A49FDF786FF0949FEF737F8094B5A
:102CB000044618680078FDF729FF01462046FDF715
:102CC00079FFFEF763F980B210BD00BF3333534084
:102CD00000F07F459C0A002038B50D4C0020257877
:102CE000FEF7A2FB0B4A05F0070322F8130001359B
:102CF000002325701846D15A02334018102B80B299
:102D0000F9D1C008FFF7CAFF034A107038BD00BFF1
:102D1000880A00208A0A002044180020074B084A2D
:102D200019781088884207D3064B1A689078884231
:102D30008CBF0020012070470020704744180020FD
:102D4000461800209C0A002038B5114B202418603A
:102D500000250020FEF768FB2D180A2002F087F9F5
:102D6000013CF6D1C5F34F10FFF798FF0849012346
:102D70000A6851786418A04202D30133062BF9D1B6
:102D8000044892780370534303490B8038BD00BF59
:102D90009C0A002001000020461800202DE9F04F79
:102DA0000446008885B048B9B4F9023043B9B4F993
:102DB0000420D2F1010138BF002102E0002100E02F
:102DC000014611F0010377D13D4D00B22B7000F0A8
:102DD00087FD0646B4F9020000F082FD0546B4F90D
:102DE000040000F07DFD0446304608F037FE07463B
:102DF000304608F0A7FE8046284608F02FFE06461B
:102E0000284608F09FFE0546204608F027FE824629
:102E1000204608F097FE394681465046FDF7CAFE27
:102E2000394683464846FDF7C5FE51460190404667
:102E3000FDF7C0FE494602904046FDF7BBFE314615
:102E400003905046FDF7B6FE1E4C4946206006F141
:102E50000040FDF7AFFE29466060A5600298FDF7CF
:102E6000A9FE01460198FDF79DFD2946E060039803
:102E7000FDF7A0FE01465846FDF792FD3146206160
:102E800008F10040FDF796FE294660615846FDF7BF
:102E900091FE01460398FDF783FD2946A061019844
:102EA000FDF788FE01460298FDF77CFD3946E0619A
:102EB0003046FDF77FFE206205B0BDE8F08F00BF11
:102EC00002000020A00A00202DE9F8434D4B0C46DB
:102ED0000168013A196080889880072A30D8DFE8B5
:102EE00002F004080F14191E2226188820805A8820
:102EF00003E0598821801A88524262809A881EE035
:102F00001988484220805A88F6E75988484220802C
:102F10001A88F2E719884842208058880CE05A88BD
:102F20002280188808E0198821805A8803E059888F
:102F3000484220801A88504260809B885A42A28072
:102F4000314B1A78002A5AD1B4F90000FDF7DEFDA2
:102F50008046B4F90200FDF7D9FD0746B4F9040034
:102F6000FDF7D4FD294D064629684046FDF722FEAF
:102F7000E96881463846FDF71DFE01464846FDF7E3
:102F800011FDA96981463046FDF714FE0146484609
:102F9000FDF708FD08F096FD696820804046FDF7C2
:102FA00009FE296981463846FDF704FE0146484678
:102FB000FDF7F8FCE96981463046FDF7FBFD014667
:102FC0004846FDF7EFFC08F07DFDA96860804046AB
:102FD000FDF7F0FD696980463846FDF7EBFD0146D7
:102FE0004046FDF7DFFC296A07463046FDF7E2FD63
:102FF00001463846FDF7D6FC08F064FDA080BDE828
:10300000F88300BFC40A002002000020A00A0020AC
:1030100070B5124D06462B78114C9BB102F016F894
:103020002268B318984218D30021297002F00EF8D4
:1030300020600C4802780AB1531E03700A4801212F
:10304000017070BD02F002F821683231884204D369
:103050000120287001F0FAFF206070BDCC0A00202A
:10306000D80A0020CE0A0020CD0A002037B58DF8FE
:1030700005101F498DF807300B788DF8040002A861
:103080008DF80620C21812F8044C0D46443CE0B2FC
:103090000A2828D81749022B31F8104003D814B158
:1030A0002046FFF7B5FF2B78022B0BD9124D2D6868
:1030B00001F0CCFF021B954204D20D490F4B0020BA
:1030C000087018700E4802780146012A00D074B9C1
:1030D000074B1878022801D8421C1A7000230B7085
:1030E00008490B7003E03224022BD9D9DBE73EBD3F
:1030F000CB0A002044F80008D80A0020CE0A00209D
:10310000CD0A0020CC0A0020014B1860704700BF98
:10311000D40A002070B53D4B04465A7B3C4802B1AE
:10312000012202704FF4007000F06CF9002828D0E2
:10313000384E394B316858780D68003018BF01207F
:103140006A68904748B13368344D18680121C268F5
:103150002970904708B1022129702E4D2B681868FC
:103160008268904728B12C494B7813B92B4A02202A
:10317000107029680B689869804710B127490022B0
:103180000A70202004F0B8FC60B12048244B827AF9
:103190000AB9C17A21B12048C27A0AB9012100E0F6
:1031A000002119701D4B1878022802D14C204E21A5
:1031B0001DE0012807D14D2153204C220B46BDE8CC
:1031C0007040FFF753BF164A1178012903D15320ED
:1031D00001464E2206E00E4B1878012804D15320F8
:1031E000014602464D23EAE724B153204D210A4609
:1031F0004423E4E70B4A117821B13220BDE8704046
:10320000FFF706BF084B1C7070BD00BF301E0020CA
:10321000CF0A0020D40A00201F1E0020CA0A002066
:10322000D00A0020CE0A0020CC0A0020014B1870E2
:10323000704700BFCE0A00200E4B1A78422A16D1E2
:103240005888B0F56C7F12D11979BE290FD193F847
:10325000AD230020EF2A0CD113F8011B064A484089
:103260009342F9D1D0F1010038BF0020704700200F
:103270007047704700F80108B0FB0108C82314210B
:103280001E22038001238170C270037164214FF4F8
:1032900096722823C18002814381704710B504468D
:1032A000272005F023FC2070102005F01FFC607023
:1032B000002005F01BFCA070002005F017FC4FF467
:1032C000E133E07052206360A360E360207510BDBD
:1032D0007FB51B4D1B4C284604F044FC2146284674
:1032E00004F05AFC1F3D04F1240001F03DFD2E4680
:1032F00004F1680004F0AAFF16F8C20B02F022F9EC
:10330000304603F055FB681C03F010FC05F1B800D3
:1033100000F0EAFD04F1280001F020FD04F149036A
:1033200004F1380005F1C00100930190029105F10C
:103330007800A11D224605F1BE0302F093FD7FBD7A
:103340001B1C00201819002008B5054BD02202FBD9
:103350000030044900F59E700AF072FB08BD00BF02
:1033600048180020FC1B0020224A38B54223137065
:103370004FF46C700023BE21EF245080117182F84D
:10338000AD4382F8AE331D461A4A985C0133B3F55B
:103390006C7F85EA0005F7D182F8AE5308F0A4F8F7
:1033A00004250024691E11F0FF0516D0342008F012
:1033B000AFF8114808F002F90F4C04280BD10F4A5E
:1033C0002046A15808F0D0F80D4B04349C42F4D1AB
:1033D0000428044601D00446E4E708F091F8042CE0
:1033E00002D1FFF729FF20B90A20BDE8384001F0DB
:1033F000B1BE38BD4818002000F801084820FE176B
:10340000B0FB0108034B996808420CBF0020012063
:10341000704700BF48180020024B9A68104398601C
:10342000704700BF481800202DE9F04FA84AA94D69
:1034300085B010685168A84C02AB03C34FF46C729E
:10344000002128460AF0AAFBD022002120460AF0DB
:10345000A5FB42200321287002206971FFF7DCFFE1
:103460002A232021A5F8EE304FF4FA702B2385F89B
:10347000F41040F24C41FA22A5F8F60085F8053127
:10348000212001F54873A5F8F22085F806016E2287
:1034900040F27E40A5F816314FF47A7300274FF0C2
:1034A00001094FF4167685F80421A5F8141140F2AD
:1034B000DC5200F52F71A5F8D00003F5CB70A5F80C
:1034C0001221A5F8F060A5F8D21085F8AC73A5F824
:1034D000FA70A5F8F870A5F8FC7085F8E27085F828
:1034E000E37085F8E470A5F8E670A5F8E870A5F833
:1034F000EA7085F8ED7085F8EC9085F8077185F82D
:10350000387185F83A7185F8397185F8107185F848
:10351000187185F8197185F81A91A5F8D430A5F8B5
:10352000D6006C30A5F8D8004FF4C870322340F2B2
:10353000B451A5F8DE0005F590709B46A5F8DA10A9
:10354000A5F8DC30A5F8E030019285F81C7185F80B
:103550001D71FFF7A3FE1E211723552040F6AC5224
:10356000E17263752173A3750B211423AA81E070A6
:103570002D2208206171A3710E21637450234FF036
:10358000280862732074A2766420E171E3765A21E0
:1035900078234FF00A0A22754122A3722172207704
:1035A000E177AF7385F81B71277084F8018084F888
:1035B0000280E77584F804B0A7732776E77367760F
:1035C00084F812A084F8098084F81E9084F82020E2
:1035D00084F8237084F8247084F82570019904F12C
:1035E0002A00E18484F821B084F8227001F096FF6B
:1035F00004203A4A84F82E0039493A48152384F8C1
:103600003430A263E163206405F584713648278570
:1036100084F82F8084F8308084F8449004F0D4FB40
:103620004FF44873C8224FF4966140F2D9303E46B9
:1036300084F8707084F8717084F8728084F87390E4
:1036400084F87670A4F8743084F8B8A084F8B920AF
:10365000A4F8BA10A4F8BC004FF47F734FF4FA62D8
:10366000A4F8783007F108006B46A2F5FA71A4F8C7
:103670007A20C25CA4F87C100137FF2184F87E20F8
:1036800084F87F100834082FE6D11348012480F80D
:10369000BE4080F8BF4080F8C040C230FFF7EEFD6A
:1036A00000200C4B0021C2181030C0281161F8D145
:1036B00000240E48D02220180749D0340AF0C0F95F
:1036C000B4F51C7FF5D105B0BDE8F04FFFF74CBE57
:1036D000CCF6000848180020FC1B00209A99193FDE
:1036E000F6287C3F3D0A773F5AF8000884190020ED
:1036F00008B5FFF7A1FD18B9BDE80840FFF794BE73
:1037000008BD0000024B9A6822EA000098607047EA
:1037100048180020214A10B59368144613F4004F4E
:1037200007D1DA0705D4180703D44FF40040FFF798
:1037300073FEA06801070CD5020403D54FF40040C6
:10374000FFF7E0FF15498A68D30702D50120FFF78C
:10375000D9FF124C48F20103A06848F2010103406E
:103760008B4203D14FF40040FFF7CCFFA26848F230
:103770004000104048F24003984202D14020FFF739
:10378000C1FF074805F09CFA054805F057FA20B933
:103790000348BDE81040FFF781BD10BD4818002068
:1037A0006819002010B5FFF747FD10B90A2001F095
:1037B000D1FC0F4C0F4920464FF46C720AF040F9CF
:1037C00094F8AC33022B02D9002084F8AC0394F8AF
:1037D000AC13D02202FB0143074803F59E710AF0A7
:1037E0002FF9FFF797FFBDE81040FFF771BD00BF4D
:1037F0004818002000F80108FC1B002008B5FFF75E
:10380000D1FF0F2014210122BDE8084007F05CB869
:1038100008B5054B93F8AC03FFF796FDFFF7A4FD41
:10382000BDE80840FFF7EABF48180020014B986840
:10383000704700BF48180020884203DB8242B4BFB3
:1038400011460146084670470023036170472DE981
:10385000F041066904460136012E0D46066105D188
:103860000023616021608360BDE8F081D0F80080B2
:1038700008464146FDF794F807463046FDF746F9FD
:1038800001463846FDF74AFA01464046FDF78AF8F8
:103890000646606031462846FDF782F80146384604
:1038A000FDF788F9A168FDF77DF82660E060A0606B
:1038B000BDE8F08110B504460069012807DD013834
:1038C000FDF724F90146E068FDF728FA10BD002055
:1038D00010BD08B5FFF7EEFFBDE8084008F0C0B91D
:1038E00008B5FCF791FD04A3D3E90023FCF7F2FD32
:1038F000FDF702F808BD00BF399D52A246DF913F97
:103900002DE9F041069C06460F46002B0CBF4FF0F8
:1039100020084FF03008204610F8013B0BB915463F
:1039200003E0002AFBDD013AF6E7002D04DD304616
:103930004146B847013DF8E714F8011B11B1304684
:10394000B847F9E7BDE8F081014B186801F032BBD8
:10395000D01C00202DE9F04389B006460F460392A3
:103960001C46039A134613F8011B0393002900F029
:103970008A80252901D0304683E0002004905578C4
:10398000911C302D039105D19578033203924FF0AD
:10399000010800E08046A5F13003D8B2092806D816
:1039A000284603A90A2204AB00F02AF905466C2D2B
:1039B00005D10399012211F8015B039100E0002277
:1039C000642D2FD010D8582D3AD006D8002D5AD0BB
:1039D000252DC6D13046294653E0632DC1D130464E
:1039E0002178251DB8474AE0752D0DD0782D27D0B8
:1039F000732DB6D1251D2468304600943946049AAB
:103A00000023FFF77DFF3AE0251D20680A2122B13F
:103A1000002205AB00F07EF802E005AB00F0AAF84A
:103A20002C4623E005AD04F104092068294612B1B3
:103A300000F095F801E000F0C2F84C46009517E060
:103A400004F104092068102142B1B5F15804634221
:103A500053EB040205AB00F05DF806E0B5F1580346
:103A60005A425A4105AB00F085F84C4605A8009033
:103A700030463946049A4346FFF742FF71E72C4629
:103A80006FE7B8476DE709B0BDE8F0830FB407B53D
:103A9000094904AB0868094953F8042B09680193E4
:103AA000FFF758FF064B186801F0A3FA0028F9D079
:103AB000BDE80E4004B07047E00A0020DC0A002098
:103AC000D01C0020034A044B044900201A600860FF
:103AD000704700BF49390008DC0A0020E00A0020D6
:103AE000014B1860704700BFD01C002070B506461F
:103AF000B6FBF2F40846154614B12046FFF7F6FF70
:103B000005FB1464024B195D00F8011B70BD00BF7A
:103B100063F80008F0B50124B0FBF4F58D4201D341
:103B20004C43F9E70026C4B1B0FBF4F504FB1500E3
:103B3000B4FBF1F41EB9002D01DC002CF4D1092DE9
:103B4000EFB204DD002A0CBF5725372500E03025F1
:103B5000ED1903F8015B0136E5E71C70F0BD0028A4
:103B60000B4603DA2D22404203F8012B0A210022E2
:103B7000FFF7D0BFF0B50124B0FBF4F58D4201D3BF
:103B80004C43F9E70026C4B1B0FBF4F504FB150083
:103B9000B4FBF1F41EB9002D01DC002CF4D1092D89
:103BA000EFB204DD002A0CBF5725372500E0302591
:103BB000ED1903F8015B0136E5E71C70F0BD002844
:103BC0000B4603DA2D22404203F8012B0A21002282
:103BD000FFF7D0BFA0F13003DAB2092A01D81846A6
:103BE0007047A0F16101052901D857387047A0F14D
:103BF0004103052B01D8373870474FF0FF3070472D
:103C00002DE9F8430D6804460F4690469946002674
:103C10002046FFF7DFFF002806DB404504DC08FBF9
:103C2000060615F8014BF3E73D602046C9F8006031
:103C3000BDE8F883931E222B88BF0A22031E10B50D
:103C40000C4603DA2D2001F8010B5842FFF74EFF16
:103C500000210170204610BD30B587B005460C46E6
:103C600003A800210C2209F099FF28460021FDF746
:103C70005DF920B128462949FCF794FE03E0284667
:103C80002649FCF78DFE2649FCF794FFFDF758F90D
:103C9000054685EAE570A0EBE5700A226946FFF764
:103CA000C9FF002D01DB202300E02D2368468DF89D
:103CB0000C300AF0A7FE012807D130228DF80D2024
:103CC0008DF80E208DF80F200CE0022805D1302150
:103CD0008DF80D108DF80E1004E0032802D130206D
:103CE0008DF80D00694603A80AF08AFD03A80AF0C2
:103CF00089FEC51EEDB22A4603A920460AF020FF20
:103D000000236355204607490AF07AFD03A920469F
:103D100049190AF075FD204607B030BD6F12033A0D
:103D200000007A447C0201082DE9F0410278034644
:103D30000130202AFAD0092AF8D02D2A02D10346D0
:103D4000414D04E02B2A08BF03464FF07E551E4626
:103D50000024334616F8010BA0F13007F9B2092907
:103D60000DD83A492046FCF725FF04463846FCF7B3
:103D7000CDFE01462046FCF715FE0446E9E72E2855
:103D800017D1324F334616F8010B3038C2B2092A28
:103D90000FD8FCF7BBFE3946FCF7C0FF01462046B2
:103DA000FCF700FE294904463846FCF703FF0746A6
:103DB000E8E71878652801D0452839D15E782D2E9E
:103DC00002D19F1C012605E02B2E01D05F1C00E0D4
:103DD0009F1C00267B1E002713F8012F303AD1B21A
:103DE000092903D80A2000FB0727F5E7B7F59A7FD2
:103DF00028BF4FF49A77B8464FF07E51B8F1070FBD
:103E000007D908461249FCF7D5FEA8F10808014673
:103E1000F4E707F0070737B108460C49FCF7CAFE7C
:103E2000013F0146F7E72EB12046FCF777FF04E09B
:103E30004FF07E512046FCF7BDFE01462846FCF7B8
:103E4000B9FEBDE8F08100BF000080BF0000204146
:103E500020BCBE4C014B00229A807047E80A00202B
:103E6000034BB3F90400D0F1010038BF00207047C4
:103E7000E80A00200649074B0A68B3F904001378E2
:103E800005214B439842D4BF00200120704700BF5A
:103E9000F00A0020E80A002010B50446FFF7EAFF08
:103EA000002814BF2046002000F0010010BD0000D3
:103EB000074B084A1968B2F904004B780A78D11800
:103EC000052251438842D4BF00200120704700BF23
:103ED000F00A0020E80A0020024B9A88501C9880C3
:103EE000704700BFE80A0020024B00221860024819
:103EF00082807047F00A0020E80A0020034B044942
:103F00001860044800220160C2807047F40A002053
:103F100088F80008E80A002008B501F0F7FA024B1B
:103F200000221A7008BD00BF1F1E002010B5FFF749
:103F3000A1FF00281ED0104B5C78201C18BF012068
:103F4000FFF7AAFF70B10D480D4B01680D484A8973
:103F500001681A805A809A804A88DA800A4BD88889
:103F6000411CD980FFF7A4FF00B91CB9BDE810407F
:103F7000FFF7D2BF10BD00BF1F1E0020F40A0020B3
:103F8000761E0020F00A0020E80A0020044B9A88E0
:103F900011B2142901DD143A00E000229A80704722
:103FA000E80A002003280B4B0AD80B4A12689288B3
:103FB0008A4205D2012101FA00F01A7810431870E4
:103FC0001B780F2B04D1034800210170FFF7DEBFDF
:103FD000704700BFE40A0020F00A002030B5754C9D
:103FE00089B0FFF76FFDFFF783FBFFF7DBFBA07BDB
:103FF000003018BF012001F045F894F8073133B1C3
:10400000012B01D0092B02D18DF80C3004E00021E6
:104010008DF80C1084F8071103A8FDF773F902203E
:10402000FFF7F0F910B16448FEF78EFE6348FEF723
:10403000B5FE022003F06AFD614D5E4AB5F92830F5
:1040400002F1E200B2F8EE1092F8ED2000F04EFF1F
:1040500010B9032001F07EF80A25192001F007F8B5
:104060006C1E192001F003F814F0FF05F5D1514C36
:1040700001F0F2FA607904F1100101F053FFFEF74C
:1040800005FE04F5907004F045FE60790E2801D01D
:10409000082803D101238DF8163001E08DF8165061
:1040A000484C0121204604F0F7FD8DF81200402015
:1040B000FFF7A8F98DF813004FF40040FFF7A2F9BD
:1040C0008DF810000120FFF79DF98DF8110002F026
:1040D0004FFB3B498DF8140091F8C02034F8423C66
:1040E000C2F3800034F8401C8DF815004FF47A724A
:1040F0004FF48040ADF81830ADF81A10ADF81C2020
:10410000FFF780F918B134F8464CADF81C40BDF803
:104110001800B0F5FA7F02D90023ADF81C3025490C
:1041200091F80741B1F81221012CADF81E2004D0FE
:10413000092C01D1072400E0002404A88DF81740C1
:10414000FDF7B8FD2048FFF7D9FE204C2060FEF7B0
:10415000DBFF1D48216803F087FD4FF48070FFF7F7
:1041600051F958B113481A4B90F81D1190F81C21C1
:10417000009300F59070C13302F028FD4FF4006009
:10418000FFF740F908B104F0D7F800F045FF0949FE
:10419000104B4A791860052A03D14FF4C87000F01B
:1041A000CBFC4FF47A7000F0E5FD0B4B0120587307
:1041B00009B030BD481800204C1900202E190020ED
:1041C000FC1B00206819002050190020D41C00207E
:1041D000FD1B0020100B00201F1E002008B5FFF75C
:1041E000FDFE00F0C9F9FCE708B5034BB3F9D400B4
:1041F00001F0AEFFFEE700BF4818002008B500F050
:10420000BFFD0B4B50B19A7842B1597879B9012270
:104210005A70084B08491888088008BD587830B98A
:104220000220FF210122BDE8084006F04DBB08BD79
:104230001F1E0020221D0020E41C00202DE9F04F4D
:10424000A94BAA4AB3F90600D18C85B088420FDB8E
:10425000B0F5FA6F92F8254007DA451A6C43A1F5DC
:10426000FA6694FBF6F4643403E0C4F1640400E0FD
:1042700064249F4A9D4BB2F8127192F9EC2093F896
:1042800023100097574293F87050019193F8716092
:10429000B9B293F824300291002103930A46924F59
:1042A000DDF8008031F907C040F2E637C8EB0C03B7
:1042B00003F2F31EBE4503D8002BB8BF5B4201E0FA
:1042C0004FF4FA73022ADFF834822CD025B1AB42C6
:1042D000CCBFC5EB030300236427DFF844A293FBA4
:1042E000F7FE6FF0630B3AF81E900BFB0E3B0EF1DE
:1042F000010E3AF91EA00FFA89FECEEB0A0E0EFB54
:104300000BFE9EFBF7FEF14428F80190DDF80480D7
:1043100003FB08FE774B9EFBF3F3DB199BB2634371
:1043200093FBF7F712E026B1B342CCBFC6EB030311
:104330000023029F5F43A8F80470039F002BB8BFBF
:104340005B427B436B4F93FBF7F76437674B02EBA2
:10435000030E9EF80190642307FB09F898FBF3F91C
:10436000DFF8C08102F808909EF80B909EF815E0E7
:1043700007FB09F807FB0EF798FBF3F9DFF8A881B4
:1043800097FBF3F302F80890DDF800805A4FC4451C
:10439000D35503DA594BCF5A7F42CF520132023103
:1043A000032A7FF47CAF524C4FF4FA62B4F8141134
:1043B000FFF742FAB4F814614FF47A75801B454355
:1043C000C6F5FA63B5FBF3F564214D4895FBF1F3AF
:1043D0006FF0630630F8132006FB0355013330F904
:1043E000130013B2C01A4543464B444C95FBF1F100
:1043F000587A8A18E280002838D0434F434D3E88CF
:104400002988721A10B2FFF76BFA074607F026FBED
:104410000646384607F096FB0546B4F90200FCF75D
:1044200075FB0746B4F90000FCF770FB3146804687
:10443000FCF7C0FB294681463846FCF7BBFB01462A
:104440004846FCF7ADFAFCF77BFD31462080384644
:10445000FCF7B0FB294606464046FCF7ABFB01469D
:104460003046FCF79FFAFCF76BFD60800220FEF7F8
:10447000C9FF90B1264806220378591CCBB20370BD
:10448000B3FBF2F002FB103111F0FF0F05D1FEF784
:1044900023FCFEF743FC1F4B18701E4A10780030B7
:1044A00018BF0120FEF736FE00F04CFB28B100F0EB
:1044B00067FC38B103F01AFF04E0022003F01CFB94
:1044C0000028F4D01449154A09681368C81A00284E
:1044D0002EDB0C4B587B48BB987001F5F42303F599
:1044E0009070106024E000BF761E0020FC1B0020AE
:1044F000481800200CFEFFFF1B1D0020461E002058
:104500004E1E00201F1E0020221D0020E41C002043
:10451000000B0020FD0A0020F80A0020180B0020E4
:10452000661E00201E1D0020181D0020012199700C
:1045300004F000FC0C4A117831B94FF40060FEF72A
:1045400061FF08B103F004FF202003F0D5FA18B191
:10455000064B186803F0BCFA054882680AB10548A2
:10456000904705B0BDE8F08F84110020F80A0020C4
:10457000001D0020D81C002038B50820FEF742FF9F
:1045800010B1994803F09CFB984B994A1B6811683D
:10459000591A002902DA002800F00E8203F59C4423
:1045A000914820349349146003F09CFB4FF4804001
:1045B000FEF728FF20B1904D2B780BB900F0A6FF35
:1045C0008E4A92F81B11B1B18D4CC81C34F91050B1
:1045D0004FF47A720021A5F57A70FFF72DF9FCF7F8
:1045E00095FA8849FCF79AFB8749FCF7E3FAFCF750
:1045F000CDFC864B18804FF40070FEF703FF20B10E
:10460000834A116808684469A0477C4D0022B5F8C8
:104610001401B5F81641134679499B08555E854249
:10462000C4BF63F07F03DBB2A542B8BF43F04003D1
:104630000232082AF0D17748774A047805469C422E
:1046400004D11078F92803D8411C00E00021117032
:104650004FF480402B70FEF7D5FE68B1674D684B74
:10466000B5F81211B5F8DC20B3F90640881A844277
:1046700002DD8B189C420CDB4FF48040FEF7C2FE3B
:10468000D8B95F4C5D49B4F90650B1F81421954290
:1046900013DA00F047FF00F04DFF6048B0F84630F5
:1046A0005BB1554C5E492578002D00F011820A78E7
:1046B000002A00F00D82FFF7A1FD574B1C78142C47
:1046C00040F0CA80564D6C78ECB1544BB3F846506C
:1046D0002DB950490C785F2C01D100F017FF474AE3
:1046E00092F81801002800F0B7804C4BB3F8465000
:1046F000002D40F0B18047490C787D2C40F0AC8013
:1047000000F004FFA8E0434D2978572911D14FF458
:104710007A7000F02FFB4FF48070FEF773FE08B143
:1047200002F0B2F9082003F0E7F9E0B93D4B188038
:1047300019E00420FEF766FEA8B12A785A2A12D1A1
:104740003948037823B104703848012202700AE026
:10475000374C257885F00101217009B1022000E075
:104760000320FEF763FD2B4C25785D2D00F0B7810B
:104770005B2D00F0B6815E2D00F0B581274BB3F8BC
:10478000465035B923490C786F2C02D1FFF736FD1E
:1047900015E01A4A1F4B92F8180118B115B91D7887
:1047A0007E2DF3D01978972904D14FF4C87000F00A
:1047B000C3F904E0A72902D1194A012494731548CA
:1047C0000378BB2B03D11548818D8D1C04E0B72BDA
:1047D00004D11248838D9D1E858531E0BE2B29D1E1
:1047E0000E4D6A8D941C2AE050190020F80A002012
:1047F000040B0020741E0020301E002048180020EA
:10480000761E002000007A4400C07F44E21C002095
:10481000D41C0020FF0A00201C0B0020FC1B0020E1
:104820001F1E0020221D0020160B00200C0B002054
:10483000FC0A0020BD2B0FD16E4D698D8C1E6C853E
:104840006D4C94F8AC03FEF77FFDFEF78DFDFEF78F
:10485000D5FF6A48002202700420FEF7D3FD00282D
:104860002CD0674B1A788AB16648457875B166498D
:10487000614AB1F90640B2F81401844206DD634D85
:104880002C781CB9624932220A801C705F4B587C1C
:1048900050B1604B1D782DB95F4C227812B95C483D
:1048A00032210180012008E05B4D2C7834B1554A5B
:1048B000517819B9594B2970012018700023584CB0
:1048C0001A4634F8020F40F2135501B2A942CCBF88
:1048D0000025012505FA03F5A0F21550B0F5C77FB4
:1048E0008CBF002001202A435D1C00FA05F0024322
:1048F00040F2A4608142D4BF00210121981C01FA3A
:1049000000F103330A430C2B92B2DAD10023394968
:104910003E4C01EB4300B0F846100A420CBF0020A9
:10492000012018550133152BF1D1627822B10220F4
:1049300003F0E2F868B914E04FF40070FEF762FD8E
:1049400078B1384C21680868836898470028EED110
:1049500007E02C4CE17839B900F0E4FD0120E0706B
:1049600002E0284C0022E270284B264C987830B1A7
:1049700021790022E27019B900F0D4FD01202071E4
:10498000224B1A7812B91F4801210170202003F030
:10499000B3F808B103F03EF81C4B1A491A7B02B178
:1049A000012215488A724379082B01D00E2B44D17D
:1049B000144A0021517240E01B480368042B3CD884
:1049C000DFE803F00305080B3400012202600168F0
:1049D0004B1C03600268511C0160134803685A1C99
:1049E00002604FF48070FEF70DFDF8B102F00CFA92
:1049F00023E000BFFC1B0020481800201C0B0020F7
:104A0000FC0A00201F1E0020761E0020301E002001
:104A1000140B0020FE0A0020160B00200C0B0020B7
:104A20007C1E0020D41C0020200B002036480021D2
:104A300001604FF40050FEF7E5FC00F0EDFA334959
:104A4000334B8A891860334B1AB11968411A00290F
:104A500059DB84181C6001F003F8FFF7EFFB00F04E
:104A6000DBFA2D4B2A4A19681060441A18602B484B
:104A70002B4A90F87630148053B12A49CC780CB97F
:104A80000A792AB12848294BC48819880A19C28092
:104A9000202003F031F840B12248C3790BB9017AE4
:104AA00019B1047B0CB102F02BFF2148214A174BAE
:104AB00000F11E011468B3F8F62000F12903A047A5
:104AC00001F058FB01F0D4FABDE8384001F02CBBEE
:104AD000487800283FF4F1AD00F018FDEDE5012124
:104AE00002E0022100E00321CCB20848621E80F8F7
:104AF000AC23FEF739FCFEF755FE022028212246A2
:104B000005F0E2FE3AE638BD200B002048180020F0
:104B1000F80A0020080B0020100B0020FC1B0020CE
:104B20000E0B00201F1E0020461E0020480C0020F7
:104B3000FD1B002008000020014B1880704700BFBB
:104B40003C0B0020034B1888D0F1010038BF002037
:104B5000704700BF3C0B0020F8B51E4B00221968BF
:104B600013461D4C2588B5F5C87F1C4D01D1002684
:104B7000EE501B4EEF5832F906C0184C6744EF5008
:104B80000025043395538D5202320C2BE9D1124B80
:104B90001A88012A18D1236803F1C8024FF4C87398
:104BA00092FBF3F20A806268C83292FBF3F24A8009
:104BB000A268C83292FBF3F30A4A12889B1A8B80D0
:104BC00000F0ACFCFEF724FE034801884A1E028078
:104BD000F8BD00BFF41C00203C0B0020300B00206F
:104BE0003C1D002004000020F8B5354B0446188811
:104BF00032280ED13349344D0A6834481688578814
:104C00009388218862882E806F80AB8001804280EB
:104C100001E0002834D02B4D00222E681346284F87
:104C20002B493888322801D10025CD502948CD584C
:104C3000175EED19CD50002104331152B1520232EA
:104C40000C2B0D46EBD11E480188012914D1224BB3
:104C5000224A022011701D70FEF7E8FA1A4A19481C
:104C60001188036850889288198058809A80174B61
:104C70001988588821806080114B1A88511E19802C
:104C800017480378DBB10F4900220B681049027006
:104C90000868322290FBF2F01880486890FBF2F02E
:104CA000588089680F4891FBF2F201882046521A19
:104CB0009A8000F033FCBDE8F840FEF7A9BDF8BDCE
:104CC000140B0020F41C00203E0B0020460B00209B
:104CD000240B00203C1D0020FE0A0020160B0020A3
:104CE0000C0B002004000020064B02881988891A4A
:104CF000198042885988891A5980808899880A1AA7
:104D00009A8070473C1D00200F4B10B5596804462F
:104D10000E4888470D480E4A01461278FEF7D4F82F
:104D20000C48038813B12046FFF716FF0420FEF756
:104D300069FB10B12046FFF757FF07490868BDE837
:104D40001040FFF7D1BF00BFE81C00203C1D002031
:104D50004A0B00203C0B0020F41C0020014B186083
:104D6000704700BFF41C0020014B1860704700BF63
:104D7000600B0020014B1880704700BF640B0020BF
:104D8000034B1888D0F1010038BF0020704700BFE6
:104D9000640B00202DE9F8433C4B3D485968884797
:104DA0003B483C4A01461278FEF78EF83A480388A1
:104DB000002B42D0394C256800242F782646254602
:104DC00035490A88B2F57A7F08D1354B354A00203B
:104DD0001421E85001FB0620FEF736FDDFF8B08015
:104DE0002F4B38F90400E9584FF014090A18EA501B
:104DF0002C4B09FB0639FBF789FE01464846FEF7B6
:104E000026FD002024F80800DFF88C802649B8F839
:104E100000206052012A2FD14846FEF75AFD8146F4
:104E2000DFB13846FBF772FE01464846FCF77EF8D4
:104E300098B14FF47A73A8F80030154B1A4A1888C5
:104E40001188401A1880518858889288401A998889
:104E50005880881A9880BDE8F883114B4FF47A7215
:104E6000E858114B00F5FA7191FBF2F0E0520F2176
:104E70000A20012205F028FD013604350234032EF4
:104E80009ED105490A88501E0880D6E7001D0020E3
:104E9000241D0020A40B0020640B0020600B0020C8
:104EA000540B0020680B00205C0C00200146034BD3
:104EB000034800221A70FCF7EFB900BFA40B0020D2
:104EC000001D002003780BB1054A1370417809B129
:104ED000044B1970807808B1034A1070704700BF06
:104EE000A40B00204A0B0020500B00202DE9F041BC
:104EF0000646084614461D46FFF7D8FF002849D04D
:104F0000254B0022022C1A7007D0072C01D024B1A7
:104F10000AE0022002F002FE06E02048FCF76AF9EF
:104F200010B11F49022008701D4A13782BB90CB12B
:104F30001C46E5E7022002F0F1FD3046FFF7C2FF14
:104F4000022002F0D9FD10B1144C206880471549A9
:104F5000154C0A689047082002F0CEFDB8B16427CE
:104F600095FBF7F63046FBF7D1FD804607FB165060
:104F700000B2FBF7CBFD0D49FBF71CFE0146404696
:104F8000FBF710FD0A49FBF715FE206001E0002346
:104F900023600120BDE8F0814A0B0020E81C0020BE
:104FA000440B0020001D0020540C00208988883C00
:104FB0000000204108B503681A68904708BD38B55D
:104FC00005460C4614F8011B19B12846FFF7F2FFFD
:104FD000F8E738BD08B503685968884708BD08B5C3
:104FE00003689968884708BD08B50368DA68904780
:104FF00008BD08B503681969884708BD08B5036886
:105000005A69904708BD7047024B1A68501C1860D7
:10501000704700BFA80B002010B5094A0949136862
:105020008C6810688342F8D1074A106811684FF401
:105030007A725043001BB0FBF1F102FB031010BD6C
:10504000A80B002010E000E0AC0B0020014B18681A
:10505000704700BFA80B002038B50446FFF7DCFFFF
:105060000546FFF7D9FF401BA042FAD338BD10B563
:1050700004462CB14FF47A70FFF7EEFF013CF8E7DD
:1050800010BD000030B587B005F098FC012126481E
:1050900006F018FB012144F61D2006F007FB012055
:1050A000014606F0F7FA002506F030FB06AC4FF695
:1050B000FF7369461D4824F8183D8DF80250FCF72F
:1050C000BDFD69461A48FCF7B9FD69461948FCF769
:1050D000B5FD1948426842F000714160FFF793FF47
:1050E00001A806F089FA019B1448154AB3FBF0F1B8
:1050F0001448116001684FF47A73B1FBF3F2124B5C
:10510000501E124A5860F021072082F823109D603B
:1051100018600F48FCF728FBFCF714FD6420FFF72C
:10512000A6FF07B030BD00BF0700400000080140E7
:10513000000C0140001001400000014040420F00FF
:10514000AC0B00207C01002010E000E000ED00E04E
:105150000058004010B540F2DB146043841E204626
:10516000FFF785FF1920FFF782FFF8E710B1034A28
:10517000034B1A6003480449C8607047EFBEADDEB8
:10518000F04F00200400FA0500ED00E02DE9F04F9B
:1051900089B00793754B07460692B3F90000B3F93F
:1051A00002200028B8BF4042002AB8BF5242002463
:1051B0008242B8BF024605922546A146A046049405
:1051C000A24626466A49CB7813B90A79002A38D014
:1051D000022E36D0674B6548EA5EDDF818B0295ECE
:1051E00002EB4100CBF100015A46FEF725FB624974
:1051F000DDF81CC06B5E3CF90520C01A8318F879F5
:10520000FA7E584364214FF0050E90FBF1F06FF0E9
:10521000040151430EFB02F20393FEF70DFBDFF88E
:1052200078B1039B824654F80B00544942F2107245
:105230001818FEF701FB7A7C44F80B005043011369
:1052400004914B48C3781BB102790AB9022E2FD1C1
:105250004649502035F90180DFF828B100FB08F2FB
:10526000BB5DDFF8389135F90B0092FBF3F154F890
:1052700009300A1AD01842494FF47A52FEF7DCFA84
:1052800035F90B1049F804000029B8BF4942B1F5BF
:10529000207F02DD002049F8040059F80420B919E4
:1052A0007D23887A92FBF3FC00FB0CFE4FEAAE19DB
:1052B0002F4B1A79B2B1022E14D0DDF814B0DDF8FC
:1052C00010C00BFB08F0CBF5FA7303FB0A020BFBD3
:1052D00009F003FB0C034FF4FA7192FBF1F293FB1C
:1052E000F1F308E0D97809B1022E02D14B464246CB
:1052F00001E0049B52462349DFF8A4B0695A16F82E
:105300000BC008B20CFB00FB6FF04F0C9BFBFCFCCE
:1053100094441D4ACDF800C035F902C0A952CCEB27
:1053200000001A4ADFF87CC0019054F80C10A05815
:105330004018019902904018A15844F80C100199A6
:10534000A150134A0434B15C202201FB00F090FB11
:10535000F2F1581A009B0F49C21801366A52023501
:10536000032E7FF42FAF09B0BDE8F08F461E00205A
:105370001F1E0020FC0E0020580C0020F0D8FFFF5C
:1053800080C1FFFF240C0020BC0B0020D80B0020A4
:105390001B1D0020121D0020D00B0020B00B002090
:1053A0001E1D0020C40B00202DE9F04F002485B005
:1053B000039305468946924606462346474AD178D6
:1053C00009B91079B8B1022C17D0454B454F33F9C4
:1053D000140037F91420CAF1000102EB40005246D4
:1053E000FEF72AFA4049039F31F9143037F91420A7
:1053F000C01A83180AE0022C08D1394A99F80570BE
:10540000B2F904101B374F43791114E03348C178C7
:1054100071B9334F99F8042037F914101B324A43FD
:105420000079111138B16A7C5A4301EB222102E064
:10543000EF795F4339112D4FDFF8C4C037F91400FD
:10544000BCF800200F1A295D7A437943DFF8B48055
:10545000D0124FEAE11B58F82420B17A01FB00205A
:10546000234948F824004FF400120293CDF804C0F9
:10547000FEF7E2F91F4BDDF804C053F8241043F89F
:105480002470791ABCF800704FF6FF723B09B2FB2A
:10549000F3F74F43184BDFF870C048F824005CF86E
:1054A000241053F82480BF1108EB010243F8247044
:1054B000337DD11959430BEB6030104A00EB2121A9
:1054C0004CF8248022F8141001340136032C029B7E
:1054D0007FF474AF05B0BDE8F08F00BF1F1E002041
:1054E000461E0020FC0E0020580C0020240C00203A
:1054F0000000E0FFF00B0020FC0B0020121D00203C
:105500000E0B0020B00B0020E40B0020024B5A7859
:105510000AB10020587070471F1E0020002303802E
:1055200043807047024B00221A605A60704700BFE8
:10553000D00B0020024B00221A605A609A6070471C
:10554000B00B00200128034B14BF034A034A1A6022
:10555000704700BF080000208D510008A9530008C3
:105560002DE9F84F384E04463768384606F076FA8B
:105570000546384606F0E6FA76688046304606F07C
:105580006DFA8346304606F0DDFAD4F804900646FC
:1055900029464846FBF70EFBA76882464146384637
:1055A000FBF708FB01465046FBF7FAF921688246F3
:1055B0005846FBF7FFFA414604464846FBF7FAFA1D
:1055C0003146FBF7F7FA01462046FBF7EBF9314687
:1055D00004463846FBF7EEFA2946FBF7EBFA01469C
:1055E0002046FBF7DFF90146504606F037FB174926
:1055F000FBF7E0FAFAF71AFF11A3D3E90023FBF750
:1056000093F8134B044618680D46FAF70FFF02464D
:105610000B4620462946FAF7ABFD00220D4BFBF75F
:1056200083F8FBF769F906F04DFA81B20A0444BF2A
:1056300000F5B47189B208B2BDE8F88FAFF300800D
:10564000182D4454FB2109401C0C00200000E144AB
:10565000540C00200000244010B5194C2088FBF7A2
:1056600055FA1849FBF7A6FA06F02CFA164B1880E3
:105670002088FBF74BFA01461448FBF74FFB14490F
:10568000FBF74CFB134908601348B0F87400FBF7B4
:105690003DFA01461148FBF741FBFAF7C7FE06A3A6
:1056A000D3E90023FAF716FFFBF726F90C4A10603E
:1056B00010BD00BFAFF300803B597E90A9E7814049
:1056C00004000020C903683F180C00200AE81C41B0
:1056D00000401C46381D0020FC1B002000006144D7
:1056E000541D0020AFF300802DE9F041044600680E
:1056F0000D460146FBF75EFAD4F8048006464146A3
:105700004046FBF757FA01463046FBF74BF9A768CE
:10571000064639463846FBF74DFA01463046FBF758
:1057200041F906F09DFA00210646FBF7D7FB70B958
:1057300020683146FBF7F2FA314628606068FBF7D3
:10574000EDFA31466860A068FBF7E8FAA860BDE8AA
:10575000F0812DE9F04F0C68836889B0D0F800A083
:10576000D0F804800646204603938B4606F076F96F
:105770000746204606F0E6F9DBF80440814620465D
:1057800006F06CF90546204606F0DCF9DBF8082047
:1057900004461046019206F061F98346019806F02E
:1057A000D1F9394602905846FBF704FA394604907D
:1057B0000298FBF7FFF9594605904846FBF7FAF9BE
:1057C000029906904846FBF7F5F929460790584696
:1057D000FBF7F0F901465046FBF7ECF9214683460A
:1057E0000698FBF7E7F901460598FBF7DBF8014659
:1057F0004046FBF7DFF901465846FBF7D3F8214650
:1058000083460498FBF7D6F901460798FBF7C8F8DA
:1058100001460398FBF7CEF901465846FBF7C2F85C
:105820003060029905F10040FBF7C4F9014650468B
:10583000FBF7C0F9214683460798FBF7BBF9014601
:105840000498FBF7ADF801464046FBF7B3F9014673
:105850005846FBF7A7F8214683460598FBF7AAF9B7
:1058600001460698FBF79EF801460398FBF7A2F95C
:1058700001465846FBF796F8214670605046FBF704
:1058800099F92946044609F10040FBF793F90146CE
:105890004046FBF78FF901462046FBF783F839466F
:1058A00004462846FBF786F901460398FBF782F980
:1058B00001462046FBF776F8B06009B0BDE8F08FEE
:1058C00080EAE073A3EBE0738B4206DB002801DD86
:1058D000401A704702D040187047002070470000FF
:1058E0002DE9F041524B86B01A685B6802F1004224
:1058F00003F1004301934F4B0646B3F900000092B9
:10590000FBF704F900F10040FAF790FD46A3D3E954
:105910000023FAF7DFFDFAF7EFFF474C0290B4F9E6
:105920000000FBF7F3F80390B4F90200FBF7EEF880
:105930000490B4F90400FBF7E9F86946059003A860
:10594000FFF707FF3D4B93F84430012B16D13C483D
:10595000417869B93B4C4025226892FBF5F7D01B92
:10596000FBF7D4F80599FBF71DF8FBF7E9FA20607F
:10597000344B4021186890FBF1F001E0324B18885D
:10598000FBF7C4F801460598FBF70AF80590304686
:10599000FBF7B8F82D490746FBF704F801463846EF
:1059A000FBF7BCF92A4D07462C6805982146FAF703
:1059B000F7FF01463846FBF7FDF801462046FAF7A7
:1059C000F1FF244C28601D4D07460398D4F8008051
:1059D00006F078F895F83010FFF772FF08EB000238
:1059E00004982260D4F8048006F06CF895F8301022
:1059F000FFF766FF08EB000338466360D4F80880C1
:105A000006F060F895F82F10FFF75AFF1249134B74
:105A10000A684044A0601868B6180E60411C1960FE
:105A200006B0BDE8F08100BF399D52A246DF913F2C
:105A30001C0C0020221D00204C1D0020FC1B0020FF
:105A40001F1E0020400C0020040000203661823C14
:105A5000500C00202C1D0020440C00204C0C002079
:105A60002DE9F04F87B0FFF795F9022002F044F8D6
:105A7000002800F0AD81AE48FFF746F9FFF7CCFAF9
:105A8000AC4C05462768C71B3846FBF73BF8AA49CC
:105A9000C968FBF78FF88346A848256090F82E80E8
:105AA00000252C462E46A64A105FFBF72FF85946D4
:105AB000FBF780F803AB5851B8F1000F27D04046F0
:105AC000FBF724F801464FF07E50FBF727F9DFF88B
:105AD000B092824651464FF07E50FAF761FF55F87A
:105AE0000910FBF767F897490346085F0193FBF736
:105AF0000DF85146FBF75EF801460198FAF752FFA0
:105B000049F80500FBF71CFA8F4A105303E08D4952
:105B10008D4A605AA0528C4B0435E15E0234062C4B
:105B200001FB0166BFD1894A6420138846435B4369
:105B3000874803A996FBF3F6FFF70BFE082001F058
:105B4000DBFF20B1834803A9FFF703FE07E082488B
:105B500003A9FFF7FEFD80480146FFF7C5FD493E5A
:105B60007E49B4B23B2CB1F8F00007D97B4E082037
:105B7000B6F8F25001F0C0FF30BB4FE0FAF7C2FFB9
:105B80004FF07E518046FAF70DFF01464FF07E50F0
:105B9000FBF7C4F8002406466D4D404655F8141036
:105BA000FBF708F881466848005FFAF7AFFF014647
:105BB0004846FAF7F7FE3146FAF7FCFF45F81400BD
:105BC0000234062CE8D1D1E7B6F8F200FAF79AFFD2
:105BD00080462846FAF796FF4FF07E51FAF7E2FE2C
:105BE00001464FF07E50FBF799F800240646594DC8
:105BF000404655F81410FAF7DDFF594A8146105F08
:105C0000FAF784FF01464846FAF7CCFE3146FAF728
:105C1000D1FF45F814000234062CE8D1514B4C4D0D
:105C2000B3F90000FAF772FFAC680146204601267E
:105C3000FBF77CF900B906464B4968684E7321466C
:105C400006F00CF8494CD5F808802060286800F16F
:105C5000004668680146FAF7ADFF414605464046F2
:105C6000FAF7A8FF01462846FAF79CFE05F0F8FF70
:105C70000146304605F0F2FF60602068FAF7D6FB77
:105C800029A3D3E90023FAF725FCFAF735FE05F03E
:105C900019FF374D28806068FAF7C8FB22A3D3E9C3
:105CA0000023FAF717FCFAF727FE05F00BFF6880D0
:105CB000082001F021FF2F4C08B1264800E02648BB
:105CC000FFF74EFC1D4D20803846FFF709FE95F882
:105CD0007620002A00F080801D4B18689C680146E1
:105CE0005F68FAF767FF394606463846FAF762FFFB
:105CF00001463046FAF756FE214606462046FAF798
:105D000059FF01463046FAF74DFE05F0A9FF01465E
:105D10002046FBF703F818490446FBF7F3F888B36D
:105D200016480021018057E03B597E90A9E7814049
:105D3000261C0020140C0020001D0020FC1B00204D
:105D4000241D00203C1D00204C1D002004000020CC
:105D5000581D0020080C00200C00002048180020CE
:105D6000F81C0020180C00201F1E00201C0C002016
:105D7000580C0020221D00208FC2753C480C0020CA
:105D80002C0C0020204605F019FF274B1968FAF764
:105D900011FF05F097FEB0F5617FA8BF4FF4617069
:105DA000FAF732FB1EA3D3E90023FAF7BDFCFAF79A
:105DB000A3FD05F0C7FE044695F87600FAF7A6FEA7
:105DC0002146FAF7F7FE05F07DFE184B188003E038
:105DD000174B188058809880164A5379012B164B20
:105DE00007D0164819885A889B8801804280838092
:105DF00011E01349B3F90420B1F9000002EB4000AF
:105E0000032290FBF2F080B20C4A088019885B886C
:105E100090801180538007B0BDE8F08FAFF3008011
:105E2000A2EB0FE5DD169640541D0020480C002023
:105E30003C1D002048180020241D0020240C0020B8
:105E4000380C0020AFF3008010B5054C00202188ED
:105E5000FCF770F861880120BDE81040FCF76AB8D3
:105E60001800002010B5094C20600948016009495C
:105E700009480A60094A0A491360029B039A0360B1
:105E80000848049B0A60036010BD00BF640C00203A
:105E9000400D00203C0D00206C0C0020440D002023
:105EA000740C0020380D0020094B1A6802EBC00169
:105EB000CB79FF2B04D01BB1064830F8130004E067
:105EC0000728D4BF888840F2DC5000B2704700BF7A
:105ED000640C0020761E0020054B1A6802EBC000FF
:105EE00090F9063019420CBF01204FF0FF30704787
:105EF000640C002010B500244FF48040FDF782FAB6
:105F000008B1054B00E0054B1868054A8188A1528D
:105F10000234182CF0D110BD400D00203C0D0020A3
:105F20007C1D0020F8B53A4B3A4E0546187006EB3A
:105F3000C0000F46384C417820202160FDF762FAFE
:105F400008B101222260162D19D1002438590021F0
:105F5000FAF7C4FF28B14FF48040FDF753FA50BB65
:105F600025E02E4A3B1916190FCB86E80F002C4866
:105F7000103401784A1CC02C0270E7D1EBE716F808
:105F8000357006EBC506264BD6F804E01F70BEF14F
:105F9000000FE0D00024BC42DDDA204E200136188C
:105FA0000EEB00010FC9013486E80F00F3E7082D5E
:105FB0001C4B23D124E01A4F3F78012FF7D91A4CFC
:105FC00000261034BE42F2DA54F8100C4FF07C5127
:105FD000FAF7F0FD4FF07C5144F8100C54F8140C13
:105FE000FAF7E8FD4FF07C5144F8140C54F80C0C0F
:105FF000FAF7E0FD013644F80C0CE2E70E2D01D172
:10600000012000E000201874BDE8F840FFF772BFDF
:10601000680C0020B8FA0008480D0020780C002019
:10602000700C00201F1E0020800C0020F0B58C4654
:10603000461C002300224CF803201033C02BF9D15A
:106040000A4800EBC6014F6807B9F0BD0024074BB2
:1060500013F83620944208DA20010CEB00053918B9
:106060000FC9013485E80F00F1E7F0BDB8FA000868
:10607000284B10B5186800284AD027490A78531EC3
:10608000142B3DD8DFE803F00B3C3C24403C3C1C87
:106090003C3C3C3C3C2C3C3C3C3C3C242C001F48C5
:1060A00001684A7832B11E4900204989BDE8104094
:1060B000FBF740BF1B4B58780028F4D10146F5E7A9
:1060C000174C0020E188FBF735FF01202189EDE71F
:1060D000134C00202189FBF72DFF01206189E5E7A2
:1060E0000F4C0020E188FBF725FF01202189FBF7F9
:1060F00021FF02206189FBF71DFF0320A189D5E75D
:106100002020FDF77FF918B1BDE81040FFF79CBED5
:1061100010BD00BF480D0020680C0020440D002079
:10612000180000201F1E002010B50024064B187810
:10613000A04208D90549204631F814100134FBF774
:10614000EDFEE4B2F2E710BD700C0020641D0020EB
:10615000064B1A780023D9B2914204D2044921F89F
:1061600013000133F7E7FFF7DFBF00BF700C00201B
:10617000641D00202DE9F74FA34B187803280FD991
:10618000A249A34CB1F904206FF06305002AB8BFFF
:106190005242A91AB4F904006432FDF74DFBA08005
:1061A000994A1678012E1DD89A4E3478651E9A4C5D
:1061B000142D00F2C981DFE815F0A400C701C70162
:1061C0007B00B300C701C7015A01C701C701C7015E
:1061D000C701C701D000C701C701C701C701C70177
:1061E0005F00A1018D488A4B884F0168B7F806B05F
:1061F000B3F800805F88B3F904A0894C01910025B1
:106200001034B542D0D20FFA8BF0FAF77FFC54F875
:10621000101CFAF7CFFC814638B2FAF777FC54F835
:10622000081CFAF7C7FC01464846FAF7BBFB814653
:106230000FFA88F0FAF76AFC54F80C1CFAF7BAFC6B
:1062400001464846FAF7AEFB019A814692F90000F2
:1062500041420AFB01F0FAF759FC54F8041CFAF722
:10626000A9FC01464846FAF79DFBFAF769FE6D4B1B
:1062700023F815000135C3E701210420FFF72CFEA8
:10628000634D654C6E88704387B204202781FFF709
:106290000BFE3818208101210520FFF71DFE2B88F9
:1062A000584385B205206581FFF7FEFD2B1826E0D7
:1062B00002210420FFF710FE554C0121A6887043EF
:1062C00087B20420FFF708FE6588534C00FB057277
:1062D000042097B2FFF7E8FD38182081022105203D
:1062E000FFF7FAFD7043012186B20520FFF7F4FDA8
:1062F00000FB056105208DB2FFF7D6FD2B186381E9
:1063000022E101210520FFF7E7FD414A424E97882F
:10631000784384B20520FFF7C7FD2018708113E190
:10632000414900200D68FFF7BFFD404F95F9063049
:10633000B7F902607343322693FBF6F2801820808F
:106340000120FFF7B1FD95F90E10B7F90050694330
:1063500091FBF6F3C7186780F6E03549354E4A7869
:10636000376812B9B888E08108E0284C3988B4F958
:1063700006007A88FDF760FA274BD881264D2E4F0C
:10638000E989284A3E681180347854B3264D0220AA
:10639000FFF78AFD2B68B3F91010B3F91220FDF74F
:1063A0004BFA2649264B0A68198854890EB2201ADE
:1063B00002B2964203DA3E683278511803E003DDF8
:1063C0003F683878091A19802D681D4F95F91630E5
:1063D000B7F90000642143430F4A93FBF1F6A41977
:1063E0009480134D0C4BAF7A67B1084801880E4A70
:1063F000D9801981868817685E814488064D9C8102
:1064000003241FE00248F1E7700C0020461E002024
:10641000121D0020680C002018000020440D0020F0
:10642000780C0020641D0020640C0020580C002013
:106430001F1E00203C0D00206C0C0020740C00205E
:10644000620C002007EBC40393F90600B5F90610AF
:106450006426414391FBF6F6EE802046FFF724FDCB
:1064600001343218EA800235072CEBD16CE0A54FDD
:10647000A54B78781E6810B9B588E58108E0A34976
:106480007288B1F906003188FDF7D6F9A04AD081AB
:106490009F4C9C4B9F48E7899E7A078001210320EF
:1064A0001EB1FFF719FD994D02E0FFF715FD9A4D5A
:1064B0006E880221704387B20320FFF70DFD2D88FF
:1064C00000FB05710420E1800121FFF705FD704309
:1064D000022186B20420FFF7FFFC00FB05620320C7
:1064E0002281FFF7E1FC8A4CE388C018E080042099
:1064F000FFF7DAFC2789C519258125E0864A0324A0
:10650000978802212046FFF7E7FC7843012186B2F5
:106510002046FFF7E1FC804DC4F10603590835F829
:1065200011207B4D00FB026086B225F814602046E6
:10653000FFF7BAFC331825F814300134072CE0D1EA
:10654000724F744AF98811802020FCF75BFF002805
:1065500045D00020FFF7A8FC6D4F0546388001208C
:10656000FFF7A2FC6D4978800B7A002B37D06C4A7C
:106570006C4B14686C4A267806F00201CCB2D4B198
:106580001468B3F9001094F90E2094F906404A43B8
:10659000322192FBF1F6B3F90230B2B26642734394
:1065A0006FF0310493FBF4F69419651993FBF1F144
:1065B0003D80561811E01168B3F9026091F9064068
:1065C0003222664396FBF2F42D193D8091F90E10AC
:1065D000B3F900304B4393FBF2F680197880002624
:1065E000514F4B4D3B68A85F03EB860233F92610F1
:1065F000B2F90220FDF720F9A8530236102EEFD190
:10660000474C2168087800F00407FBB22BB9414AD7
:10661000464C1688277801231CE0454D2E780E2E17
:106620000AD0082E08D0434A02EBC604617800293C
:1066300014BF0225002500E0042500263E4F7019F6
:1066400007EB4603C0B219890136FBF773FC042E31
:10665000F4D1DCE7BB4209D22E4C36B234F9131028
:106660000133B142A8BF0E46B6B2F3E70024274675
:106670002E490878874272D2234D31B22B685A884E
:10668000914204DD2348951B235AEA1822524FF405
:106690008040FCF7B7FE1F4DC0B1284A264B10685A
:1066A000B3F906104389184A9942254905DD09685E
:1066B0001268285F4988528804E012680B68285FD6
:1066C00091881A88FDF7B8F828533EE0DFF8388043
:1066D000285FD8F8003005EB040919885A88FDF7BF
:1066E000ABF8164A144913682853B1F90600998982
:1066F00088422ADA1020FCF785FED8F8002008BB73
:10670000108820E01F1E00203C0D0020461E0020A7
:1067100018000020641D0020121D0020301E0020E3
:10672000380D0020580C0020640C0020700C002054
:10673000680C0020B8FA0008761E0020740C0020B7
:10674000400D00209088A9F80000064843781BB946
:1067500005490648625A22520137023488E7BDE8EB
:10676000FE8F00BF1F1E00207C1D0020641D002026
:10677000024B1868003018BF01207047480D0020F8
:1067800044F25063984203DDA0F50C40A0387047F6
:1067900003498842BCBF00F50C40A030704700BFE1
:1067A000B0B9FFFF10B5FAF7B1F900210446FAF7C6
:1067B000BDFB08B1204601E004F100400549FAF7AD
:1067C000ADFA0549FAF7F6F905F048F9034B1860F8
:1067D00010BD00BF8096184B35FA8E3C2800002073
:1067E00010B5044C002320702361FEF72FFC60617C
:1067F00010BD00BFBC1D0020F8B51D4614460E4656
:10680000FAF784F96968FAF7D5F93146FAF7D2F957
:106810002168FAF7C7F82060FAF792FBED6807469F
:1068200005F10040FAF78CFB06462846FAF788FB8C
:10683000314602463846FCF7FFFFFAF767F9206059
:10684000FAF77EFBF8BD0000F8B5101A0C461F469B
:10685000FAF75CF90546381BFAF758F9174B079E0B
:106860001968FAF7A7F9294604462846FAF7A2F963
:10687000214607462046FAF79DF901463846FAF7C1
:1068800091F805F0EDF90E49FAF794F9FAF77EFB65
:1068900006990860214605F1004005F0DFF9094935
:1068A000FAF788F90849FAF77DF8FAF749FB002862
:1068B000BCBF00F50C40A0303060F8BD28000020BF
:1068C0002C7D8E3FA00CB34500A00C4610B50446AD
:1068D000002003460D49CA5CA2B12E2A04D101331F
:1068E00094B1C91800220A55084A0A21D25C4843CB
:1068F000A2F13001092901D8303880180E2B02D8B6
:106900000133E7E710BD002010BD00BFEC0E0020F2
:106910002DE9F843224B074648681D68381A0C4693
:106920009146FAF7F3F82946FAF7F8F91D4920617C
:106930000A6880469078FAF7E5F8F9F777FD16A32C
:10694000D3E90023F9F7C6FD02460B46002016499D
:10695000F9F7EAFEF9F7D0FF2946FAF723F80146DE
:106960002846FAF7DBF9A668054631464046FAF7AD
:1069700017F801462846FAF71DF901463046FAF79E
:1069800011F8D9F8081020616760A060FAF712F9D1
:10699000FAF7D6FABDE8F883182D4454FB211940C4
:1069A000180F0020D00E00200000F03FAFF3008051
:1069B000014B1860704700BFD00E0020F8B52D4B7A
:1069C000187810B1012850D10AE02B4B2B4A587887
:1069D0002B4B02EB001149681868FEF705FB41E0FC
:1069E000274D2868FEF705FB00283ED0224C217871
:1069F000264601291ED1FEF729FB06466069321A98
:106A0000632A35D92169042912D81C4F286807EB5D
:106A100001135968FEF7E8FA607807EB0017B968C8
:106A20002868FEF7CCFA22696661511C21611CE0DE
:106A3000022018E022693AB96478104B286803EB09
:106A400004114968FEF7D0FA33690B4C8B2B09D837
:106A50000C4A0B48D15C0068FEF7ACFA21694B1C6C
:106A6000236102E00320FFF7BBFE034A00205060D1
:106A7000F8BD00BFFB0E0020BC1D002038FF000841
:106A8000CC0E0020AAFE000810B50B4CE37A8BB1A7
:106A90000A48017804290DD9094A0A4B106851683F
:106AA00018605960FFF77EFE0748084B02880121F5
:106AB0001A80217310BD00BF1F1E00200C1E002075
:106AC000F41D0020D81D0020221D0020DC0E002017
:106AD000002370B51C460F48002119521420604352
:106AE0000D4A0E4E0E4D9952002232505953351810
:106AF0000C4E6960AA60325035180B4E0134696043
:106B0000AA6002333518022C32506960AA60E2D1C3
:106B100070BD00BFA81D0020FC0E0020C80D002085
:106B2000AE1D0020780D0020280F002070B504460F
:106B30000079F9F7E7FF1E49FAF7F0F81D4D1E4EF0
:106B40002860A07BF9F7DEFF1949FAF7E7F8EE6055
:106B500068606079F9F7D6FF1849FAF7DFF8184D41
:106B60002860E07BF9F7CEFF1149FAF7D7F86860A3
:106B7000607EF9F7C7FF1349FAF7D0F8EE60A86016
:106B8000A079F9F7BFFF0D49FAF7C8F80E4D286054
:106B9000207CF9F7B7FF0649FAF7C0F86860A07ED5
:106BA000F9F7B0FF0749FAF7B9F8EE60A86070BDD1
:106BB0000000C842B80E00200000FA440000204146
:106BC000080F002000007A44B40D00202DE9F341A5
:106BD0001A4F0E461A491B4D3A701B4A0860002096
:106BE0001360DDF82080FFF7FBFD6E70FEF72EFAD4
:106BF000A860387800246C60A0420CBF01250325F2
:106C00004046FFF793FF114B214603EB0616009415
:106C1000102072682B4601F0BBFF0D49086030B9A7
:106C20004FF4807002B0BDE8F041FCF76BBD01206D
:106C300002B0BDE8F041FFF7D3BD00BFFB0E00205E
:106C4000840F0020BC1D0020D00E002038FF00085B
:106C5000CC0E002073B51D4B1D78032D32D12020A2
:106C600001F066FF1A4E044638B102F06DF8316843
:106C70002046C968FEF7B8F909E03268009021465D
:106C80002020D2682B4601F083FF0446E0B1114D6D
:106C90002868FEF79FF930B12868FEF7A0F9014691
:106CA0002046FEF787F92046FEF794F90028EED03B
:106CB000084806682046FEF792F901463046FEF77E
:106CC00079F9E4E7022000E028467CBDBC1D0020E5
:106CD000840F0020CC0E0020F7B50368164C174D2A
:106CE00023600968164E61600068FFF75BFD94E859
:106CF0000C0014480196009095E80300FFF7A4FDEE
:106D00006B68114A61683668C81A1660F9F7FEFEAA
:106D10000E4A0F4F1168F9F74DFFFAF711F929687C
:106D2000786020680B4A431A0B483B600168166084
:106D30000A4BCA881A80FEBDE40E0020F41D002014
:106D4000580F0020000F0020E00E00202800002037
:106D5000880F0020680F0020D00E00207A0F00203E
:106D6000264BF0B51D68024600F110011678144656
:106D7000AB195B78013203F00403DBB263B18A42E2
:106D8000F4D10020F0BD13B10A225343DBB210F856
:106D9000011B30395B18DBB2211A0229F3DC002118
:106DA000844209D911B10A225143C9B210F8012B0A
:106DB000303A8918C9B2F3E72E2E11D101340420DC
:106DC00000220A2672432678AF197F7807F004075D
:106DD000FFB217B1303A921901340138F1D100E015
:106DE0000022074C6420614300FB02110624054881
:106DF000B1FBF4F200FB0320F0BD00BF98010020BE
:106E000040420F00809698002DE9F04F9A4B8BB0CE
:106E10001868B8B9994C21784A1E032A00F2658592
:106E2000DFE812F0F704F70442052C052068FEF7AE
:106E3000D6F8934904460B78012B00F0DF8008D385
:106E4000022B06D08C4C2068FEF7C4F80028EDD148
:106E5000E0E7242C07D18B4B8B4A8C4C0021197016
:106E600011702170C5E02C2C02D02A2C40F08280B9
:106E7000854D844A2978864B157800205854854AD8
:106E8000B5B918781570472868D15978502965D157
:106E90009878472840F01785D978472940F013851E
:106EA0001B79412B40F00F850120107000F00BBDC5
:106EB000117801293AD1022D05D11846FFF750FF6C
:106EC000754908604AE0032D07D11978532945D147
:106ED000714802685342036040E0042D05D1184612
:106EE000FFF73EFF6C4B586038E0052D07D11B784B
:106EF000572B33D168494A68504248602EE0062D2E
:106F000007D119786548302994BF00210121C17249
:106F100024E0072D04D1FFF7D9FC614A10701DE071
:106F2000092D1BD1FFF7D2FC5E4B16E0022915D1CB
:106F3000072D0CD10120FFF7C9FC41F21842504344
:106F40004FF47A71584BB0FBF1F0188006E0082D31
:106F500004D10120FFF7BAFC544B1880494B4A4931
:106F6000013500202A2C1D70087039D150480124A9
:106F700004703EE00D2C4E4A01D00A2C26D1147824
:106F8000FCB1434C21786478A1F13000C3B2092BE5
:106F900084BFA1F13703DBB2A4F1300003F00F028C
:106FA000C3B21101092B84BFA4F13703DBB2374C04
:106FB00003F00F0289182078CBB2C21A514251EB6C
:106FC00002043B4B002018707CB912E02E490B786C
:106FD0000E2B03D82E48C45401330B70127842B9DB
:106FE0002A4B1A7854401C7003E02A4A1078012872
:106FF00000D00020C00700F1338123E72D4B002291
:10700000197808293FF61EAFDFE801F00A051119CB
:1070100027607C96A000622801D1022105E01A7049
:10702000B52C7FF40FAF1C78611C19700AE7224958
:10703000224A03261E7008701070214B0BE01F4E71
:107040000421197032781E4BA1181878CAB2101892
:1070500018701C4B32701C70F4E605211970174B28
:10706000174E1A783078A118CAB210183070164E20
:107070001A703480E6E600BFCC0E0020BC1D002054
:10708000FB0E0020750D0020790F0020A00D0020C0
:10709000EC0E0020C40D0020F41D00201F1E002057
:1070A0000C1E0020A61D0020B21D0020640F002031
:1070B000910F0020D90E00206C0F0020C80E002078
:1070C000DA0E00206D0F0020B20D00206C4906265C
:1070D0001E700A786B4BA6181878F2B21018187048
:1070E000694B0A70198801EB0424A6B2B6F5007F3B
:1070F00001D81E8003E000221A80644B1A7000241D
:10710000634983E35E495F4E0A783078A318DAB2A8
:10711000101830705E4E0A7033885B4AC72B98BFD8
:107120005C49108898BFCC545C1CA1B28842318065
:107130007FF488AE072107E0514808261E700378C7
:10714000A3423FF47FAE0021504B6EE74D4E1A70C4
:10715000337883427FF476AE4F4C207806283BD0BC
:1071600005D8022813D003287FF46CAE23E0122840
:1071700047D030287FF466AE464A484C1679454AD7
:10718000102E88BF102626702178002347E0414C3E
:10719000434E6368A06821697360424B4FF47A7272
:1071A0003060414C91FBF2F6187840492680C87255
:1071B00001223F4923E037494A7912F0010004D007
:1071C0000E79F41E634253EB040036490870002820
:1071D00039D1364AD07236E02E4EF47A14F00101DD
:1071E00004D0B07AC21E534253EB02012D4E3170CF
:1071F00009B92E4CE17227482E4990F82F200A70C9
:1072000021E024482C498669426942F210742B4BD4
:1072100096FBF4F00A80188001222949EFE70C322E
:107220008B4210DA12F8046C264812F8034C1E54F4
:10723000254E26489C5512F8014C16781C54244CB7
:107240001E550133EBE71A490A78002A3FF4FAADDC
:107250001B4B1E78002E3FF4F5AD00240C701C7003
:107260001C4CA068E060FDF7F1FEA060202000F05B
:107270004DFC19490A78012A30D100232FE000BFC4
:10728000C80E0020DA0E0020B20D0020D90E00201A
:10729000660F0020F00D00206D0F00200D1E002055
:1072A000F41D0020780F0020A61D00201F1E0020C6
:1072B000D80E00200C1E0020B21D0020640F0020FC
:1072C0006E0F0020951D0020E21D0020FC1D0020F7
:1072D0000E1E0020BC1D0020800F002001230B701B
:1072E0000C787E497E48CA7AC480002A3FF4AAAD51
:1072F0007C4B1C78042C7FF6A5AD4F7807B90F7333
:107300000D7B15B90FB1FFF7BFFB774E0521307824
:10731000764F421C92FBF1F301FB13243470744E40
:1073200097F800C0734D06EB84020023724873493E
:107330001C58DFF814E2724E5C5094FBFEF103EB34
:10734000000A06FB01406F4F42F21074DFF8FC9117
:10735000D95190FBF4F71668BCB253F8097010606D
:10736000C6EB07084044052643F8090090FBF6F0F9
:107370000EFB01016448BCF1010F25F8024F1950C2
:1073800005D1023CB4F5797F98BFCAF800100433E8
:107390001432082BCAD1FDF759FE5C4D5C4C2A68AB
:1073A000801AF9F7AFFB5B49F9F7B8FC2060FDF7ED
:1073B0004DFE286025684FF07E512846F9F798FD6C
:1073C00008B94FF07E55256006A907AC4A48524BD4
:1073D0000194009103C80CCBFFF736FA069A642398
:1073E0004E49B2FBF3F00880079A3C4892FBF3F356
:1073F0004B4C027B23800AB90A80228049490C78D1
:10740000002C36D0424F4FF07E503968F9F786FC99
:10741000454D394E2B6804463068C01AF9F776FBA3
:107420002146F9F7C7FBF9F78BFD726869683F4D94
:107430000746501AF9F76AFB2968F9F7BBFB2146A2
:10744000F9F7B8FBF9F77CFD04B239480225B0F929
:1074500002303FB2E21892FBF5F1B0F900208BB296
:10746000B918344C91FBF5F291B2638021804380CE
:1074700001802C4B0120204C1870184B61682A4A5F
:1074800020681C7A516010601CB9DA79002A3FF438
:10749000D9AC294E294D2A4C01960095164F94E8F7
:1074A0000C00FFF7D1F961687868264E081AF9F7E1
:1074B0002DFB1E4B1968F9F77DFBF9F741FD706054
:1074C0000A48226890F900303C68012BC4EB0201A5
:1074D00031603DD0022B7FF4B5ACA0E01F1E002030
:1074E000DA1C00200C1E0020900F0020740D0020DC
:1074F0004C0D0020020F0020F41D0020700F002012
:10750000806967FF1C0F0020A80D0020D40E00200A
:10751000180F002000007A44D81D0020D61D00203E
:10752000E01D00206F0F0020500F002028000020D9
:107530007C0F0020240F0020580F0020000F002097
:10754000E40E0020880F0020809698005C0F002039
:10755000002634463546DFF818C3AF4F5CF825B037
:10756000CDF80CC05846F9F7D1FA3968F9F722FB83
:10757000F9F7E6FCDFF8DC92A84934F80920DFF8D7
:10758000DC82801A83B21FB2635238460497A44F3C
:10759000F9F7BCFA3968F9F70DFBF9F7D1FC4FF0B0
:1075A000140A0AFB058A82B29E4B04981968059258
:1075B0003B4658445246FFF71FF90599DFF8B4B22D
:1075C000DDF80CC00A1824F80B205CF825005146A1
:1075D0003A46FFF79DF994494FF4FA62FCF72CF90B
:1075E00034F8093034F80B20313399B2622998BF4E
:1075F0000020801883B224F80B308C4940F6B83252
:1076000018B2FCF719F958F80610894A01352BF819
:107610000400B15002341436022D9CD112E4854F7F
:107620002D683E686C08B6F90820A24228BF2246A1
:10763000814C97B2268839B230B2814209DD794B4C
:107640007E491868F9F7B6FAF9F77AFC8719BFB2DC
:1076500027807B4A7B4E14683168661A3046FFF7F4
:107660008FF80028D8BF404241F293139842CCBF14
:107670000020012050B33046F9F748FA7249F9F773
:1076800099FA04F05FFA06462846F9F73BFA0146F4
:107690003046F9F78FFAF9F753FC6C4A63491080CA
:1076A00000B240F6B832FCF7C7F8201848F6A044FC
:1076B000A04203DDA0F50C40A03804E00028BCBFC8
:1076C00000F50C40A0306249086001E0604D2C607C
:1076D0005F4B1D68C5F50C502830F9F717FA5A4969
:1076E000F9F768FA064604F0B9F90990304604F053
:1076F00029FA002508902C462E4638B2F9F706FAEA
:1077000008AA52F82610F9F755FA80465148DFF8D2
:107710000C91005FF9F7FAF901464046F9F740F994
:10772000F9F70EFC4FF47A7224F809004A4900B2C6
:10773000FCF782F881B20BB2DFF83C8124F8091023
:1077400018460493F9F7E2F9D8F80010F9F732FA7D
:10775000F9F7F6FBDFF8D8A04FF0140B0BFB06ABE4
:10776000049A30491FFA80FC0968434610465A467D
:10777000CDF80CC0FFF740F842460346594639F9A8
:1077800004000493FFF7C4F8049ADDF80C80801815
:1077900008EB000CDFF8DC801FFA8CF124F80810ED
:1077A00008B240F6B8322149FCF746F855F80A20ED
:1077B0002A4B013628F80400EA5002341435022E10
:1077C0009BD11C480368197931B1214A642014689F
:1077D000234A94FBF0F11180224C1B8820689842C8
:1077E0000ED91749174B0A681C68101BFEF7C8FF13
:1077F00042F210710028B8BF404288427FF722ABA6
:10780000194B1A4A01201C88154910700C80FFF78B
:1078100019BBFFF7D3F868E0B80E0020A20D0020D6
:10782000080F0020180F002030F8FFFF48F4FFFF7A
:10783000280F0020D00E00207A0F00200000C84240
:10784000580F0020680F0020D3023739B00D0020F8
:10785000E00E0020240F002018FCFFFF780D002010
:10786000101D0020000F0020DC0E0020740D0020F1
:10787000880F0020AE1D0020B40D002062686078E3
:10788000531C411CCAB263600523B2FBF3F003FB37
:1078900010216170FDF7DAFB154AA060154800233E
:1078A000C372137001200BE0FDF7D0FBA36840F614
:1078B000C411C01A884218D9202000F02FF90420E2
:1078C000FEF78EFF11E00C498A78522A7FF446AB0E
:1078D000CB784D2B7FF442AB087943287FF43EAB45
:1078E000064A02211170FFF739BB0BB0BDE8F08FDB
:1078F0000C1E00201F1E0020EC0E0020C40D0020D6
:107900003D4B2DE9F047B3F90000F9F7FFF83B498B
:10791000F9F750F9044604F015F90646204604F03C
:107920009DF8DFF8EC900546D9F80000344F90F848
:107930000380B8F1000F2BD0324CB7F90210B4F825
:1079400002A00FFA8AF2881AFEF71AFFC8F10001A6
:107950004246FBF771FFB4F8008000EB0A03B7F969
:1079600000000FFA88F7C01B6380FEF709FFD9F803
:107970000010CA785142FBF75FFF00EB080297B294
:107980002780B4F90200F9F7C1F8804638B206E062
:10799000B7F90200F9F7BAF88046B7F90000F9F72D
:1079A000B5F8294607464046F9F704F931468146BD
:1079B0003846F9F7FFF801464846F8F7F1FF124953
:1079C000F9F7ACF9F9F7BCFA104C31462080404683
:1079D000F9F7F0F8294606463846F9F7EBF801467C
:1079E0003046F8F7DFFF0849F9F798F9F9F7A8FAF0
:1079F0006080BDE8F08700BF221D002035FA8E3C74
:107A0000AE1D0020A81D002000002041FC0E00201B
:107A1000D00E002038B5254CE37A2246002B3ED00C
:107A20002348017804293AD92248817A79B1E17949
:107A3000002939D12048214B012221721970011DE2
:107A4000E271FFF749F91E490220087038BDC37A78
:107A5000E171C3B11B4A1068408900F06DF890B124
:107A6000237A002B20D115481749037017480A685C
:107A70004B680125011D026043602572FFF72CF958
:107A80000F48057038BD0D48084B02780021197267
:107A900052B901210170BDE83840FFF719B8002341
:107AA000D3711372064A137038BD00BF1F1E002029
:107AB0000C1E0020301E0020D81D00202C000020AD
:107AC000740D0020D00E0020F41D0020B41D0020F5
:107AD000074B1A68811A002908DB064A1178042925
:107AE00004D900F5123000F5F8721A60704700BF33
:107AF000940F00200C1E0020034B196808420CBF95
:107B000000200120704700BF980F0020024B1A6828
:107B100010431860704700BF980F0020024B1A688E
:107B200022EA000018607047980F0020014B186887
:107B3000704700BF980F0020094BB3F90020002ABE
:107B4000B8BF5242824209DAB3F902100029B8BF25
:107B500049428142ACBF002001207047002070479D
:107B6000461E002010B544780078002303FB03F183
:107B70001939614301F6C4115943414340F6C41217
:107B800091FBF2F1034A22F813100133072BEDD1D8
:107B900010BD00BF661E00202DE9F04384780A273F
:107BA0006743C678C4F1640C1A4D5FFA8CFCC6F1C9
:107BB000640800231A1B12B2002A04DCB8BF204656
:107BC00002DB012000E0604602FB02F9404309FBB2
:107BD00006F999FBF0F0404442434FF00A0992FB4A
:107BE000F9F2B81882B26A800888B1F8029012B22D
:107BF000C0EB090902FB09F20A334FF47A7992FBD0
:107C0000F9F29BB28018782B25F8020FD2D1BDE88B
:107C1000F08300BF4C1E002008B5037A042B18D84F
:107C2000DFE803F00303080D12000D490D4A00F0D0
:107C3000CFFA0DE00A490B4A00F03CF908E0084988
:107C4000084A00F0FBF903E00549064A00F0E6F8AF
:107C500028B90820FBF756FD02480022026008BD43
:107C6000741E0020AC0F002010B50023044660896C
:107C70000F4A98520233242BF9D10E480160082094
:107C8000FBF7C0FB10B12046FFF7C6FF0120FBF752
:107C9000B9FB28B108480949BDE8104000F0CAB84E
:107CA0004FF40040FBF7AEFB0028F3D110BD00BF3E
:107CB000761E0020B00F0020741E0020AC0F0020A4
:107CC000037A042B0CD8DFE803F00303050709004F
:107CD00000F0B6BA00F01CB900F0CEB900F094B8CC
:107CE000002070472DE9F84F80464FF400708B4616
:107CF000FBF788FB20B12E4B186801680A69904792
:107D00000820FBF77FFB40B92A4C257805F10107D5
:107D1000FBB2237003F0030A01E04FF0000A0025D4
:107D2000254C4FEA4A0A2F462448026822B9B8F87F
:107D30000A20234BEA5233E018F807905846494688
:107D4000904706464FF40070FBF75CFB30B11849D2
:107D50000B6831461868C26948469047A6F2EE2182
:107D600088B240F2DC53984288BFB8F80A60082015
:107D7000FBF748FB10B112482E5211E024F80A60BC
:107D800022886188A3885018E288C11888180D4994
:107D900083B26B5218B20422094990FBF2F36B5282
:107DA000013702350834082FBED1BDE8F88F00BF77
:107DB000B00F0020B40F0020B60F0020AC0F002041
:107DC000761E00209C0F0020F8B505460F46441E85
:107DD00014F8011F49B1054E304606F037FD002862
:107DE000F6D0861B631BBB55F2E7F8BD88FF000881
:107DF000014B33F811007047761E0020014B012221
:107E00001A707047F60F0020034B187810B100224B
:107E10001A700120704700BFF60F00200AB1024B14
:107E200013600120704700BFF17D00080846FAF793
:107E300087B90000024B0B6008210170704700BF3A
:107E40002D7E0008034B53F82100410801F577729D
:107E500090B27047FC0F002038B50446FDF7DCF8FF
:107E6000104B40F6C4111A68821A8A421A460E4B09
:107E700001D9002119701B7810600BB90F2C10D19B
:107E80000A4800210170084A4BB1094D182B1D44C6
:107E900005F8014C03D101230370117038BD013383
:107EA000137038BDF80F00201C1000203610002081
:107EB0001D10002073B50023044600930E460523D1
:107EC0000E49154608200E4A00F062FE62890D4BED
:107ED0000D49A2F57774640008601C605C609C60CA
:107EE000DC601C615C619C61DC610DB1074929604B
:107EF00008220030327018BF01207CBD597E000876
:107F0000A0860100FC0F002038100020457E0008EC
:107F1000264970B50878002847D0254B987DC0F3D6
:107F2000C00000283FD15D781C78224A05F0070682
:107F300044EA062414609C7804F03F06760146EA81
:107F4000D5055560DE78B50045EA94151C7904F036
:107F5000010645EA862595605D7905F00F06F60174
:107F600046EA5404D4609C7904F07F06360146EA60
:107F700015151561DE79750045EAD4141D7A05F0F2
:107F8000030644EA462454615C7A04F01F06B601F5
:107F900046EA950595619B7A0870DB0043EA541424
:107FA000D461012070BD0020087070BD3610002023
:107FB0001D100020FC0F0020024B53F82100C0F3DD
:107FC000CF0070476410002010B50446FDF724F878
:107FD000154B1A68811AB1F57A6F1A46134B01D9FD
:107FE000002119701060187820B9A82C1AD1104BF4
:107FF000187006E0022802D10E4A147001E014281D
:1080000001D80D490C540B490130C3B20878074A16
:108010004100481D8342137004D1002304491370AA
:1080200001220A7010BD00BF5410002084100020EF
:1080300058100020601000203C10002037B50023AD
:1080400000930D461446094908204FF4E1320123FC
:1080500000F09EFD064908600CB1064A2260082324
:1080600000302B7018BF01203EBD00BFC97F000843
:108070005C100020B97F0008124B10B51A780AB9BD
:10808000002010BD1049002018704B78012BF7D14B
:108090000E480278082A01D90821017001780C4A9B
:1080A0000023D8B2023288420AD212F8010C12F828
:1080B000024C40EA0424074840F823400133F0E72B
:1080C000012010BD581000203C100020601000203E
:1080D0003F10002064100020114B012210B51A70CF
:1080E0000446FCF799FF0F4A0146106811600B1A0D
:1080F0000D4841F288318B4203600C4B01D90022BC
:108100001A7018780A49E4B20F280C5403D10949AF
:108110000120087010BD054A431C137010BD00BF3C
:10812000901000208C10002094100020851000205A
:1081300099100020881000201E4B2DE9F0411A787C
:108140001AB31D4C1D4D2678077895F800C0022300
:108150001B4A03F10108D45C44FA06F404F00F044E
:10816000E5B2BD420BD20B2D09D8D55C12F8082020
:1081700005EA0C0502EB0525124A42F824500233A9
:10818000102BE5D10B4B00221A70007888420ED9D3
:108190000D4A107860B10D4B0A481A7850F821103A
:1081A00002B1490801F5777398B2BDE8F08100206B
:1081B000BDE8F08188100020861000209810002073
:1081C00099100020AC100020901000208710002093
:1081D00013B5037A14465BB1012B13D1124A032065
:1081E0001070124A07201070114803700C2308E029
:1081F0000D4A022010700D4A032010700C480370C5
:1082000007230B70002100914FF4E1320820094947
:10821000012300F0BDFC084A10600CB1074B23603D
:10822000003018BF01201CBD8610002098100020CF
:1082300087100020D9800008DC1000203981000858
:10824000014B1878704700BF88100020014B186060
:10825000704700BFE4100020034B18680178D1F18B
:10826000010038BF00207047E4100020034B18685D
:1082700001784A1E534253EB02007047E41000207D
:1082800008B54FF40060FBF7BDF820B10420BDE84D
:10829000084000F039BC08BD08B50420012100F0F9
:1082A0003BFC60B1074B1868417811B10648037D6B
:1082B00001E0064A5378181C18BF012008BD0120B0
:1082C00008BD00BFE4100020301E00201F1E00204B
:1082D00008B5FFF7C1FF08B100F08CF8FFF7C6FF43
:1082E00018B1BDE8084000F073BA08BD0F4B10B5D7
:1082F0001878D0B1FFF7D0FF0D4904460A788242C2
:1083000013D070B1FFF7A8FF18B10A4B186800F03E
:1083100089F8FFF7ABFF30B10648006800F070FA4B
:1083200001E0FFF7D5FF02490C7010BDE8100020F6
:10833000E0100020E410002008B5FFF7A1FF034B78
:108340001870BDE80840FFF7D1BF00BFE81000205B
:1083500008B5094B187870B1FFF79EFF58B1FFF7C9
:108360007BFF08B100F0A0F8FFF780FF18B1BDE86F
:10837000084000F079BA08BDE810002038B5064C76
:1083800005465E212068FCF715FE20682946BDE8F9
:108390003840FCF70FBE00BFF8100020024B5E21F2
:1083A0001868FCF707BE00BFF810002010B50A4C93
:1083B0005E280146206805D15D21FCF7FBFD2068A1
:1083C0003E2105E05D2903D1FCF7F4FD20683D2145
:1083D000BDE81040FCF7EEBDF810002010B50446D3
:1083E000C0B2FFF7E3FFC4F30720BDE81040FFF77A
:1083F000DDBF000010B5084B084C19782068FCF769
:10840000FDFD074920680968FCF7EEFD206804219E
:10841000BDE8104000F000BCF1100020F810002072
:10842000EC10002037B50546042000F081FB154C08
:1084300001462060A0B14279134B81681A70134A3B
:1084400011604FF41651FCF7CFFD20680221FCF7B4
:10845000D5FD2068042103B0BDE8304000F086BBA4
:10846000AB784FF4165200930420022300F090FBE7
:10847000054942792060054B80680A70186003B096
:1084800030BD00BFF8100020F1100020EC100020DB
:1084900008B5044B1868FCF79DFDD0F1010038BF0A
:1084A000002008BDF81000202DE9F041FFF7F0FF93
:1084B000002800F04081FCF7C9FDA04B1A68811A22
:1084C0007C2940F2388118609D480478651C05704D
:1084D000002404F12406F0B2FFF750FF994B33F962
:1084E0001400F8F713FB984A05461088F8F70EFBBE
:1084F00001462846F8F712FC9449F8F75BFBF8F7B9
:108500001FFD013400B2FFF769FF032CE1D13020D9
:10851000FFF734FF8E49B1F90000FFF75FFFFFF767
:108520003DFF8748067816F0030629D1894D1020B3
:10853000FFF724FF2B68642493FBF4F210B2FFF7DB
:108540004DFF2120FFF71AFF296891FBF4F004FB8F
:10855000101484EAE473A3EBE47318B2FFF73EFF50
:108560001420FFF70BFF7C4AB2F90000FFF736FF3B
:108570001C20FFF703FF3046FFF730FFFFF70EFF29
:108580006F490878430740F0B080744D0220FFF730
:10859000F5FEB5F900300A2593FBF5F0FFF71EFF55
:1085A0000220FAF72FFF002847D06D4F6D4E387824
:1085B000347840F63401B4FBF0F26B4C4A43218826
:1085C0002A2391FBF0F800FB1810B2FBF3F24FEAFC
:1085D000001399B241EA022C1FFA8CFEC2F3032267
:1085E0004EEA02080620FFF7C9FE0FFA88F0FFF7EF
:1085F000F5FE20883F78431C9AB292FBF7F107FB07
:108600001120367820806E247443152394FBF3F4F4
:108610003A206427FFF7B2FEB4FBF7F63046FFF7C7
:10862000DDFE3B20FFF7AAFE07FB164291B24C1D70
:1086300094FBF5F000B2FFF7D1FE2020FFF75CFAC3
:10864000002850D0494C1320FFF798FE2568484F6A
:10865000002DB8BF6D4295FBF7F630B2FFF7BEFEB6
:108660001B20FFF78BFE23680A26002BB8BF5B4256
:1086700093FBF6F142F2107591FBF5F205FB121037
:1086800000B2FFF7ABFE2320FFF778FE2368002B34
:10869000ACBF4E205320FFF7A1FE1220FFF76EFE65
:1086A00061680029B8BF494291FBF7F210B2FFF7A9
:1086B00095FE1A20FFF762FE60680028B8BF4042AE
:1086C00090FBF6F696FBF5F305FB136108B2FFF796
:1086D00085FE2220FFF752FE6268002AACBF4520CB
:1086E0005720FFF77BFEFFF759FE15480378282B2C
:1086F00021D100240470FCF7A9FC4FF47A753C24C6
:10870000B0FBF5F61720FFF739FEB6FBF4F5B5FB25
:10871000F4F104FB1152100200B2FFF75FFE1820C3
:10872000FFF72CFE04FB156318B2FFF757FEBDE8F8
:10873000F041FFF733BEBDE8F08100BFF410002028
:10874000F01000204C1D00200400002000007A449E
:108750003C0C00204C0B0020221D0020D81C0020C7
:108760000100002044180020F2100020F41D002019
:10877000A0860100154B2DE9F04180460F46186890
:108780000221FCF73BFC00242646781E84420F4D54
:108790000DDA18F8041028688E190134FCF70AFC69
:1087A0004FF47A70B6B2FCF757FCE4B2EDE7F1B2E1
:1087B0002868FCF7FFFB4FF47A70FCF74DFC286843
:1087C0000121BDE8F041FCF719BC00BF2C110020CD
:1087D00010B5084B084C19782068FCF70FFC0749C6
:1087E00020680968FCF700FC20680421BDE81040FF
:1087F00000F012BA5E1100202C1100202811002078
:1088000013B5042000F094F9144C01462060A0B187
:108810004279134B81681A70124A11604FF49641E5
:10882000FCF7E2FB20680121FCF7E8FB206804214B
:1088300002B0BDE8104000F099B900904FF49642A4
:108840000123042000F0A4F9054B4279206005497A
:1088500080681A70086002B010BD00BF2C110020A3
:108860005E11002028110020F8B5544C2068FCF758
:10887000B1FB002800F0A0802068FCF7B0FB0546A3
:108880000520FCF7F4FB8A2D21D08E2DEDD14C4C28
:1088900000212E22204605F081F94A4A7C232370CC
:1088A0001378E0207D21E07084F82C1014204FF420
:1088B000FA71A37723754822782320766076618346
:1088C0006570628484F8243020462E2171E02020D7
:1088D000FFF712F90028C8D03B4C00212C2220467B
:1088E00005F05CF9A021E170384B39497C207D22EC
:1088F000207084F82B201878CA7A6570A076002A38
:1089000052D0344934480F686625FE0F97FBF0FCBF
:108910006672324E5FFA8CFC06FB0C7284F82950AA
:1089200006256A4342F21073B2FBF3FE03FB1E27D7
:108930004968277391FBF0F03F0AC0B26773CF0F0D
:1089400006FB00116943B1FBF3F5642203FB151329
:10895000E9B202FB0010010AE0732148217401888A
:108960005FFA8EFE63741B0A02FB0CECA374B1FB6E
:10897000F2F224235A4390B21A4A010A1388E07192
:108980002172180A1849207518480A8801884FEA88
:108990001C2EE374130A84F80AC084F80BE0A77352
:1089A0006275A375217702E0202384F829300648F8
:1089B0002C21FFF7DFFE58E7F8BD00BF2C11002087
:1089C0003011002044180020FC1000200C1E002054
:1089D0001F1E0020F41D0020A08601006079FEFF0C
:1089E000B21D0020D61D0020A61D0020E01D002085
:1089F00010B500230C245C430549DAB2615C814266
:108A000003D00133042BF5D11A46104610BD00BF28
:108A1000300000202DE9F84F07460023244A12F8C1
:108A2000130002EB4306B84205D00133062BF5D103
:108A30000020BDE8F88F1F4804210C221E4B05F0D2
:108A400043F900250C2068431A4A02EB000999F803
:108A500008100F4227D0125C0024184B2001195C2B
:108A60009B46914203D00134E4B2042CF5D14FEA85
:108A7000041A40200BEB0A08FAF7C4FC20B91BF8D3
:108A80000A20931E012B0ED9707840B90C4804704F
:108A9000C0F80880C0F80490C660BDE8F88F98F868
:108AA0000C100842F2D10135042DCBD1C0E700BF34
:108AB000DCFF000830000020C58A00089CFF000889
:108AC00060110020037A002023B15A1E01301340A8
:108AD000C0B2F9E70A7A22B1511E01330A40DBB273
:108AE000F9E7984294BF0020012070470023054910
:108AF000DAB2595C814203D00133092BF7D11A460F
:108B00001046704791FF000808B5C0B2FFF782FF1A
:108B1000003018BF012008BD10B50C46FFF77AFFE2
:108B200028B14368187A04420CBF0020012010BD10
:108B300000220D4B0C2101FB0233197A814211D026
:108B40000132D2B2042AF4D10022074B0C2101FBDE
:108B50000233197A014005D10132D2B2042AF4D18C
:108B600008467047586870473000002010B5002351
:108B7000064A0C2404FB03225468844203D00133C8
:108B8000042BF5D10022517210BD00BF300000202F
:108B90002DE9F04385B00391029280461E469DF870
:108BA0003040FFF737FF03990546029A48B38368C0
:108BB00090F800901F78032F23D8DFE807F0020514
:108BC0000C0E0094114801E0114800943346F9F767
:108BD0004DFD044609E0002000E001202346F9F79E
:108BE0002FFB31460446FCF709FA54B12771696836
:108BF00008484C6040F8294041462046FFF7B6FF40
:108C000000E00024204605B0BDE8F08300380140B4
:108C100000440040701100200023074A0C2101FB92
:108C200003225168814203D00133042BF5D1002285
:108C300000205072704700BF3000002010B50120A6
:108C4000FFF7E8FE08B9002010BD0220FFF7E2FEA2
:108C50000028F8D01020FFF7DDFE04464FF48070A6
:108C6000FAF7D0FB08B1002CEDD00820FFF7D2FEB8
:108C700004460820FAF7C6FB08B1002CE3D0042014
:108C8000FFF7C8FE04464FF40060FAF7BBFB08B1DB
:108C9000002CD8D0012010BD38B50D460024074B5C
:108CA000185DFFF7B7FE80680178A94204D002344E
:108CB0000C2CF4D1002038BD012038BDDCFF0008A9
:108CC000F8B505460020FFF793FE104E0C272B78D1
:108CD0000F4C07FB0060E15C01720120FFF788FE8A
:108CE00007FB00626878235C02201372FFF780FEA6
:108CF000AA7807FB0061A05C08720320FFF778FEEA
:108D0000EB7807FB0061E25C0A72F8BD30000020DE
:108D100091FF000838B5064C05462060FFF7D0FFEC
:108D2000284600F0FFFF2068BDE8384000F0E0BEB4
:108D300080110020034B187808B100F0E1BD01F06C
:108D40007BB800BF8411002010B504462046FCF714
:108D500050F918B90A20FCF78AF9F7E710BD0000AE
:108D6000232801D100F0CCBD044B19680A7D824252
:108D700002D10120FCF7FAB9704700BF8011002032
:108D800010B5441E14F8011F21B1034B1868FCF7FD
:108D900011F9F7E710BD00BFBC1100200148FFF733
:108DA000EFBF00BF6C01010810B50748FFF7E8FFEF
:108DB0000024064B06481A19E15852680C34FAF799
:108DC00065FEC02CF5D110BDAA010108880001087C
:108DD000C001010870B5FCF739F9244C244B4FF45D
:108DE0007A71B0FBF1F11A7822482378FAF74EFE37
:108DF000FEF79CFE05462048204902682048B2FB49
:108E0000F1F1FAF743FE00241E4B53F8241051B140
:108E1000012000FA04F0284202D01B48FAF736FE7F
:108E20000134E4B2F0E70220FEF766FE68B1174AAB
:108E3000174B1178174853F82110FAF727FE1648F8
:108E4000017A11B11548FAF721FE154C1548FFF7C4
:108E500097FF2488F8F746FE0246134821464FF450
:108E60006C73BDE87040FAF711BE00BF010000202E
:108E700044180020C80101087C01002040420F0076
:108E800006020108FC0F010824020108440B00201F
:108E90004801010828020108E81C002032020108EC
:108EA0000E0B0020980401083602010838B50C6842
:108EB0000546204605F0A6FD024628682146BDE885
:108EC000384005F0CFBD000037B5037904460D46A4
:108ED000052B34D8DFE803F003060A0D111481686E
:108EE00009782DE0806890F9001029E083681988DE
:108EF00026E08268B2F9001022E0816809681FE06C
:108F0000806869460068FAF7A7FE01461148FAF73B
:108F1000BDFDF5B1E068F7F7F9FD6946FAF79CFE8B
:108F200001460D48FAF7B2FD2069F7F7EFFD6946F3
:108F3000FAF792FE01460848FAF7A8FD09E0002179
:108F40000648FAF7A3FD25B10548E1682269FAF75A
:108F50009DFD3EBD2F0201082E0201086C02010892
:108F60006802010808B50648FFF70AFF054B1868B4
:108F7000FFF7EAFE0020BDE80840FCF7F7B800BFA5
:108F80006F020108BC11002008B50748FFF7F8FE82
:108F9000064B93F8AC03FAF7D7F9FAF7E5F9BDE811
:108FA0000840FFF7DFBF00BF7E020108481800201D
:108FB0007FB5044605F026FD082825D100231F496A
:108FC000E25C086885186E7806F00301022908BF84
:108FD000203AE2540133082BF1D10025665D184890
:108FE000314605F033FC28B101356019314605F0F2
:108FF0002DFC18B11348FFF7C3FE1DE0082DEDD17D
:1090000020461149FEF7E0FE1048FFF7B9FE0023A5
:109010000F4A04A9981890F808218818084A995C02
:109020000133082B00F80C1CF2D100208DF80C0045
:1090300001A90848FAF72AFD7FBD00BF980100206A
:1090400088FF00088802010850190020A8020108C2
:1090500048180020C301010808B5FDF7FBFD0228F0
:1090600001D0032804D10348BDE80840FFF788BEBB
:1090700008BD00BFBD0201082DE9F041054605F01D
:10908000C1FC0446FAF7D2FB064694B92A48FFF71A
:1090900077FE2A4951F8241049B1012202FA04F25C
:1090A000324202D02648FAF7F1FC0134F1E72548B4
:1090B00021E028462449224605F0D4FC58B923482B
:1090C000FFF75EFE224C54F8041F0029EFD01C4825
:1090D000FAF7DCFCF7E72B782D2B04D10135013CA6
:1090E0004FF0010801E04FF000080026134850F847
:1090F000267027B91748BDE8F041FFF741BE284662
:109100003946224605F0AEFCA0B9012000FA06F06F
:10911000B8F1000F03D0FAF7F5FA0F4802E0FAF7BA
:109120007BF90E48FFF72CFE0D483946BDE8F041AB
:10913000FAF7ACBC0136D9E7E3020108E8FF000802
:109140002402010898040108EF0D0108F602010845
:10915000E4FF00080B030108250301082F030108A1
:10916000C301010810B504460848FFF709FE084A84
:10917000084809490023036013700B70FCF7BAFE1E
:109180002046BDE81040FFF7FFBE00BF38030108CE
:1091900085110020B81100208411002008B5044872
:1091A000FFF7EEFDFAF740F9BDE80840FFF7DABE39
:1091B000500301082DE9F04389B0044605F022FC74
:1091C000C6B2002E6AD17A48FFF7DAFD794C2069E1
:1091D0000021F7F783FE38BB013677483146FAF7AE
:1091E00055FC206904A9FAF737FD01467348FAF7E0
:1091F0004DFC606904A9FAF72FFD01466F48FAF7A4
:1092000045FCA06904A9FAF727FD01466B48FAF767
:109210003DFCE06904A9FAF71FFD01466848FAF72A
:1092200035FC10340C2ED2D10025664C2F46A846B2
:109230004FF000091034B14514DA404654F8101CC0
:10924000F7F7B0FB54F80C1C80462846F7F7AAFB4A
:1092500054F8081C05463846F7F7A4FB09F1010944
:109260000746E7E75848CDF8048002950397FFF7D3
:1092700087FD002401A82358544923F00040F7F744
:1092800055FE5349534A0434002814BF104608467B
:10929000FFF776FD0C2CEDD14F4871E020464F4989
:1092A000052205F0DFFB38B9424B0022C11810300F
:1092B000C0280A61F8D177E020464949042205F028
:1092C000D1FB054620460DBB202105F0BFFA002842
:1092D0006AD0461C304605F095FB2C4607464148AF
:1092E00050F824500DB940484AE030462946FAB2B9
:1092F00005F0B8FB40B920463C49FCF797FE3C48D6
:109300002946FAF7C3FB47E00134E8E704F0FCFA2A
:10931000461E0B2E074643DC2046202105F096FA18
:10932000054640B1451C2846FAF7FEFC214B3F019B
:10933000D851012400E004462846202105F086FA91
:10934000054640B1451C2846FAF7EEFC19490134A0
:1093500001EB061250612846202105F077FA0546F8
:1093600040B1451C2846FAF7DFFC124B013403EBF1
:10937000061188612846202105F068FA18B91D48B1
:10938000FFF7FEFC10E00130FAF7CEFC094A032C8F
:1093900002EB0616F061F2D11748FFF70BFF03E06E
:1093A00016480C21FAF772FB09B0BDE8F08300BF44
:1093B00071030108481800209C030108A20301085A
:1093C000C30101085C180020A60301080AD7233C4A
:1093D0006D0301086903010898040108B503010839
:1093E000BB0301082C000108C00301085818002025
:1093F000D8030108EB030108D7060108250401087A
:10940000F8B5074605F0FEFA044638B91A491B4B71
:109410004A791B48511E53F8211028E03846194953
:10942000224605F01FFB60B91748FFF7A9FC174C4F
:1094300054F8041F19B11648FAF728FBF8E7154845
:1094400005E000250D4B53F8256026B91248BDE80C
:10945000F840FFF795BC38463146224605F002FB3E
:1094600001350028EED10448314645710B48BDE86E
:10947000F840FAF70BBB00BF481800202C00010889
:109480004D040108EF0D01086104010828000108DE
:109490002402010898040108C003010874040108AB
:1094A0002DE9F047064605F0ADFA054620B1012842
:1094B00019D133782A2B16D14748FFF761FC0024D5
:1094C00014266643454F4648F159FAF7DFFAB819B2
:1094D0002946FFF7F9FC01344248FFF751FC722C92
:1094E000EED1BDE8F08730463D2105F0AFF9002808
:1094F00057D0441C204604F007FA82462046FAF76B
:1095000013FC0027054614247C43DFF8D09054F860
:109510000980404605F076FA41460246304605F09D
:10952000A1FA002835D14C44E068F7F7EFFA01467C
:109530002846F7F7F1FC002829D02069F7F7E6FA6A
:1095400001462846F7F7DEFC002820D02079227952
:10955000052818BF5546052A0FD8DFE802F0030397
:109560000606090CA1680D7007E0A268158004E0EA
:10957000A068056001E0A1680D6041461A48FAF74D
:1095800085FA20460021BDE8F047FFF79DBC17484B
:1095900003E00137722FB6D11548BDE8F047FFF759
:1095A000EFBB0446142565430C4F314655F8078040
:1095B000404605F029FD50B109484146FAF766FAE0
:1095C00078190021FFF780FC0648FAF75FFA0134AA
:1095D000722CE7D1BDE8F087860401081C10010851
:1095E00060060108980401089B040108A60401080C
:1095F000CB04010810B50446204605F003FA10F02C
:10960000FF0F07D10B490C4891F8AC13BDE810408F
:10961000FAF73CBA204604F077F9022808D8054B3F
:10962000064C83F8AC03F9F79FFEFAF7BBF8E3E7C3
:1096300010BD00BF48180020E8040108D706010843
:1096400070B5044605F0DEF908B9204830E0204640
:109650001F4905F04FFE00242646254678B12CB15F
:10966000012C06D104F050F9064602E004F04CF952
:10967000054600201649013405F03CFEEEE70B2DAF
:1096800005D914480C21BDE87040FAF7FFB9012C48
:1096900008DC114A114832F915202946BDE870400E
:1096A000FAF7F4B9A6F57A73B3F57A7F04D90C48C2
:1096B000BDE87040FAF7EAB90A4829463246FAF797
:1096C000E5F9054820F8156070BD00BFFE040108EB
:1096D000A1060108380501087C1D00205E0501086F
:1096E000760501089805010838B5054605F08AF9A0
:1096F000C0B268B904461249124801EB4402B2F8FC
:10970000462021460134FAF7C1F9152CF3D138BDB2
:10971000284604F0F9F8142804460BDC20212846DA
:1097200005F094F804F0F0F8054B03EB4404A4F8BA
:10973000460038BD04481521BDE83840FAF7A6B9FF
:10974000FC1B0020B1050108BD0501082DE9F0430F
:10975000584885B0584CFAF799F95848FFF7C4FFB4
:109760006279574B511E574853F82110FAF78EF97A
:1097700020690021F7F7B2FB002858D1002526699F
:1097800000213046F7F7AAFB00284CD101354E489E
:109790002946D4F81490D4F81880E769FAF776F9D6
:1097A00030460021F7F7A4FB10B14848FAF76EF9EC
:1097B00069463046FAF750FA01464548FAF766F925
:1097C00048460021F7F794FB10B14048FAF75EF9DC
:1097D00069464846FAF740FA01463D48FAF756F915
:1097E00040460021F7F784FB10B13848FAF74EF9EC
:1097F00069464046FAF730FA01463548FAF746F925
:1098000038460021F7F774FB10B13048FAF73EF9FB
:1098100069463846FAF720FA01462E48FAF736F933
:1098200010340C2DABD12C48691CFAF72FF9F9F73D
:10983000FDFF2A4C064654F8041F19B12848FAF7D0
:1098400025F9F8E70D46274850F8251049B10122BF
:1098500002FA05F2324202D02348FAF717F901352D
:10986000F1E7154B214ACE1896F808418B5C04A805
:1098700001310519082905F8103CF2D100241C48D3
:1098800069468DF80840FAF701F914256543194E29
:109890001948A959FAF7FAF800217019FFF714FBD3
:1098A00001341648FFF76CFA722CEED105B0BDE812
:1098B000F08300BFE305010848180020D70601081F
:1098C0002C000108130601081E060108A106010864
:1098D0002F020108C301010826060108E4FF000861
:1098E00038060108E8FF00084606010888FF00085E
:1098F000530601081C1001085C06010898040108C1
:10990000F0B56D4B87B01A787AB96C4C012018709D
:1099100002212068FFF72AF92068FAF7E1F8684881
:10992000FFF72EFA6748FFF72BFA644C2068FBF725
:1099300051FB002800F0BD802068FBF750FB092890
:109940000146614A01D03F2851D1002517685F4C7C
:109950002E462FB15E4821683A4605F083F810B9CB
:10996000254606B926465B490C348C42F1D3C6B174
:109970003468D5F800E03B46E05C1EF803108142F5
:109980000DD1534A41B92D2B06D820244E48D4542A
:1099900001330360D15404E0D0540133ECE74A4969
:1099A0000B60494A14681CB1AE4201D13C4612E03A
:1099B0004948FFF7E5F9AE4209D856F80C0BFFF716
:1099C000DFF93E4B09211868FBF7F4FAF3E73D484D
:1099D000FFF7D6F900243C4B18688442A5D23749DA
:1099E0003B4A0868115DFBF7E5FA0134F3E71368B9
:1099F0002BB9042838D13648FFF7B4FB59E00C28BE
:109A000001D136488CE70A2901D00D2948D12E4DC5
:109A10003348FFF7B5F92E4C2A6832480023A35487
:109A200004930090294903A810220C23039403F007
:109A30006FFF054638B1006804F0E4FF411CAA68D6
:109A40006018904702E02848FFF79AF90021302279
:109A50001F4804F0A3F818491B4B0A78002018602F
:109A6000002A7FF45FAF24E00C28CAD07F2903D1FD
:109A70005BE72F2B3FF659AF1F297FF656AF7E29A4
:109A80003FF653AF13B920293FF44FAF104C581C89
:109A9000E1540A4A0C4B18601068FBF78BFA44E754
:109AA0007F29E6D10A4C581E0021106021540F482E
:109AB00039E707B0F0BD00BF84110020BC110020C1
:109AC000660601089E060108B811002088000108FA
:109AD0008511002048010108A3060108A806010815
:109AE00098040108AD8E0008B3060108D4060108E9
:109AF00037B505460220FFF71BF8064C01462060EB
:109B000030B90090AA6802200323FFF741F82060D3
:109B10003EBD00BFBC110020F8B5174E174C184DC4
:109B20000746C1B230682170FBF744FA22782B78DF
:109B3000C7F3072182EA0300287030682170FBF721
:109B400039FA21782A78306881EA0203C7F307419D
:109B50002B702170FBF72EFA2078297880EA010219
:109B6000390E306821702A70FBF724FA2B782078A0
:109B700080EA03012970F8BDC4110020C81100203B
:109B8000C0110020F8B50D4E0D4D0E4CC1B2074668
:109B900030682970FBF70EFA2A782378391282EAA6
:109BA0000300207029703068C9B2FBF703FA2378EC
:109BB0002A7882EA03002070F8BD00BFC41100209B
:109BC000E0110020C0110020054B10B504462146CD
:109BD0001868FBF7EFF9034802785440047010BD91
:109BE000C4110020C0110020034B04491A78885C7E
:109BF00001321A70704700BFC1110020E11100202E
:109C000010B5FFF7F1FF0446FFF7EEFF04EB00206D
:109C100080B210BD10B5FFF7F3FF0446FFF7F0FF69
:109C200004EB004010BD000038B5044624200D466A
:109C3000FFF7CAFF4D20FFF7C7FF002C0CBF3E20E7
:109C40002120FFF7C1FF064B002228461A70FFF7BC
:109C5000BBFF04480078BDE83840FFF7B5BF00BF40
:109C6000C0110020DE11002001460020FFF7DCBFFC
:109C700001460120FFF7D8BF014B1878FFF7A4BFBA
:109C8000C011002070B5054608460E46FFF7ECFFF0
:109C90002C467219D0B2E3B2984204D014F8010BEA
:109CA000FFF792FFF5E770BD10B5441E14F8010FE1
:109CB00010B1FFF789FFF9E710BD00002DE9F84367
:109CC000002701240025144B187885421CDA13491B
:109CD000134B15F801800C2202FB0830406804F099
:109CE00091FE81460CB13F180CE026464E4509DA3C
:109CF0000B4A0C2101FB08235868805DFFF764FFC5
:109D00000136F3E70135DEE724B1F8B2FFF7ACFF27
:109D10000024D7E7BDE8F883C2110020C911002054
:109D200060000020F7B5404DFF2115220746284668
:109D300003F034FF002302202B70FDF7DDFE012429
:109D400018B102206C70A87003240420FDF7D4FE23
:109D500068B1354E03214FF400503155651CF9F7B9
:109D600051FB18B104227255023400E02C46022047
:109D7000FDF7C2FE48B12C4B05201E190621072510
:109D800018557170B570033404E00820FDF7B4FE77
:109D90000028F0D12020F9F735FB18B1224B08221A
:109DA0001A5501344FF48070F9F72CFB30B11E487E
:109DB0000A2601190B2506554D7002341B4A1A4B11
:109DC0005079082801D00E2802D10C261E550134E6
:109DD0000D2104201955651CF9F714FB18B1124820
:109DE00011224255A51C1149132391F839210E4E19
:109DF0006C1C101C18BF01207355F9F703FB10B140
:109E000014203055AC1C0A4B01201C70FEF790FE4C
:109E1000084C0146206030B900907A680120032385
:109E2000FEF7B6FE2060FEBDC911002048180020D4
:109E3000C2110020C4110020F8B5B54C2068FBF712
:109E4000C9F8002800F033852068FBF7C8F8B14A4C
:109E50000346117871B9B0F12404634253EB040155
:109E600011700029E9D1AC4A5478002CE5D1FEF7F5
:109E700077FFE2E7012904D14D280CBF022300231C
:109E800021E0022904D13C280CBF032300231AE05F
:109E900003290FD140284FF0000101D91170CCE700
:109EA0009E489F4C03709F48217001709E490B7023
:109EB000042308E0042908D19B499C480C780370CE
:109EC00063400B7005231370B7E70529B5D194489B
:109ED000924C017822788A42934A07D914785C40E0
:109EE0001470934A53544B1C0370A6E710789842A1
:109EF00040F0D8848D4B19787B2900F01F8300F245
:109F0000C5806E2900F0698360D8682900F032832B
:109F100025D8652900F0068219D8642940F0BD844F
:109F20000720844CFFF7A0FEE620FFF74DFE607986
:109F3000FFF74AFE0020FFF747FE94F819017E4B19
:109F40007E4A00280CBF1046184600F059BC66290E
:109F500000F06682672940F0A08479480BE36B2902
:109F600000F0198323D8692900F009836A2940F099
:109F700094841020FFF778FE6748724CC07AFFF790
:109F800023FE71490878FFF71FFE2068FFF7C4FD24
:109F90006068FFF7C1FD6D4AB2F90000FFF7F2FDFE
:109FA0006B4BB3F90000FFF7EDFD6A4A12E36C2931
:109FB00000F003836D2940F070840620FFF754FE03
:109FC00065490868FFF7A8FD644A03E3732900F0B8
:109FD00071833CD8702900F02F83C0F00F83712962
:109FE00000F03D83722940F05884524C1620FFF750
:109FF0003BFE0020FFF7C6FDB4F9D000FFF7C2FD1D
:10A00000574DB4F9D200FFF7BDFDB4F9D400FFF706
:10A01000B9FDB5F9BA00FFF7B5FD0020FFF7B2FDB5
:10A020000020FFF779FDB5F928000A2390FBF3F033
:10A03000FFF7A8FD94F80401FFF7C6FD94F80601A8
:10A04000FFF7C2FD94F80501FFF7BEFD61E3762935
:10A0500000F03B830DD8742900F01983752940F076
:10A060001C842F20FFF700FE3E48FFF71DFE00F086
:10A0700017BC772900F00E83782940F00E84384C05
:10A080003820FFF7F1FD04F1400507E2D02900F088
:10A09000758300F2CA80CA2900F005816CD8A42912
:10A0A00000F0DA8310D8A02940F0F7830C20FFF7E6
:10A0B000DBFD2D492D4C0868FFF72EFD2C4A10685A
:10A0C000FFF72AFD20689BE3C82900F0DE80C9293C
:10A0D00040F0E383FFF788FD0F4B1A4CD872FFF76F
:10A0E00083FD19490870FFF795FD2060FFF792FD89
:10A0F0006060FFF785FD154A1080FFF781FD144B66
:10A1000018801C48017841F002040470DAE000BFB6
:10A11000C4110020C31100201F1E0020DF110020E9
:10A1200021120020C1110020C0110020DE110020EA
:10A13000E1110020481800201C000080140000805D
:10A1400018000020F41D00200C1E0020A61D002079
:10A15000B21D0020640F0020441D00203C0C002094
:10A16000FC1B002004190108E8F7FF1FF0F7FF1F90
:10A17000ECF7FF1F800F0020CD2900F0098322D8C3
:10A18000CB2900F0A180CC2940F08783FFF72CFD7C
:10A19000CC4CE077FFF728FD84F82000FFF724FD82
:10A1A00084F82300FFF720FD84F82400FFF71CFD4E
:10A1B00084F82500FFF718FD84F82100FFF714FD4F
:10A1C00084F822007EE0CE2900F0EC82CF2940F016
:10A1D0006483FFF715FDFFF713FDBB4CB94DA4F8E1
:10A1E000D000FFF70DFDA4F8D200FFF709FDA4F899
:10A1F000D400FFF705FDA5F8BA00FFF701FDFFF752
:10A2000009FDFFF7FDFC0A2358432885FFF7ECFC06
:10A2100084F80401FFF7E8FC84F80601FFF7E4FC8A
:10A2200084F80501FFF7E0FC4CE0D52900F09481AB
:10A230000FD8D22961D0C0F07082D3296DD0D42933
:10A2400040F02B839F4C0020FFF70EFD04F14005EA
:10A2500056E1F02900F0C7820CD8D62944D0EF2966
:10A2600040F01B83FFF7CCFC964CA085FFF7C8FCA1
:10A27000608527E0FA2900F09D82FE2940F00D83D9
:10A280000820FFF7F1FC0024A5E20024FFF7B8FC4A
:10A290008E4A10530234102CF8D10020FFF7E4FC52
:10A2A000FDF7ACFDFCE28A4C04F10A05FFF79CFCCB
:10A2B00001346070FFF798FCE072FFF795FCAC4248
:10A2C0006075F3D1002083E20024824801788C423B
:10A2D000F8D2814D655DFFF793FC7A4A013402EBB9
:10A2E0004505A5F84600F0E70024FFF789FC7B4A06
:10A2F00010530234102CF8D1E4E7794C6478002C28
:10A30000E0D1FFF771FC7049022881F8AC0388BFE7
:10A3100081F8AC43F9F728F837E2FFF771FC714B8D
:10A320001880CFE7704D0B20FFF79EFCB5F90000B9
:10A33000FFF728FCF7F7D6FB00B2FFF723FC02205B
:10A34000FDF7DAFB05460420FDF7D6FB044608209E
:10A35000FDF7D2FB820042EA4401294320208CB25F
:10A36000FDF7CAFB44EAC00084B21020FDF7C4FB2D
:10A3700044EA001318B2FFF705FC594A1079D17866
:10A3800084005378907944EA4101194341EAC004BA
:10A390005179537A44EA411040EA83145348C17911
:10A3A00044EAC113047A417A43EA042343EA41248C
:10A3B000D379117A44EA8324927A44EAC123417B17
:10A3C00043EA0234827B44EA4133017C43EA82342B
:10A3D000027944EA0143417C43EA0214827C44EA64
:10A3E0004143C17C43EA8244007D44EAC142394B87
:10A3F00042EA00540020197803468B420AD2364DB7
:10A4000001225D5D02FA05F525421CBF9A4010430A
:10A410000133F2E72C4CFFF77FFB94F8AC0379E1B2
:10A420001220FFF721FC32490C88B4F5806F314CC3
:10A43000B4F9000008D8FFF7A5FBB4F90200FFF754
:10A44000A1FBB4F904000EE0082590FBF5F0FFF73E
:10A4500099FBB4F9020090FBF5F0FFF793FBB4F918
:10A46000043093FBF5F0244CFFF78CFBB4F90000AB
:10A47000FFF788FBB4F90200FFF784FBB4F904008E
:10A480001E4CFFF77FFBB4F90000FFF77BFBB4F92C
:10A490000200FFF777FBB4F90400AEE1B4F97800ED
:10A4A000FFF770FBB4F97A00FFF76CFBB4F97C009E
:10A4B000FFF768FB94F87E000834FFF785FBAC4299
:10A4C000ECD1EDE1FC1B002048180020761E002096
:10A4D000FB1B0020C2110020C91100207C1D0020A0
:10A4E0001F1E0020101D00200E0B0020301E00201B
:10A4F000040000204C1D0020240C0020F81C00202B
:10A50000FFF77EFBA4F87800FFF77AFBA4F87A0047
:10A51000FFF776FBA0F57A7107288AB298BF84F816
:10A520007F00B2F57A7F98BFA4F87C00FFF75CFB50
:10A5300084F87E000834AC42E2D1B1E10820FFF794
:10A5400093FB0024B04AA31893F87F000834FFF768
:10A550003BFB402CF6D1A3E10020FFF785FB002454
:10A56000FFF742FBA84AA3180834402C83F87F0069
:10A57000F6D195E1A5481021FFF784FB90E110206A
:10A58000FFF772FB0024A248005F0234FFF7FAFADB
:10A59000102CF8D184E10520FFF766FB9D4BB3F941
:10A5A0000000FFF7EFFA9C48B0F90000FFF7EAFA65
:10A5B0009A490A7802F00100ACE0994C0620FFF7B6
:10A5C00053FBB4F90000FFF7DDFAB4F90200FFF71E
:10A5D000D9FA944AB2F900000FE10720FFF744FBD3
:10A5E00091480078FFF7F0FA0020FFF7CBFA8F4B85
:10A5F000B3F90000FFF7C6FA0020FEE0824C072006
:10A60000FFF732FBE07FFFF7DFFA94F82000FFF757
:10A61000DBFA94F82300FFF7D7FA94F82400FFF749
:10A62000D3FA94F82500FFF7CFFA94F82100FFF74A
:10A63000CBFA94F822006DE01E20FFF715FB7C4C4E
:10A6400004F10A0501346078FFF7BEFAE07AFFF7FB
:10A65000BBFA607DFFF7B8FAAC42F3D120E175494F
:10A660000A78540004F0FE00FFF7FEFA0024714857
:10A6700003789C4280F014816F496348625C013426
:10A6800000EB4203B3F94600FFF77CFAEFE7FFF770
:10A6900015FB05E1674900240878FFF7E5FA654AEC
:10A6A0001078844280F0FC80634B185DFFF78CFAD1
:10A6B0000134F4E70820FFF7D7FA0124E0B20134AF
:10A6C000FFF782FA092CF9D1EAE0FFF78DFA064686
:10A6D0001220FFF7C9FA0EB9584902E0102E03D133
:10A6E00057490D684C6801E0002425463046FFF7C5
:10A6F0006BFA2846FFF710FA2046FFF70DFA514A89
:10A700001068FFF709FA0020FFF73CFA0020FFF776
:10A7100039FA0020FFF758FAC2E0FFF765FA05465C
:10A72000FFF778FA0746FFF775FA0646FFF772FA61
:10A730000446FFF765FAFFF763FAFFF755FA65B9C4
:10A740003E484149012207604660CD710A73002CE2
:10A750003FF4B8AD3B4B1C60B4E5102D7FF4B2ADB7
:10A760003748076046600CB136490C603448374BB7
:10A770000222011D1A70FCF7AFFAA3E532484178B6
:10A7800000297FF49FADF8F74FFEF9F70BF899E534
:10A790002D4C6378002B7FF495AD4FF4C870FAF719
:10A7A000CBF98FE52848417800297FF48BAD012251
:10A7B000827387E5244B5C78002C6ED1244991F894
:10A7C000AC03F8F7C1FDF8F7CFFDF8F7EBFF204633
:10A7D000FFF74AFA64E01F48005F0234FFF7D2F93E
:10A7E000082CF8D15CE0084C0420FFF73DFAB4F9DE
:10A7F0002C00FFF7C7F9B4F92A00FFF7C3F94FE0BF
:10A80000FFF78AF94CE000BFFC1B0020641D00200C
:10A81000761E0020D61D0020E01D0020800F0020A5
:10A82000580C0020221D002044180020E21C0020AB
:10A83000FB1B0020C2110020C9110020D81D0020E0
:10A84000B41D0020481D00201F1E0020740D002094
:10A8500048180020DA1C0020154C23789800411C71
:10A86000C8B2FFF701FA2078FFF7AEF90024104ACA
:10A8700013789C4214D20F48005DFFF7A5F90E49EA
:10A88000085DFFF7A1F90D4A105DFFF79DF90C4B2C
:10A89000185DFFF799F90134E9E70020FFF7E8F9BF
:10A8A000FFF7EAF9074900200870FFF7C6BAF8BDBC
:10A8B0000D1E0020951D0020E21D0020FC1D002023
:10A8C0000E1E0020C31100202DE9F04107468846E6
:10A8D00016460024B4420ED00025BD4205D04046A5
:10A8E0000135FAF7C4FBEDB2F7E73C200134FAF783
:10A8F000BEFBE4B2EEE7BDE8F08100000F4B1A6842
:10A9000042F00100186059680D4A0A405A60186800
:10A9100020F0847121F480321A60186820F48021BC
:10A9200019605A684FF41F0122F4FE0058609960C4
:10A93000044B4FF000629A60704700BF0010024065
:10A940000000FFF800ED00E0164A174B516801F0D7
:10A950000C00042803D0082805D0144801E014494D
:10A960000868186011E051685068C1F383410231F2
:10A97000C00301D40F4A06E052680D4812F4003FAC
:10A98000026818BF520851431960064B0A485A68BA
:10A99000054BC2F30311415C1A6822FA01F21A60F6
:10A9A000704700BF001002407C01002000127A00B6
:10A9B0007801002000093D00680100201FB5002338
:10A9C000574C4FF4E01100930193029303912268D6
:10A9D00042F480332360A16941F01002A261504C1F
:10A9E000236803F400310191009A531C00930199EC
:10A9F00019B9009AB2F5A06FF1D12168484B11F452
:10AA0000003401D0022416E01A6842F001011960F6
:10AA10000094434B1C6804F00202019200994C1C04
:10AA20000094019A1AB90099B1F5A06FF1D11B6891
:10AA300099073BD501243B4902940A6842F0100370
:10AA40000B600C6824F003020A600B6843F00204F8
:10AA50000C60A1F58053596859605A685A605C6867
:10AA6000314A44F480615960146824F070411160E7
:10AA70002E4C2F490C605C6824F47C145C601468D4
:10AA800044F000441460946824F400449460043A50
:10AA90009268120449BF274A4FF4E0120A604FF44B
:10AAA000801203920299012901D119E0FEE70229DF
:10AAB0001AD168B10398B0F5801F02D14FF4A012EB
:10AAC00005E0039BB3F5E01F02D14FF4001203929F
:10AAD000134B5968039841EA000242F4803002E0C7
:10AAE000596841F4601058600D4B1A68184642F0DE
:10AAF0008071196002680A4B9201FBD5596821F0F8
:10AB0000030058605A6842F002015960044B5868CB
:10AB100000F00C02082AF9D1FFF716FF1FBD00BF95
:10AB200000100240002002400410014000127A0090
:10AB300078010020001BB70008B5154B98420BD1D7
:10AB400001214FF4805000F0C9FD4FF480500021E6
:10AB5000BDE8084000F0C2BD0E49884207D14FF45D
:10AB60008040012100F0C6FD4FF4804009E00A4A10
:10AB700090420BD14FF40040012100F0BBFD4FF497
:10AB800000400021BDE8084000F0B4BD08BD00BF92
:10AB90000030014000380040003C00400B8810B5F8
:10ABA0004C88028823438C8802F441522343CC888A
:10ABB00023430C8923434C8923438C892343CC8929
:10ABC000098A23431A4393B20380828B22F40063E1
:10ABD0001A04130C8383018210BD038819B199B242
:10ABE00041F0400303E023F040010A04130C03800A
:10ABF000704781817047808980B27047038919420C
:10AC00000CBF002001207047426810B522F4702369
:10AC10000A6823F4807444EA02030C7943EA0422AC
:10AC20004260CB688A6884681A43084B2340134308
:10AC30004A7943EA42038360097CC26A4B1E22F4CC
:10AC40007002D9B242EA0152C26210BDFDF7F1FFB3
:10AC5000836811B143F0010101E023F0010181603B
:10AC60007047836811B143F4807101E023F480716F
:10AC700081607047836843F0080181607047806895
:10AC8000C0F3C0007047836843F0040181607047DF
:10AC90008068C0F380007047836811B143F4A0015D
:10ACA00001E023F4A00181607047092970B54FF0DD
:10ACB00003040CD94C4307251E3C05FA04F503FA9E
:10ACC00004F3C66826EA05052B43C3600BE04C433A
:10ACD000072505FA04F503FA04F3066926EA0505D3
:10ACE00045EA03040461062A4FF005030DD8013A32
:10ACF00053431F2202FA03F201FA03F1446B24EAE0
:10AD0000020242EA0103436370BD0C2A0DD853438B
:10AD10001F22233B02FA03F201FA03F1046B24EA37
:10AD2000020242EA0103036370BD53431F22413B09
:10AD300002FA03F201FA03F1C46A24EA020211439F
:10AD4000C16270BD40F0BF60024B40F40031D96079
:10AD5000704700BF00ED00E0C37810B503B3164C98
:10AD6000E168CB43C3F302244178C4F1040201FA41
:10AD700002F10F2222FA04F28478037822400A4377
:10AD8000110103F16043CAB203F5614181F8002368
:10AD90000078012200F01F03410902FA03F007E0E6
:10ADA0000078012200F01F03410902FA03F020316C
:10ADB000024B43F8210010BD00ED00E000E100E08F
:10ADC00030B5048C24F001052C04250C0584048B7B
:10ADD000A5B225F0F3052A4342EA0313114A048C75
:10ADE0009042A4B29DB215D002F50063984211D0F2
:10ADF000B0F1804F0ED0A3F5983290420AD002F500
:10AE00008063984206D003F58062904218BF24F018
:10AE10000A0401D124F0020444F001042143058313
:10AE2000018430BD002C014030B5048C24F01005A5
:10AE30002C04250C0584048B058C24F44074240513
:10AE4000240D44EA022242EA0333144AADB290428E
:10AE50009BB212D002F5006290420ED0B0F1804F4A
:10AE60000BD0A2F59832904207D002F58062904252
:10AE700003D002F58062904207D125F0200242F013
:10AE8000100545EA011189B204E025F0A00545F05E
:10AE9000100529430383018430BD00BF002C01400D
:10AEA000224A038890429BB212D002F5006290427F
:10AEB0000ED0B0F1804F0BD0A2F59832904207D05F
:10AEC00002F58062904203D002F58062904203D185
:10AED0004A8823F070031343154A904208D002F5C4
:10AEE0008062904204D023F44073CA889BB213431B
:10AEF00003808B880A8883850C4B028598420FD08B
:10AF000003F5006290420BD002F54063984207D0EF
:10AF100003F58062904203D002F58063984201D12C
:10AF2000097A018601228282704700BF002C01400D
:10AF300000100040038C70B523F001021404250CAE
:10AF40000584068C8388028B9CB222F073052B0447
:10AF50000D881A0C26F0020633042A434E880D8908
:10AF60001B0C3543ADB22B43134DA8420FD005F552
:10AF70000065A8420BD005F54065A84207D005F54D
:10AF80008065A84203D005F58065A8420ED123F064
:10AF900008064B898D881E4326F004032B43CE8977
:10AFA0008D8924F440743543ADB22C43C988848024
:10AFB00002838186038470BD002C0140038C30B570
:10AFC00023F010021404250C0584038C8288048B62
:10AFD00023F0200324F4E6452C040D88240C44EAD5
:10AFE00005241D042B0C0D8992B243EA05134D88EC
:10AFF000A4B243EA0513124D9BB2A84203D005F553
:10B000000065A84215D14D8923F080039BB243EA25
:10B0100005134FF6BF751D408B8822F4406245EA48
:10B020000315ABB28D8942EA8502CD8942EA8502D9
:10B0300092B2C988828004830187038430BD00BF37
:10B04000002C0140038C30B523F480721404250CCD
:10B050000584038C8288848B23F4007324F07305A9
:10B060002C040D88240C2C431D042B0C0D8992B24A
:10B0700043EA05234D8843EA0523124D9BB2A842BB
:10B0800003D005F50065A84215D14D8923F400636E
:10B090009BB243EA05234FF6FF351D408B8822F40F
:10B0A000405245EA0325ABB28D8942EA0512CD89AB
:10B0B00042EA051292B2C988828084838187038420
:10B0C00030BD00BF002C0140038C30B523F480520A
:10B0D0001404250C0584038C8288858B94B225F496
:10B0E000E64215042A0C0D8823F4005342EA052297
:10B0F0001D042B0C0D8992B243EA05334D8843EAB7
:10B1000005330A4D9BB2A84203D005F50065A8425D
:10B1100005D18D8924F4804444EA8514A4B2C988F9
:10B1200084808283A0F84010038430BD002C01404D
:10B1300000214FF6FF7383800180C180418001723E
:10B1400070470023038043808380C3800381438151
:10B150008381C38170470023012203804380828062
:10B16000C38003817047038819B199B241F001038C
:10B1700003E023F001010A04130C03807047B0F8C8
:10B18000443029B16FEA43436FEA53418AB201E088
:10B1900059044A0CA0F84420704783899BB20AB135
:10B1A000194301E023EA010181817047038B23F0F9
:10B1B000080213041A0C114301837047038B23F414
:10B1C000006213041A0C42EA01218BB20383704718
:10B1D000838B23F0080213041A0C114381837047F8
:10B1E000838B23F4006213041A0C42EA01218BB210
:10B1F0008383704781847047038B23F00C02130410
:10B200001A0C0283038B9AB2114301837047038B9C
:10B2100023F4406213041A0C0283038B9AB242EAAD
:10B2200001218BB203837047838B23F00C0213043C
:10B230001A0C8283838B9AB2114381837047838B6C
:10B2400023F4406213041A0C8283838B9AB242EA7D
:10B2500001218BB283837047F8B50B880D460446F5
:10B260004988AA8843B92B89FFF7AAFDE9882046B7
:10B27000BDE8F840FFF7C0BF042B08D12B89FFF7CA
:10B28000D3FDE9882046BDE8F840FFF7C0BF082B92
:10B290000E462F89008C3BD120F480731804030CD8
:10B2A0002384A08B83B223F0F30343EA0717374BC1
:10B2B000208CBFB29C4280B247EA020212D003F552
:10B2C00000639C420ED0B4F1804F0BD0A3F59833AD
:10B2D0009C4207D003F580639C4203D003F5806352
:10B2E0009C4207D120F4007040EA06218BB243F45F
:10B2F000807305E020F4206041F4807140EA01038E
:10B30000E9882046A2832384BDE8F840FFF78CBF7C
:10B3100020F480531804030C2384A38B208C23F483
:10B3200040731B051B0D43EA022242EA0733174A0A
:10B3300080B294429BB212D002F5006294420ED0C9
:10B34000B4F1804F0BD0A2F59832944207D002F5A9
:10B350008062944203D002F58062944207D120F4C7
:10B36000005040EA063291B241F4805205E047F6BF
:10B37000FF52024041F480510A43E9882046A383EA
:10B380002284BDE8F840FFF75ABF00BF002C0140FF
:10B39000808E80B27047008F80B27047808F80B2FD
:10B3A0007047B0F8400080B27047038A828911EA82
:10B3B000030092B203D011420CBF0020012070475D
:10B3C000C9438AB202827047038A30B50D460446EB
:10B3D000EA8898B220F4405111432182A389288938
:10B3E000A98823F4B05340EA0102688923F00C01D4
:10B3F00002430804030C1A4391B2A181A08AAA89CE
:10B4000083B223F4407187B01143A18201A800F0F8
:10B41000F3F81848A38984420CBF0498039819B222
:10B4200000294FF019032A6803FB00F001DA5100EC
:10B4300000E09100B0FBF1F16423B1FBF3F21201E3
:10B44000100903FB1011A08900B2002806DAC90018
:10B450003231B1FBF3F303F0070005E009013231AB
:10B46000B1FBF3F303F00F00024390B2208107B069
:10B4700030BD00BF00380140838919B199B241F451
:10B48000005303E023F400510A04130C8381704736
:10B49000C1F3421310B5012401F01F01A34204FAC5
:10B4A00001F101D10C3004E0022B01D1103000E099
:10B4B0001430036812B143EA010201E023EA0102F9
:10B4C000026010BD838A9BB20AB1194301E023EAEE
:10B4D000010181827047090A012303FA01F3DA436B
:10B4E00091B2018070470000034A044B02F188309A
:10B4F0005A605860704700BF230167450020024032
:10B50000024B1A6942F08000186170470020024027
:10B51000014BD860704700BF00200240084BDA683A
:10B52000D20709D4D868400708D4D96811F0100FA1
:10B530000CBF042003207047012070470220704791
:10B540000020024010B50446FFF7E8FF012806D1AD
:10B550001CB1FFF7E3FF013CF8E7052010BD002C0C
:10B5600008BF052010BD000073B5002306464FF448
:10B5700000500D460193FFF7E5FF04281AD10E4C49
:10B58000AAB2206940F0010121614FF400503280DD
:10B59000FFF7D8FF042808D102360196019B2D0C35
:10B5A0001D804FF40050FFF7CDFF216941F6FE7278
:10B5B0000A4022617CBD00BF0020024038B505462C
:10B5C0004FF43020FFF7BEFF042812D1094C236945
:10B5D00043F002002061656121694FF4302041F0A1
:10B5E00040022261FFF7AEFF216941F6FD730B4077
:10B5F000236138BD00200240204B10B55A6802F08C
:10B600000C01042903D0082905D01D4B01E01D4C75
:10B610002368036011E05C685968C4F38342941C9A
:10B62000C90301D4184A06E016495B680A6813F496
:10B63000003F18BF520854430460104B5968C1F3CF
:10B64000031212498C5C026822FA04F242605C68C0
:10B65000C4F302240C5D22FA04F484605C68C4F331
:10B66000C224095D22FA01F2C2605B680849C3F393
:10B670008133CB5CB2FBF3F2026110BD00100240DB
:10B6800000127A007801002000093D0084010020AA
:10B6900080010020044B5A6909B1104301E022EAFD
:10B6A00000005861704700BF00100240044B9A69C7
:10B6B00009B1104301E022EA00009861704700BF21
:10B6C00000100240044BDA6909B1104301E022EA9C
:10B6D0000000D861704700BF00100240044BDA68D8
:10B6E00009B1104301E022EA0000D860704700BFB2
:10B6F00000100240044B1A6909B1104301E022EA2C
:10B7000000001861704700BF00100240024B5A6AE7
:10B7100042F08070586270470010024008B50B4B31
:10B72000984207D14FF400100121FFF7E3FF4FF4D7
:10B73000001006E04FF480000121FFF7DBFF4FF41B
:10B7400080000021BDE80840FFF7D4BF005400404E
:10B75000F0B58688044687B026F03F000D46010408
:10B7600001A80E0CFFF748FF2C4A0399B1FBF2F039
:10B7700087B23E43A680238823F0010213041A0CEB
:10B7800022802B68264A93420AD85B00B1FBF3F073
:10B79000013783B2BFB22784032B98BF042320E074
:10B7A000EE884BF6FF72964204D103225343B1FB5D
:10B7B000F3F305E019225343B1FBF3F141F4804365
:10B7C00099B20A054FF4967208BF41F00101504347
:10B7D00041F400434FF47A7190FBF1F0421C91B2B6
:10B7E0002184A383228891B241F001032380208821
:10B7F00020F4816222F002010B04AA886989180CE6
:10B8000041EA02032989AA89184380B241EA020366
:10B81000208098B2208107B0F0BD00BF40420F00E9
:10B82000A086010041F28833002103604BF6FF72CD
:10B830004FF480438180C2800181418183817047C0
:10B84000038819B199B241F0010303E023F001012B
:10B850000A04130C03807047038819B199B241F4AC
:10B86000807303E023F480710A04130C0380704793
:10B87000038819B199B241F4007303E023F4007115
:10B880000A04130C03807047038819B199B241F47C
:10B89000806303E023F480610A04130C0380704783
:10B8A00083889BB20AB1194301E023EA0101818038
:10B8B000704701827047008AC0B2704712B141F0F0
:10B8C000010101E001F0FE010182704702684FF6BC
:10B8D000FE73134003602D4B0021984201604160CC
:10B8E0008160C16022D02A49884229D0294B9842E0
:10B8F00030D02949884237D0284B98423ED0284B37
:10B90000984206D153F8681C41F4700043F8680C63
:10B9100070472449884206D151F87C0C40F070628F
:10B9200041F87C2C7047204B984206D153F8042CE8
:10B9300042F00F0143F8041C70471C49884206D1AD
:10B9400051F8183C43F0F00041F8180C7047184BC0
:10B95000984206D153F82C2C42F4706143F82C1C09
:10B9600070471449884206D151F8403C43F4704076
:10B9700041F8400C7047104B984205D153F8542CB5
:10B9800042F4702143F8541C704700BF0800024085
:10B990001C000240300002404400024058000240B7
:10B9A0006C00024080000240080402401C04024077
:10B9B00030040240440402405804024070B5066856
:10B9C0008C680D6A26F4FF4222F070060A6945EA87
:10B9D00004034C6913438A692343CC6913431C4312
:10B9E0004B6A44EA03028B6A1A4332430260CB6813
:10B9F0000A68496843608260C16070BD00230360CB
:10BA000043608360C360036143618361C361036218
:10BA100043628362704719B1016841F0010303E09A
:10BA200002684FF6FE7313400360704703680AB163
:10BA3000194301E023EA010101607047416070474A
:10BA4000406880B270470000C3004CBF014B024BFE
:10BA500058607047000402400000024000B540F604
:10BA6000D87320F00042C3F649739A4283B001466E
:10BA700015DDB2F1FF4F03DBF4F792FF03B000BD19
:10BA8000694600F095FB00F00302012A0098019935
:10BA90000ED0022A07D082B900F0A0FDEEE7002107
:10BAA00000F09CFDEAE700F099FD00F10040E5E7B9
:10BAB00001F040FC00F10040E0E7012201F03AFC17
:10BAC000DCE700BF30B5C0F3C754A4F17F031E2BE1
:10BAD00083B0014621DC581C1DDBCD0F162B0CDD7D
:10BAE00021F07F4323F4000040F40000963C00FA6C
:10BAF00004F005B1404203B030BD114850F8254074
:10BB00002046F4F74FFF019021460198F4F748FFD3
:10BB100020F0004121B90020EDE7F5F711FAEAE73E
:10BB200020F07F4222F40003C0F3C75043F4000129
:10BB3000C0F1960221FA02F0002DDCD0DAE700BF56
:10BB4000E419010800B540F6D87320F00042C3F6AE
:10BB500049739A4283B0014616DDB2F1FF4F03DB11
:10BB6000F4F71EFF03B000BD694600F021FB00F0B2
:10BB70000300012815D002280BD0B8B9009801990C
:10BB8000012201F0D7FBEDE70021002201F0D2FBFA
:10BB9000E8E700980199012201F0CCFB00F1004098
:10BBA000E0E70098019900F019FDDBE700980199A2
:10BBB00000F014FD00F10040D4E700BF70B58AB07A
:10BBC000064600F09BF8224C054694F900300133FC
:10BBD00003D0304601F0B0FD10B928460AB070BD60
:10BBE000304601F05BFD4FF07E51F5F79FF90028DC
:10BBF000F3D0184A012100253046019200910895A2
:10BC0000F4F714FC02460B461348CDE90423CDE9B2
:10BC1000022301F011FC94F90030CDE90601022B5A
:10BC20000BD0684601F006FC38B1089850B9DDE940
:10BC30000601F4F761FE0546CFE701F089FE2121F8
:10BC40000160F2E701F084FE089A0260EFE700BFAE
:10BC500094010020EC190108F419010800F002BA5F
:10BC600070B58AB0054600F04FFC224C064694F9A8
:10BC70000030013308D0284601F05EFD20B128468F
:10BC80000021F5F735F910B930460AB070BD1A4AEF
:10BC9000012128460026009101920896F4F7C6FB80
:10BCA0002478CDE90401CDE902017CB9002200230A
:10BCB000CDE90623684601F0BDFB88B10898A0B91C
:10BCC000DDE90601F4F718FE0646DDE70020002155
:10BCD00002460B46F4F728FD022CCDE90601E9D116
:10BCE00001F036FE21230360E8E701F031FE0899F8
:10BCF0000160E5E794010020F8190108F8B520F08B
:10BD00000043B3F17E5F044613D00BDCB3F17C5FDC
:10BD100014DAB3F10C5F00F3A48040F6DB70C3F6D5
:10BD2000C970F8BD0146F4F73BFE0146F4F7F6FF93
:10BD3000F8BD002840F30E810020F8BD0028C0F2B5
:10BD40000E8101464FF07E50F4F72AFE4FF07C51F1
:10BD5000F4F730FF044600F0D7FB4EF608710646B4
:10BD600020F47F65C3F611012046F4F723FF47F660
:10BD70000471C3F64F21F4F715FE2146F4F71AFFBC
:10BD800041F24611C3F62451F4F70AFE2146F4F7B6
:10BD900011FF40F6A821C3F64E61F4F703FE2146D9
:10BDA000F4F708FF4BF29001C3F6A661F4F7F8FD33
:10BDB0002146F4F7FFFE4AF6AB21C3F62A61F4F7F9
:10BDC000F1FD2146F4F7F6FE4CF22E610746C3F66C
:10BDD0009D512046F4F7EEFE43F26131C3F6307117
:10BDE000F4F7DEFD2146F4F7E5FE45F22D71C4F2CD
:10BDF0000101F4F7D7FD2146F4F7DCFE4DF23911CD
:10BE0000C4F21901F4F7CCFD2146F4F7D3FE4FF04C
:10BE10007E51F4F7C7FD01463846F4F77FFF3146FF
:10BE2000F4F7C8FE25F00F05074629462846F4F723
:10BE3000C1FE01462046F4F7B3FD294604463046CC
:10BE4000F4F7B0FD01462046F4F768FF0146384696
:10BE5000F4F7A8FD2946F4F7A5FD0146F4F7A2FD85
:10BE6000F8BD0146F4F7A6FE4EF60871C3F61101BF
:10BE70000546F4F79FFE47F60471C3F64F21F4F729
:10BE800091FD2946F4F796FE41F24611C3F624517E
:10BE9000F4F786FD2946F4F78DFE40F6A821C3F697
:10BEA0004E61F4F77FFD2946F4F784FE4BF29001D2
:10BEB000C3F6A661F4F774FD2946F4F77BFE4AF653
:10BEC000AB21C3F62A61F4F76DFD2946F4F772FE43
:10BED0004CF22E610646C3F69D512846F4F76AFEE1
:10BEE00043F26131C3F63071F4F75AFD2946F4F795
:10BEF00061FE45F22D71C4F20101F4F753FD2946AC
:10BF0000F4F758FE4DF23911C4F21901F4F748FD67
:10BF10002946F4F74FFE4FF07E51F4F743FD0146FA
:10BF20003046F4F7FBFE01462046F4F743FE014697
:10BF300042F26810C3F2A230F4F732FD0146204607
:10BF4000F4F72EFD014640F6DA70C3F6C970F4F737
:10BF500027FDF8BD40F6DB70C4F24900F8BD4FF094
:10BF60007E51F4F71FFD4FF07C51F4F723FE4EF69F
:10BF70000871C3F611010446F4F71CFE47F604717C
:10BF8000C3F64F21F4F70EFD2146F4F713FE41F2FC
:10BF90004611C3F62451F4F703FD2146F4F70AFED7
:10BFA00040F6A821C3F64E61F4F7FCFC2146F4F7F5
:10BFB00001FE4BF29001C3F6A661F4F7F1FC2146B5
:10BFC000F4F7F8FD4AF6AB21C3F62A61F4F7EAFC70
:10BFD0002146F4F7EFFD0646204600F095FA4CF2B4
:10BFE0002E610546C3F69D512046F4F7E3FD43F26A
:10BFF0006131C3F63071F4F7D3FC2146F4F7DAFD72
:10C0000045F22D71C4F20101F4F7CCFC2146F4F79E
:10C01000D1FD4DF23911C4F21901F4F7C1FC2146EA
:10C02000F4F7C8FD4FF07E51F4F7BCFC01463046F2
:10C03000F4F774FE2946F4F7BDFD42F26811C3F22D
:10C04000A231F4F7ADFC01462846F4F7ABFC0146FB
:10C05000F4F7A8FC014640F6DA70C4F24900F4F7A0
:10C060009FFCF8BDF8B521F00044B4F1FF4F034642
:10C0700017DC20F00045B5F1FF4F064611DCB1F1A9
:10C080007E5F42D08F1707F0020040EAD37775B980
:10C09000022F35D0032F08D140F6DB73CCF24903D1
:10C0A00003E01846F4F77EFC03461846F8BDD4B109
:10C0B000B4F1FF4F2DD0B5F1FF4F14D02C1BE41578
:10C0C0003C2C18DC002952DB1846F4F727FE01F05F
:10C0D000E5FA01F0B7F9012F46D0022F35D0002F35
:10C0E00025D10346E1E7002E40F6DB731CDBC3F6E7
:10C0F000C9731846F8BD40F6DB70C3F6C970EAE7AD
:10C1000040F6DB73C4F24903CFE7BDE8F84001F025
:10C1100099B9B5F1FF4F2FD0022FF1D0032FBBD02B
:10C12000012F34D00023C0E7CBF6C973BDE74BF62F
:10C130002E51C3F2BB31F4F735FC40F6DB71C4F28B
:10C140004901F4F72DFC0346AFE74BF62E51C3F23D
:10C15000BB31F4F727FC014640F6DB70C4F249001E
:10C16000F4F71EFC0346A0E700F100439DE714F13D
:10C170003C0FA9DA0020AEE7022F13D0032F0CD01A
:10C18000012F40F6DB7305D0C3F649738DE74FF0FE
:10C1900000438AE7CBF6497387E74CF6E433CCF2E9
:10C1A000160382E74CF6E433C4F216037DE700BFC2
:10C1B0002DE9F04F40F6D87320F00044C3F64973E0
:10C1C0009C4289B006460D4640F38B804CF6E33125
:10C1D000C4F216018C4226DC4FF478610028C3F6C5
:10C1E000C97140F32B81F4F7DBFB4FF47D6224F03F
:10C1F0000F04C3F6C9729442064600F0818044F2EF
:10C200004341C3F23571F4F7CBFB01462860304659
:10C21000F4F7C6FB44F24341C3F23571F4F7C0FBB7
:10C220000127686061E04FF47867C4F24937BC4287
:10C2300040F38180B4F1FF4F5BDA4FEAE459A9F192
:10C240008609A4EBC9542046F4F77AFEF4F75EFCA5
:10C250000246014620460592F4F7A2FB4FF08741C3
:10C26000F4F7A8FC0746F4F76BFEF4F74FFC014621
:10C27000044638460694F4F793FB4FF08741F4F7F1
:10C2800099FC00210790F4F729FE002800F0F680C1
:10C290000327204600210DF11808013FF4F71EFE88
:10C2A00040B158F8044D00212046013FF4F716FE36
:10C2B0000028F6D1924B02200090019305A83B463E
:10C2C00029464A4600F066FA002E07460DDA95E840
:10C2D0000C0002F1004103F1004229606A6047420C
:10C2E00003E00023286000274B60384609B0BDE812
:10C2F000F08F0146F4F754FB002768602860F4E7EC
:10C300004FF48841C3F23571F4F74AFB4AF2083121
:10C31000C2F685610446F4F743FB014628602046D7
:10C32000F4F73EFB4AF20831C2F68561F4F738FBB8
:10C3300001276860D9E701F0B1F94FF68411C3F61F
:10C3400022718046F4F736FC4FF07C51F4F72AFB5B
:10C35000F4F7F6FD0746F4F7D9FB4FF47861C3F61E
:10C36000C9718346F4F726FC01464046F4F718FBF2
:10C3700044F243418146C3F235715846F4F71AFC42
:10C380001F2F8246514648461FDC5E4B7A1E53F8EB
:10C39000223024F0FF029A4217D0F4F701FB8046C6
:10C3A000C5F8008041464846F4F7FAFA5146F4F7DA
:10C3B000F7FA002E686098DA08F1004800F10041B1
:10C3C000C5F8008069607F428FE7F4F7E9FAE3156A
:10C3D0008046C0F3C750191A0829E1DD4FF488419F
:10C3E000C3F2357158460393F4F7E4FB8246514695
:10C3F0004846F4F7D5FA044621464846F4F7D0FA01
:10C400005146F4F7CDFA4AF208318146C2F6856109
:10C410005846F4F7CFFB4946F4F7C2FA8246514634
:10C420002046F4F7BDFA039BC0F3C7528046981A22
:10C43000192841DCC5F80080A146B3E7F4F7B2FA49
:10C440004FF47D6724F00F04C3F6C977BC4206465B
:10C4500016D044F24341C3F23571F4F7A3FA014612
:10C4600028603046F4F79CFA44F24341C3F2357138
:10C47000F4F798FA4FF0FF37686036E7032719E7BB
:10C480004FF48841C3F23571F4F78CFA4AF208315F
:10C49000C2F685610446F4F785FA01462860204615
:10C4A000F4F77EFA4AF20831C2F68561F4F77AFAB7
:10C4B0004FF0FF37686018E74FF42341C2F68561FB
:10C4C0005846F4F777FB804641462046F4F768FA71
:10C4D000814649462046F4F763FA4146F4F760FA8C
:10C4E00043F232110446C2F28D415846F4F762FB22
:10C4F0002146F4F755FA8246514648464DE700BFBB
:10C50000801A0108001A010820F00042B2F1FF4F22
:10C51000F8B50446034646D2002A42D0002852DB32
:10C52000C415B2F5000F09D210F4000553D15B0019
:10C5300001351902FBD5C5F10100241823F07F4114
:10C540007F3C21F40006E20746F4000048BF4000AB
:10C5500043004FF08072002760109A423C462CDD69
:10C560005B004FF400021825A61851089E4205F101
:10C57000FF3502DCB4189B1BBF185B0062189A429F
:10C5800002DC9B1A54187F185B004A08013DEBD16E
:10C5900013B107F001017F187C1004F17C5303EB09
:10C5A000C0542046F8BD0146F4F704FB014620467E
:10C5B000F4F7F8F904462046F8BD4FF0007403F193
:10C5C0007F431746CCE70146F4F7EAF90146F4F752
:10C5D000A5FB0446E5E70120AFE700BF2DE9F843DE
:10C5E00020F00046B6F1485F05460F465BDAF4F7E7
:10C5F000A7FC002800F0CA8029462846F4F7DAFA9A
:10C600004DF24E71CAF647510446F4F7D3FA47F299
:10C61000F641C3F20F11F4F7C5F92146F4F7CAFA4F
:10C620004FF27C21C3F29341F4F7BAF92146F4F7B3
:10C63000C1FA40F60151C3F2D071F4F7B3F92146C3
:10C64000F4F7B8FA40F66131C3F6B621F4F7A8F969
:10C650002146F4F7AFFA4AF6AB21C3F62A51F4F7B4
:10C66000A1F92146F4F7A6FA804620464FF07C5106
:10C67000F4F7A0FA414606462046F4F79BFA3946FD
:10C6800004462846F4F796FA01462046F4F788F95E
:10C6900001463046F4F784F901464FF07E50F4F736
:10C6A0007FF9BDE8F8830146F4F784FA4DF24E7144
:10C6B000CAF647510446F4F77DFA47F2F641C3F251
:10C6C0000F11F4F76FF92146F4F774FA4FF27C2159
:10C6D000C3F29341F4F764F92146F4F76BFA40F69C
:10C6E0000151C3F2D071F4F75DF92146F4F762FA13
:10C6F00040F66131C3F6B621F4F752F92146F4F75A
:10C7000059FA4AF6AB21C3F62A51F4F74BF9214600
:10C71000F4F750FA49F69913C3F699639E4280469E
:10C72000A3DD0020C3F64870864227DC06F17F4671
:10C730004FF07E503146F4F733F9814620464FF0F2
:10C740007C51F4F737FA3146F4F72AF941460646A8
:10C750002046F4F72FFA394604462846F4F72AFA19
:10C7600001462046F4F71CF901463046F4F718F963
:10C7700001464846F4F714F9BDE8F8834FF0000984
:10C780000026C3F63879C3F69066D7E74FF07E509F
:10C79000BDE8F8832DE9F04FDFB00C930C9D224BE0
:10C7A000689C0A91691ED61E48BF161D834653F821
:10C7B0002400F71027EAE7730890049104980D937A
:10C7C000089DDC43DDF834C002EBC4024119079236
:10C7D000C0EB0C0750D47E18699BC7EB06090136E5
:10C7E000002F03EB870522AC09F0010AC0F2FE829C
:10C7F0002868F4F78BF90137B74220604FF004083E
:10C800003AD0BAF1000F26D0002FC0F2F18255F8CD
:10C810000800F4F77BF90137B74244F8080008F143
:10C82000040818D128E000BF981D010855F8080039
:10C83000F4F76CF9013708F1040944F8080013D43F
:10C8400055F80900F4F762F90137B74244F80900D6
:10C8500009F1040810D0002FE8DA0020013708F1B0
:10C86000040944F80800EBD501370020B74244F82A
:10C87000090009F10408EED1089A002AC0F24585A2
:10C8800008990C9E8D004AAB5C19039549AF029440
:10C890004FEA860A049A002AC0F296820DF18808AF
:10C8A00008EB860555F8041CAAF10403DBF8000028
:10C8B000C3F38009F4F77EF901460020F4F772F81B
:10C8C0000424043D544580462BD0B9F1000F0DD00F
:10C8D00055F8041DDBF80400F4F76CF901464046F6
:10C8E000F4F760F80824544580461AD055F8041C23
:10C8F0005BF80400F4F75EF901464046F4F752F89D
:10C900000434804655F8081C5BF80400F4F752F92B
:10C9100001464046F4F746F80434083D5445804645
:10C92000E4D1029847F8048F01368742B2D1039FC1
:10C930000EA9CE190996089EB2005EAB9D18002E76
:10C94000029255F8509C7DDD0DF5947C4FF06E51B0
:10C9500048460DACA7180CEB0205F4F72BF9F4F7D9
:10C96000EFFAF4F7D3F84FF087410190F4F722F98A
:10C9700001464846F4F714F8F4F7E2FA0EAC2060EA
:10C980000198014655F8040DF4F70CF8BC428146B5
:10C99000C7F3800156D0E9B14FF06E51F4F70AF9B0
:10C9A000F4F7CEFAF4F7B2F84FF087410190F4F7BC
:10C9B00001F901464846F3F7F3FFF4F7C1FA019A8B
:10C9C0000FAC2060114655F8040DF3F7EBFFBC42A5
:10C9D000814637D04FF06E514846F4F7EBF8F4F744
:10C9E000AFFAF4F793F84FF087418046F4F7E2F896
:10C9F00001464846F3F7D4FFF4F7A2FA41466060D7
:10CA000055F8040DF3F7CEFF4FF06E518146F4F761
:10CA1000D1F8F4F795FAF4F779F84FF087418046AA
:10CA2000F4F7C8F801464846F3F7BAFFF4F788FA76
:10CA30004146A06055F8040DF3F7B4FF0834BC423A
:10CA40008146C7D10799484600F0A2FE4FF07851C1
:10CA50000546F4F7AFF800F025FE4FF08241F4F7F9
:10CA6000A9F801462846F3F79BFF0746F4F768FA52
:10CA70008146F4F74BF801463846F3F791FF0799E2
:10CA80000746002940F33981721E0EAC079D54F809
:10CA90002230C5F1080043FA00F101FA00F0C5F1B7
:10CAA00007041B1A43FA04F40DF1380C89444CF8BE
:10CAB0002230002C55DD002E09F1010940F394814C
:10CAC000029D0EABDDF808C053F8042B281F0DF1B2
:10CAD000380E00250EEB0C01C0F3800022B1C2F528
:10CAE000807243F8042C01258B4226D060B10F9A46
:10CAF0000433002D40F0F38022B1C2F5807543F875
:10CB0000045C01258B4218D053F8042B002D40F013
:10CB1000EC80C2F5807012B143F8040C012553F883
:10CB2000042B002D40F0DB80C2F58070002AE9D094
:10CB300001258B4243F8040CE6D1079900290DDD4D
:10CB4000012900F0E280022908D1701E0DF1380E93
:10CB50005EF8202002F03F034EF82030022C00F057
:10CB6000E08038460021F4F7B9F9002800F0F3809E
:10CB70000898751EA84225DC029B0DF1380E0EEBBD
:10CB800003010B46DDF824C053F8042DCCEB010063
:10CB9000011F6345C1F3800011D030B153F8041D6B
:10CBA000DDF824E00A43734509D0099F53F8040DCA
:10CBB00053F8041D0243BB4242EA0102F6D1002AA7
:10CBC00040F01A81089F0EAD781E55F82020002AEB
:10CBD00040F0108105EB8004012354F8041D01335B
:10CBE0000029FAD0F018771C87420B9075DCDDF82D
:10CBF00010E00D9D0B9B0C9C0EEB0702DDF808C0AE
:10CC0000699F991B06EB05094AA8A61922AB07EBF9
:10CC1000890900EB0C05571C8A0003EB860102957D
:10CC200006920591002659F8040FF3F76FFF059C53
:10CC3000A051049800285EDB22AD05EB8702AAF123
:10CC40000403C3F3800452F8041CDBF800000394CF
:10CC5000141FF3F7AFFF01460020F3F7A3FE4FF0D8
:10CC60000408D04505462DD0039971B154F8041D30
:10CC7000DBF80400F3F79EFF01462846F3F792FE27
:10CC80004FF00808D04505461CD054F8041C5BF84A
:10CC90000800F3F78FFF01462846F3F783FE08F1FB
:10CCA0000408054654F8081C5BF80800F3F782FFF7
:10CCB00001462846F3F776FE08F10408083CD04503
:10CCC0000546E2D1DDF808E0069804364EF8045F28
:10CCD00001378642CDF808E0A5D10B9E2CE6C2F1C3
:10CCE000FF0243F8042C01250CE7C2F1FF0543F8CD
:10CCF000045C012513E70025E4E75ED1701E0DF109
:10CD0000380E5EF820301C12D3E6711E0DF1380C7F
:10CD10005CF82100022C00F07F024CF821207FF407
:10CD200020AF39464FF07E50F3F73AFE0746002D0C
:10CD30003FF417AF07994FF07E5000F029FD0146F0
:10CD40003846F3F72DFE074638460021F4F7C6F8BB
:10CD500000287FF40DAF0294079C38466142CDF85D
:10CD6000109000F015FD4FF087410546F4F7D4F818
:10CD7000002800F0D2824FF06E512846F3F71AFFD8
:10CD8000F4F7DEF8F3F7C2FE4FF087410746F3F7FA
:10CD900011FF01462846F3F703FEF4F7D1F80EA978
:10CDA00041F826003846F4F7CBF8079A01360832E6
:10CDB0000EAC079244F8260034E04FF07C51F4F7B3
:10CDC000ABF858B90024CCE64FF00008029847F8B9
:10CDD000048F013687427FF45DADA8E50224002E62
:10CDE00009F101093FF76CAE0025A6E6002002E537
:10CDF000002010E50123F5E6079A0EAE56F825301F
:10CE0000083ACDF8109002940792002B40F08E82E1
:10CE100006EB85042E4654F8045D013E083A002DC9
:10CE2000F9D007924FF07E50079900F0B1FC002E28
:10CE30000446C0F2AC804FEA860AC6EB867B0EAF92
:10CE40004FEA8B095744C9F100034AA9386801EB3E
:10CE50000A08C3F3800BF3F759FE2146F3F7AAFE45
:10CE60004FF06E51C8F800002046F3F7A3FEA9F179
:10CE700004096FF0030ACA45054631D0BBF1000F23
:10CE80000BD057F8040CF3F741FE2946F3F792FE56
:10CE90006FF0070A48F8040C1AE057F80A00F3F795
:10CEA00035FE2946F3F786FE4FF06E5148F80A002A
:10CEB0002846F3F77FFEAAF1040405463859F3F734
:10CEC00025FE2946F3F776FEAAF1080A48F8040081
:10CED00028464FF06E51F3F76DFECA450546DCD18A
:10CEE000701CDFF84C94DDF820A003900027059615
:10CEF000BAF1000FC0F20582002FC0F202820026B4
:10CF000000241AF0010F354620D0D8F80010D9F8C7
:10CF10000000F3F74FFE01462046F3F743FD0125DD
:10CF2000AA45044626DB0426BD420FDD22E0BB45B0
:10CF300020DC58F8021059F80200F3F73BFE0146D6
:10CF40002046F3F72FFDBD42044613DC58F80610C7
:10CF500059F80600F3F72EFE01462046F3F722FDAE
:10CF600005F1010B06F104020235DA45044602F12F
:10CF70000406DCDA5EABDDF80CC003EB8701013799
:10CF8000674541F8A04CA8F10408B1D1059E689C02
:10CF9000032C16D8DFE814F085011F011F011B00C8
:10CFA00000230299002900F00B81379C369804F188
:10CFB00000420A9C00F1004503F1004325606260D5
:10CFC000A360049D05F007005FB0BDE8F08F002E60
:10CFD000E6DD06F1FF3836AF07EB88094D4655F818
:10CFE00004290DF1D40AD5F808B01046594601922B
:10CFF000F3F7D8FC804641460198F3F7D1FC01468F
:10D000005846F3F7CFFC5545C9F38003A860C5F82F
:10D01000048044D0BBB155F80429D5F808B01046B7
:10D0200059460192F3F7BEFC0199804608464146F5
:10D03000F3F7B6FC01465846F3F7B4FC5545C5F87E
:10D040000480A8602BD02C4654F80439D4F808B0DA
:10D05000184659460193F3F7A5FC804641460198CE
:10D06000F3F79EFC01465846F3F79CFCC4F8048095
:10D07000A06055F804BC251FD5F8088058464146E5
:10D08000F3F790FC044621465846F3F789FC014625
:10D090004046F3F787FC55456C60A860D3D1012E5C
:10D0A0007FF77EAF4D4655F804B9C7EB090ED5F8AA
:10D0B00008A058465146AEF10409F3F773FC8046C8
:10D0C00041465846F3F76CFC01465046F3F76AFCBC
:10D0D000BD42C9F38009C5F80480A86043D0B9F106
:10D0E000000F15D055F804A9D5F8089050464946C8
:10D0F000F3F758FC804641465046F3F751FC014691
:10D100004846F3F74FFCBD42C5F80480A8602AD01A
:10D110002C4654F804A9D4F8089050464946F3F731
:10D1200041FC804641465046F3F73AFC01464846EA
:10D13000F3F738FCC4F80480A06055F8049C251F60
:10D14000D5F8088048464146F3F72CFC04462146B2
:10D150004846F3F725FC01464046F3F723FCBD4261
:10D160006C60A860D4D1013607EB860708353E46CF
:10D170007A1B131F56F8041D0020C3F38007F3F732
:10D1800011FCAE4203463FF40CAF3FB156F8041D0C
:10D19000F3F708FCAE4203463FF403AF184656F8D7
:10D1A000041C341FF3F7FEFB083E54F8041CF3F78D
:10D1B000F9FBAE42F3D10299034600297FF4F5AEA4
:10D1C000DDF828C036993798CCF80010CCF8040068
:10D1D000CCF80830F5E60023002E29DB36AF751CAD
:10D1E00007EB85042546E21B55F8041DA2F1040E49
:10D1F0000020CEF38008F3F7D5FBBD42034617D0DD
:10D20000B8F1000F06D055F8041DF3F7CBFBBD4273
:10D2100003460DD0184655F8041C2C1FF3F7C2FB2B
:10D22000083D54F8041CF3F7BDFBBD42F3D103469F
:10D230000299002967D003F10040DDF828C01946A3
:10D24000CCF800003698F3F7ABFB002E034621DD47
:10D2500036AF07EB8606F51B2A1F3799C2F3800706
:10D26000F3F7A0FB37ACB442034613D037B1616883
:10D27000F3F798FB38ACB44203460BD0184654F889
:10D28000041FF3F78FFB54F8041FF3F78BFBB44232
:10D29000F5D10346029909B103F100430A9C63608A
:10D2A0008FE6002E40DB36AF013607EB86000546E1
:10D2B000C21B55F8041D0020141FF3F773FBBD4279
:10D2C000C4F38006034615D036B155F8041DF3F7B4
:10D2D00069FBBD4203460DD0184655F8041C2C1FAF
:10D2E000F3F760FB083D54F8041CF3F75BFBBD4209
:10D2F000F3D10346029909B103F100430A9C23606C
:10D300005FE6002436E6184697E7DDF830E0900047
:10D3100003904FEA8E0AFFF70ABB2846F3F710FE88
:10D320000EAB43F826007DE50023E3E72E4679E5C2
:10D33000A41D01082DE9F84320F00043B3F1485F34
:10D3400004460F46904603DAF3F7FAFD002859D059
:10D3500021462046F3F72EFC21460546F3F72AFC2A
:10D360004CF6D311C2F62E7106462846F3F722FC7E
:10D3700042F63471C3F2D721F3F712FB2946F3F7D3
:10D3800019FC4EF61B71C3F23861F3F70BFB29460B
:10D39000F3F710FC40F60151C3F65011F3F700FB10
:10D3A0002946F3F707FC48F68901C3F60841F3F76D
:10D3B000F9FA8146B8F1000F27D04FF07C5138467A
:10D3C000F3F7F8FB494680463046F3F7F3FB014696
:10D3D0004046F3F7E5FA2946F3F7ECFB3946F3F755
:10D3E000DFFA4AF6AB210546C3F62A613046F3F769
:10D3F000E1FB01462846F3F7D5FA01462046F3F74C
:10D40000CFFA04462046BDE8F88301462846F3F7E4
:10D41000D1FB4AF6AB21C3F62A61F3F7C1FA3146D4
:10D42000F3F7C8FB01462046F3F7BCFA0446204652
:10D43000BDE8F8830020704700210020C7F6F8718E
:10D44000704700BF2DE9F04120F00045B5F1A14F34
:10D45000044606460DDBB5F1FF4F00F39C80002823
:10D4600040F6DB7440F3D480C3F6C9742046BDE8AF
:10D47000F0814FF6FF73C3F6DF639D4200F3A28095
:10D48000B5F1445FC0F28E804FF0FF372146204651
:10D49000F3F790FB01468046F3F78CFB46F6D71175
:10D4A000C3F685410546F3F785FB4DF65921C3F6D2
:10D4B0004B51F3F777FA2946F3F77CFB46F6353103
:10D4C000C3F68851F3F76EFA2946F3F773FB42F679
:10D4D0006E61C3F6BA51F3F765FA2946F3F76AFBB2
:10D4E00044F62511C3F61261F3F75CFA2946F3F707
:10D4F00061FB4AF6AB21C3F6AA61F3F753FA414642
:10D50000F3F758FB4AF221218046CBF61551284605
:10D51000F3F750FB4FF26B11C3F66E51F3F740FA7D
:10D520002946F3F747FB48F29571C3F69D51F3F78F
:10D5300037FA2946F3F73EFB48F63861C3F6E35164
:10D54000F3F72EFA2946F3F735FB4CF6CD41C3F637
:10D550004C61F3F725FA2946F3F72CFB7B1C0146B7
:10D56000404658D0F3F71EFA2146F3F723FB494B08
:10D5700053F82710F3F714FA2146F3F711FA01468E
:10D58000454850F82700F3F70BFA002E3DDB044620
:10D590002046BDE8F0810146F3F704FA0446204630
:10D5A000BDE8F0814FF2CA21C7F24911F3F7FAF949
:10D5B0004FF07E51F3F7BAFC00283FF465AF2046E8
:10D5C000BDE8F08100F06AF84FF6FF71C3F697717D
:10D5D0008D4204464FF6FF7228DCC3F62F72954247
:10D5E00046DC0146F3F7DEF94FF07E51F3F7D8F948
:10D5F0004FF0804105462046F3F7D4F9014628460E
:10D60000F3F78CFB0027044640E700F100442DE7C8
:10D61000CBF6C9742AE7F3F7C5F92146F3F7CAFA3E
:10D6200001462046F3F7BCF904461FE7C4F21B028B
:10D63000954214DC4FF07F51F3F7B2F94FF07F5170
:10D6400005462046F3F7B6FA4FF07E51F3F7AAF9F4
:10D6500001462846F3F762FB0227044616E700203E
:10D660002146CBF68070F3F759FB032704460DE7FC
:10D670004FF07E51F3F794F94FF07E510746204664
:10D68000F3F790F901463846F3F748FB01270446C3
:10D69000FCE600BFD01D0108E01D010820F000409D
:10D6A000704700BFF8B520F00046F50D7F3D162D00
:10D6B000014604461BDC002D074620DB4FF6FF73B6
:10D6C000C0F27F0343FA05F606420ED04FF2CA219C
:10D6D000C7F24911F3F766F90021F3F727FC18B1F7
:10D6E000002C1BDB27EA060421460846F8BDB6F1EC
:10D6F000FF4FFAD3F3F756F901460846F8BD4FF24B
:10D70000CA21C7F24911F3F74DF90021F3F70EFCD6
:10D710000028E9D0002C07DB0024E5E74FF40000E7
:10D7200040FA05F56719DDE70021CBF68071002E80
:10D7300018BF0C46D8E700BF08B902207047B0F107
:10D74000004FFAD0A0F500026FF001439A4201D8D1
:10D750000420704700F1FF419942F9D94FF6FE735A
:10D76000421EC0F27F039A4201D80320704700F1A5
:10D7700000414A1E9A42F8D9B0F1FF4F05D010F58A
:10D78000000F14BF0020012070470120704700BF28
:10D7900038B530F00044034602460D460FD0B4F1D0
:10D7A000FF4F0ED2B4F5000F11D3E40D6419FE2C17
:10D7B00033DC002C1BDD22F0FF4141EAC453184644
:10D7C00038BD0146F3F7EEF80346184638BD4FF072
:10D7D0009841F3F7EFF943F6B041CFF6FF718D4270
:10D7E000034612DBC0F3C7540246193CDEE714F1CE
:10D7F000160F21DA4CF25032954219460EDC44F2F3
:10D800006020C0F6A25000F023F844F26021C0F678
:10D81000A251F3F7CFF90346D1E719464FF2CA20D8
:10D82000C7F2491000F014F84FF2CA21C7F24911AB
:10D83000F3F7C0F90346C2E722F0FF4304F11900F1
:10D8400043EAC0504FF04C51F3F7B4F90346B6E742
:10D8500001F0004120F00040084370472DE9F041FD
:10D86000274C84B025680746D5F84841002C41D0A4
:10D8700066681F2E1CDD234810B94FF0FF301FE0F3
:10D880004FF4C870039102920193AFF300800399A3
:10D890000446029A019B0028EFD0D5F84861002089
:10D8A00060602660C5F84841C4F88801C4F88C015E
:10D8B000656847B9A81C013544F820106560002050
:10D8C00004B0BDE8F081012000FA05F0D4F88861C9
:10D8D00004EB85080643022FC8F88820C4F8886145
:10D8E000C8F80831E6D1D4F88C3143EA0002C4F814
:10D8F0008C21DFE705F5A674C5F84841B8E700BFFD
:10D90000F81E01080000000000210A2201F0C4BD39
:10D910002DE9F84FDDF828B081468A4698469AB13D
:10D9200093B11646002503E00FD0651CAE420BD91B
:10D930007419640808FB04A748463946D8470028EC
:10D94000F2DA2646AE42F3D800273846BDE8F88F13
:10D9500040F2C853C2F2000318687047114B124AD4
:10D9600070B5981A831018D0591E02EB83040D4627
:10D9700054F8042D01F00106904775B126B154F812
:10D98000040D8047013D08D054F8043D9847013DFF
:10D9900054F8041D8847013DF6D1BDE8704004F0FD
:10D9A000B3BA00BF201F01081C1F0108F8B5204FA3
:10D9B000204C381B871017D07A1E2368012502F0EF
:10D9C00001069847AF420FD02EB154F8041F02252C
:10D9D0008847AF4208D0606880470235A268261D9C
:10D9E00090470834AF42F6D1134F144C04F086FA36
:10D9F0003B1B9F1018D07D1E216805F001060125F4
:10DA00008847AF4211D02EB154F8040F0225804749
:10DA1000AF420BD0626890470235A368261D984735
:10DA20000834AF42F6D1F8BDF8BDF8BDF8BD00BF6F
:10DA3000141F0108141F01081C1F0108141F0108EE
:10DA40000F2A2DE9F00340F2A18041EA00039B0771
:10DA500040F09E800C68A2F1100504604B68AC4653
:10DA600043608C68BCF10F0F8460CC68C5F300156F
:10DA7000C46000F1100301F110042BD975B12568C1
:10DA8000ACF1100C1D6065685D60A5689D60E5687F
:10DA90001034DD601033BCF10F0F1BD9276804F17F
:10DAA00010061F60676803F110055F60A768ACF19E
:10DAB000200C9F60E768DF6024691C61776806F1CD
:10DAC00010046F60B7682033AF60F668BCF10F0FC9
:10DAD000EE60E3D8A2F1100828F00F0302F00F0463
:10DAE00003F1100C032C00EB0C0301EB0C0851D9D3
:10DAF000211F4FEA9109444608EB890C54F8046B46
:10DB0000C8EB0C010CF1040C1D46644545F8046B90
:10DB1000C1F3800112D029B154F8041B644545F8C3
:10DB2000041B0BD0274657F8041B2E4646F8041B4F
:10DB300064686C603C1D351D6445F3D109F1010C2E
:10DB40004FEA8C0902F0030208EB09014B44D2B101
:10DB50000D789A18DC4303F8015B1419934204F022
:10DB6000010410D02CB111F8014F03F8014B93427E
:10DB700009D04D781C4604F8015B8D7802315D7048
:10DB8000631C9342F5D1BDE8F00370470346DEE71E
:10DB90000346DDE741462246D9E700BFF0B48407DB
:10DBA000034600F08D80541E002A00F08780E507B0
:10DBB000CEB211D41A4602F8016B134615469207ED
:10DBC00010D0621E002C79D003F8016B14469A071E
:10DBD0001D4607D0013CEDE7034603F8016B9A07A9
:10DBE0001D46F7D1032C52D9CEB246EA06270F2C98
:10DBF00047EA07432DD9A4F1100217460F2FC2F3AD
:10DC000000162B606B60AB60EB6005F1100216D95B
:10DC10003EB1103F136053609360D36010320F2FFA
:10DC20000DD9203F02F11006136053609360D3605A
:10DC3000136153619361D36120320F2FF1D8A4F1A6
:10DC4000100222F00F0204F00F041032032C1544CE
:10DC50001DD9271F3E462A46032E42F8043BC7F330
:10DC600080070DD927B1043E032E42F8043B07D9A3
:10DC7000174647F8043B083E53603A1D032EF7D879
:10DC8000231F23F00302131D04F00304ED18ACB1AD
:10DC9000C9B2EA432C1905F8011BA318A54203F0E9
:10DCA00001020BD01AB105F8011BA54206D02B4684
:10DCB00003F8011B69705D1CA542F8D1F0BC7047E8
:10DCC000054614468EE700BF2DE9F04F89B0144693
:10DCD0008046019202EB4202A508500004F00304C2
:10DCE00018F0030F0291994603950694079040F0AF
:10DCF000D6800699002940F05A82019A151F18BF54
:10DD000001250095029D062D40F2CF80DDF808C068
:10DD1000019F64464FEA5C06072C07FB068A40F029
:10DD2000E281DDF81CC008EB0C06009B002B40F0E4
:10DD3000FB81D8F80010DAF80030C8F80030CAF8D3
:10DD400000100198DDF804A008EB00054946002208
:10DD500005952F4604953446CAF1000A91460D46B2
:10DD6000A74240F213812B464D469946002D00F004
:10DD7000C183DDF810B00299CBEB070AC8EB0B02A8
:10DD80005245A8BF5246DDF804C0002A0CFB018BA7
:10DD90003ADD009BB91A022B404640F0D28210F8BF
:10DDA000015B91F800C0029500F801CCDDF808C0D5
:10DDB0000B468A18CD4303F801CBAD1801309342CE
:10DDC00005F0010520D04DB110F8015C497800F84C
:10DDD000011C03F8015B0130934215D0014611F894
:10DDE000015C93F800C0184601F801CC00F8015B13
:10DDF00011F8015B93F801C0034601F801CC03F868
:10DE0000015B01319342EAD10199C6EB0B03341B4C
:10DE1000581AA04228BF204600282FDD009DC0EBE5
:10DE20000B02022D40F053821578FB4339783818E5
:10DE300007F8015B874203EB0005134603F8011B5B
:10DE400005F001011AD039B155783A7807F8015B2D
:10DE5000874203F8012B11D03D781E781A463946C7
:10DE600001F8016B02F8015B5B787D780F4607F8DB
:10DE7000013B8742134603F8015BEDD1019D5545F7
:10DE8000C0F08C81DDF804C0A4457CD2C4EB0B0843
:10DE900018F0030FB4FBFCF402943FF42AAF029D88
:10DEA0000223062D00933FF631AFDDF804C00CFBD2
:10DEB000058A08EB0C01514565D2019CDDF804B0E0
:10DEC00065420434009E02940091CDF810A04F46A4
:10DED000DDF80090C14509D84DE0D9F8000021686F
:10DEE000C9F8001020604445A14644D909EB050457
:10DEF00020464946B84700283DDD002EEDD0012ED2
:10DF000000F0A7831BF804E094F800900BF1FF31B8
:10DF10000BEB04000246234601F0010C002902F835
:10DF2000019B03F801EBDEDDBCF1000F09D0407866
:10DF300094F801E00139002902F801EB03F8010B24
:10DF4000D1DD93F800A092F80090944618460CF8A2
:10DF500001AB00F8019B92F801E093F801A00239AF
:10DF600062460346002902F801AB03F801EBE8DC46
:10DF70004445A146BAD8DDF800C0049BDC449C456A
:10DF8000CDF800C0A4D309B0BDE8F08F38464146B3
:10DF9000A84700280BDC8CE02068326822603060E3
:10DFA00056444FF001095444A7423FF6DCAE2046E8
:10DFB0004146A8470028C0F29A83F4D1009B002B69
:10DFC000EAD00099012935D0DDF804E0207896F8F0
:10DFD00000C00EF1FF312246334601F0010900294D
:10DFE00002F801CB03F8010BDADDB9F1000F09D01B
:10DFF000107893F800C00139002902F801CB03F82A
:10E00000010BCDDD93F800B092F800E0944618467D
:10E010000CF801BB00F801EB92F8019093F801B005
:10E02000023962460346002902F801BB03F8019B4E
:10E03000E8DCB5E721463346DDF80CE053F8042B65
:10E0400051F8040B0EF1FF3C41F8042C0CF00102D6
:10E0500043F8040C04310433BCF1000FA0DD72B1AD
:10E0600051F8040C53F8042C0CF1FF3C41F8042C3B
:10E0700043F8040C04310433BCF1000F90DD53F875
:10E08000042C51F8049C084641F8042C1A4643F825
:10E09000049C50F8043B52F8041BACF1020C40F80D
:10E0A000041C011D42F8043C131DBCF1000FE6DC0A
:10E0B00076E714D1009A002A7CD104983B68026864
:10E0C000DDF810C0CCF800303A60DDF810E0DDF883
:10E0D00004900EEB090CCDF810C04FF00109DDF8EB
:10E0E00004E077443CE602980199431E282801FB8E
:10E0F000038600F2AB803446454651462846C84761
:10E10000002821465046C0F29580C84700283FF7B6
:10E110000CAE28462146C847009B34EA200A28BF97
:10E12000AA46002B3FF405AE00994246012900F0B3
:10E130004781DDF804C012F8015B9AF800400CF149
:10E14000FF3102F8014C574601F00100013200296D
:10E1500007F8015B7FF7F5AD58B13D7812F8013C47
:10E16000013902F8015C0132002907F8013B7FF711
:10E17000E8AD12F8014C3B78384602F8013C00F853
:10E18000014B12F8014B7D78023902F8015C074619
:10E190000132002907F8014BEBDCD2E5019D404636
:10E1A000BAFBF5F12A464B46FFF78EFD6AE60224DC
:10E1B0000094A7E50098012800F03B81DDF810E00D
:10E1C000DDF804B039789EF800000BF1FF3B724691
:10E1D00002F8011B3B460BF00101BBF1000F03F8F5
:10E1E000010B7FF772AF59B1117818780BF1FF3B33
:10E1F000BBF1000F02F8010B03F8011B7FF765AFBD
:10E2000092F800C093F800901046194600F8019B60
:10E2100001F801CB92F801E093F801C0ABF1020BD9
:10E2200002460B46BBF1000F02F801CB03F801EBED
:10E23000E6DC4AE7C8470028FFF677AD28462146C6
:10E24000C84735EA200A28BFA2466EE5019AC408ED
:10E2500002FB04F408EB04054FEA440B2946404650
:10E26000CDF810B0C84708EB0B0700283946284600
:10E27000C0F23481C847002840F33182C4F1000B5A
:10E280000AEB0B0751463846C8475444002821463C
:10E290005046C0F21781C847002840F318820498FE
:10E2A00006EB0B04371A21463846C847002831468A
:10E2B0002046C0F2FB80C84700283FF71EAF384613
:10E2C0003146C84736EA200428BF3C4615E73946A0
:10E2D000134653F8042B51F8045B8008013841F8C9
:10E2E000042C00F0010243F8045C043104330028DC
:10E2F0007FF7C4AD6AB151F8045C53F8042C0138BF
:10E3000041F8042C43F8045C0431043300287FF7FF
:10E31000B5AD51F8046C53F8042C0D4641F8042CAB
:10E3200043F8046C1A4652F8041B55F8046B023883
:10E3300045F8041C131D291D002842F8046CE8DC74
:10E340009CE50B4653F8045B50F8041B920802F15D
:10E35000FF3C40F8045C021D0CF0010543F8041C6E
:10E360000433BCF1000F7FF74FAD7DB152F8041CB0
:10E3700053F8040C0CF1FF3C42F8040C43F8041C65
:10E3800004320433BCF1000F7FF73EAD52F8045C59
:10E3900053F8040C114642F8040C43F8045C184688
:10E3A00050F8042B51F8045BACF1020C41F8042C3A
:10E3B000031D0A1DBCF1000F40F8045CE6DC23E5F8
:10E3C0005746039952F8043B57F8040B013942F8B9
:10E3D000040C01F0010447F8043C04323B1D002901
:10E3E0007FF7AFAC6CB152F8045C53F8047C013990
:10E3F00042F8047C43F8045C0432043300297FF7BC
:10E40000A0AC52F8045C53F8040C144642F8040C17
:10E410001F4643F8045C57F8042B54F8045B023998
:10E4200044F8042C3B1D221D002947F8045CE8DC5D
:10E4300087E404993B46DDF80C9053F8042B51F81F
:10E4400004EB09F1FF3041F8042C00F0010243F81D
:10E4500004EC0431043300287FF737AE6AB151F879
:10E4600004CC53F8042C013841F8042C43F804CCB4
:10E470000431043300287FF728AE53F8042C51F8F8
:10E4800004EC894641F8042C1A4643F804EC59F888
:10E49000043B52F8041B023849F8041C42F8043CBF
:10E4A000131D002809F10401E7DC0EE6C847002827
:10E4B000FFF623AE38463146C84737EA200428BF66
:10E4C00034461AE6C8470028FFF6E9AE384621462A
:10E4D000C84737EA200A28BFA246E0E6C847002816
:10E4E000FFF6CCAE40463946C84738EA200528BF7B
:10E4F0003D46C3E60298019C059D04FB008A5545F4
:10E50000BFF441AD019FDDF814B03C1D009ECDF875
:10E5100000B0DDF804B07D420494CDF808A01F4699
:10E52000DDF80090C84509D34CE0D9F80000216817
:10E53000C9F8001020604445A14643D909EB050401
:10E5400020464946B84700283CDD002EEDD0012E7C
:10E5500041D01BF804E094F800900BF1FF310BEB75
:10E5600004000246234601F0010C002902F8019B39
:10E5700003F801EBDFDDBCF1000F09D0407894F81F
:10E5800001E00139002902F801EB03F8010BD2DDAB
:10E5900093F800A092F80090944618460CF801AB4E
:10E5A00000F8019B92F801E093F801A0023962465D
:10E5B0000346002902F801AB03F801EBE8DC44450F
:10E5C000A146BBD8DDF800C0029BDC449C45CDF8D9
:10E5D00000C0A5D3D7E4DDF81090234609EB040270
:10E5E000DDF80CE053F8041B52F804CC0EF1FF30B8
:10E5F00042F8041C00F0010143F804CC0432043357
:10E60000002898DD61B152F8049C53F8041C0138CD
:10E6100042F8041C43F8049C0432043300288ADDC9
:10E6200053F8041C52F804EC944642F8041C1946B2
:10E6300043F804EC5CF8043B51F8042B02384CF826
:10E64000042C41F8043C0B1D00280CF10402E7DC0B
:10E6500071E7029A23461219DDF80C9053F8041B57
:10E6600052F804CC09F1FF3042F8041C00F001011B
:10E6700043F804CC0432043300287FF734AC69B18A
:10E6800052F804EC53F8041C013842F8041C43F817
:10E6900004EC0432043300287FF725AC53F8041C43
:10E6A00052F8049C944642F8041C194643F8049C12
:10E6B0005CF8043B51F8042B02384CF8042C41F868
:10E6C000043C0B1D00280CF10402E7DC0BE4384687
:10E6D0002146C84734EA200A28BFBA46DFE540464B
:10E6E0003946C84737EA200528BF4546C6E5A74250
:10E6F0003FF639AB009B63B9386822683A60206006
:10E70000DDF804E04FF001097744CEEB0404FFF795
:10E7100027BB0098012833D0DDF80490207897F8C3
:10E7200000E009F1FF313A4602F8010B234601F0FF
:10E730000100002903F801EBE2DD48B1107893F8FD
:10E7400000C00139002902F801CB03F8010BD7DD25
:10E7500093F800B092F800E0944618460CF801BB1C
:10E7600000F801EB92F8019093F801B0023962468B
:10E770000346002902F801BB03F8019BE8DCBFE770
:10E7800039462346DDF80CE053F8042B51F8040B0E
:10E790000EF1FF3C41F8042C0CF0010243F8040C8C
:10E7A00004310433BCF1000FAADD72B151F8040C3E
:10E7B00053F8042C0CF1FF3C41F8042C43F8040CF2
:10E7C00004310433BCF1000F9ADD53F8042C51F8E6
:10E7D000049C084641F8042C1A4643F8049C50F85F
:10E7E000043B52F8041BACF1020C40F8041C011D60
:10E7F00042F8043C131DBCF1000FE6DC80E700BFCB
:10E80000830770B5064614D10368A3F1013222EAEA
:10E81000030010F0803F0CD1331D1A4653F8044B0F
:10E82000A4F1013525EA040414F0803FF5D0104628
:10E8300000E0304603782BB1421C147810460132B8
:10E84000002CFAD100F080F8304670BDC9B2F0B4A7
:10E8500000294BD082070FD00278002A71D0914254
:10E8600042D0431C05E013F8012B002A3BD0914213
:10E870003AD09A071846F6D1036841EA0127A3F176
:10E88000013222EA030212F0803F47EA07471CD117
:10E890007B40A3F1013222EA030313F0803F14D13D
:10E8A000021D02E014F0803F0FD1104652F8043BE5
:10E8B000A3F1013687EA030426EA0303A4F1013534
:10E8C00013F0803F25EA0404ECD00278002A38D007
:10E8D000914209D0431C01E0914205D0184613F83B
:10E8E000012B002AF8D11046F0BC704783070BD0EB
:10E8F0000278002AF8D0431C03E001780133002994
:10E90000F2D099071846F8D10168A1F1013323EA42
:10E91000010212F0803F0AD1031D184653F8041B70
:10E92000A1F1013424EA010212F0803FF5D003780E
:10E93000002BD9D0421C1178104601320029FAD19F
:10E94000D2E71046D0E700BF80EA0102844612F009
:10E95000030F4FD111F0030F32D14DF8044D11F0D8
:10E96000040F51F8043B0BD0A3F101329A4312F08B
:10E97000803F04BF4CF8043B51F8043B16D100BF64
:10E9800051F8044BA3F101329A4312F0803FA4F1F5
:10E9900001320BD14CF8043BA24312F0803F04BF7C
:10E9A00051F8043B4CF8044BEAD023460CF8013BE9
:10E9B00013F0FF0F4FEA3323F8D15DF8044B704793
:10E9C00011F0010F06D011F8012B0CF8012B002AD1
:10E9D00008BF704711F0020FBFD031F8022B12F0C0
:10E9E000FF0F16BF2CF8022B8CF8002012F47F4F7B
:10E9F000B3D1704711F8012B0CF8012B002AF9D183
:10EA0000704700BF20F0030110F00300C0F10000C8
:10EA100051F8043B00F1040C4FEACC0C6FF00002FB
:10EA20001CBF22FA0CF213434FF0010C4CEA0C2CE1
:10EA30004CEA0C4CA3EB0C0222EA030212EACC12C1
:10EA400004BF51F8043B0430F4D013F0FF0F1FBF94
:10EA5000013013F47F4F013013F47F0F18BF0130E2
:10EA6000704700BFF0B4002A63D0344B04461B68E3
:10EA700014F8010B571E1D186E7807F0010706F0F9
:10EA80000305012D58D011F8015B5E19767806F068
:10EA90000306012E08BF2035401B4BD1002D49D065
:10EAA000013A47D02FB314F8010B1D186E7806F009
:10EAB0000305012D11F8015B08BF20305E1976783F
:10EAC00006F00306012E08BF2035401B32D18DB35E
:10EAD000013A0ED12EE011F8012B9E18767806F03F
:10EAE0000306012E08BF2032801A23D112B36A1EFA
:10EAF00020D014F8010B1D186E7806F00305012DC7
:10EB000011F8015B08BF20305E19767806F0030625
:10EB1000012E08BF2035401B0CD15DB114F8010B4C
:10EB2000551E1A18567806F00302012AD3D1203058
:10EB3000D1E71046F0BC70472030A4E798010020D0
:10EB400041EA00039B07F0B474D1032A72D90C4642
:10EB500054F8045B161FA5F1013727EA050717F0E3
:10EB6000803F0346C6F3800C31D10346032E324664
:10EB700043F8045B2AD9BCF1000F0AD0214654F8AF
:10EB8000045BA5F1013626EA050616F0803F18D091
:10EB90001DE0264656F8045B2146A5F1013727EA19
:10EBA000050717F0803F12D143F8045B65683146D2
:10EBB000A5F1013626EA0506043A0C1D16F0803F41
:10EBC00005D1043A032A43F8045BE2D821467AB31C
:10EBD0000D78013A03F8015B9DB112F0010F1C465C
:10EBE0002AD1234622B311F8015F013A03F8015BF1
:10EBF0003DB111F8015F013A65705C1C2346002DA0
:10EC0000EFD1AAB100219C18DA4303F8011BA21826
:10EC1000A34202F001020BD01AB103F8011BA34278
:10EC200006D01A4602F8011B5970531CA342F8D1B2
:10EC3000F0BC70470346CAE711F8015F1C4604F8B0
:10EC4000015B013A2346002DCBD1DAE72DE9F0072D
:10EC500001273C4600254FF0FF3663198B4200EB3D
:10EC6000060C0DD21CF804A010F80380D0452ED25B
:10EC700001241D469F1B63198B4200EB060CF1D348
:10EC80004FF0010A1760544600254FF0FF3C63190E
:10EC9000994200EB0C080ED918F8048010F8039084
:10ECA000C1451AD901241D46CCEB030A63199942C8
:10ECB00000EB0C08F0D80CF101000136B0423CBF6B
:10ECC000BA463046C2F800A0BDE8F00770470BD046
:10ECD00001272E463C46ED19BFE709D04FF0010A47
:10ECE000AC4654465544D2E7BC4205D00134B4E7A3
:10ECF000544505D00134CAE727461D460124ACE738
:10ED0000A2461D460124C2E72DE9F04FADF2244D85
:10ED10001546064689461046194607AA1C46FFF7BF
:10ED200095FF07AB82460DF21C411A1D5C6008334B
:10ED30008B425460F9D114B301232F78611E08A8C7
:10ED4000A34240F8271001EA030218D032B16A78D2
:10ED500002234F1EA34240F8227010D0B046A446B2
:10ED60005C1C15F803E0CE1A2A5D02330F1B6345C5
:10ED700040F82E6040F82270F2D14646644607996A
:10ED800028466918524600F045FC002840F0B6803D
:10ED90000AF1FF3E05EB0E0CCDF808E0CAF1010EBA
:10EDA000834604F1FF38CDF80CC0CDF814E00746D7
:10EDB000CDF810A04A460095019408E027B1079FBE
:10EDC000BB4201D20199CB1B9B4400272246019CE8
:10EDD000B0185C440021A21A00F07CFB002840F02F
:10EDE0008780002C00F08480301910F8013C08A9BD
:10EDF00051F82330002BE1D1049B9F4228BF3B46B2
:10EE0000434527D2DDF8009006EB0B0119F80350BB
:10EE1000CA5C09EB0300954266D1DD43454415F019
:10EE2000010F024613D00133434513D24078CD5C25
:10EE3000013285420BD057E012F8010FCD5C8542BC
:10EE400052D1013312F8010FCD5C85424CD1013310
:10EE50004345F1D3DDF81090029B4F4528BF4B4648
:10EE600039D2DDF808C0DDF8009006EB0B0519F883
:10EE70000C1015F80C00814240F0C080DDF80CE069
:10EE800009EB070ACAEB0E01C80772461ED5DDF86A
:10EE9000089009F1FF31DDF80C90685C19F801CC9D
:10EEA00009F1FF32844516D10B460FE012F8019CA0
:10EEB00015F800E04A1EF1450DD10346013815F85A
:10EEC00000C011F8011C614505D10346581E52458A
:10EED00002F1FF31EAD101379F4200F29180079F92
:10EEE000019ABB44D71B71E7DDF814E0F3446BE7EC
:10EEF000002009B00DF5806DBDE8F08FCAEB04006D
:10EF0000504538BF5046CAF10102431C0AF1FF3C8C
:10EF100005EB0A0704F1FF3B019200944A46079370
:10EF2000B1464FF0000864463E46009909EB0200E6
:10EF300008EB0107BA1A002100F0CCFA0028D7D15B
:10EF4000002FD5D009EB070010F8013C08AA52F8B1
:10EF5000230000284AD1DA4509EB08002AD210F82C
:10EF60000A303178994218BF534642D16FEA0A03FA
:10EF700003EB0B01C9073246534618D50AF10103CA
:10EF80005B4517D2324612F8011F10F803E08E4598
:10EF90000DD02EE012F8011F10F803C08C4528D1C7
:10EFA000013312F8011F10F803E08E4521D101331F
:10EFB0005B45EFD3621C23469BD0295D025D9142E5
:10EFC00013D1E10709D5631EE95CC25C914204D00C
:10EFD0000BE0E95CC25C914207D15A1E002B88D03D
:10EFE000A95C825C023B9142F3D0079880443A4688
:10EFF0009BE7DDF804C0E0449844F8E7049B6AE727
:10F0000006EB0B0075E700BF2DE9F04F037889B0E0
:10F0100080460D46002B00F065810A789AB184463F
:10F020000131012602E011F8012B5AB1934214BFBD
:10F03000002606F001061CF8013F0C46002BF2D119
:10F04000207820B936B1404609B0BDE8F08F4FF0C6
:10F050000008F8E708F101002978FFF7F7FB641BC7
:10F0600006460028F3D0012C00F0B580A0444045AE
:10F0700094BFC0EB080701271F2C06D939462A4642
:10F080002346FFF741FE8046DDE7214607AA2846D2
:10F09000FFF7DCFD0799039069182846039A00F0F2
:10F0A000B9FA002840F09980DDF80CC0DDF80C902A
:10F0B0000CF1FF3E05EB0E01C9F1010C8346CDF8C2
:10F0C00008E080460491CDF814C03A46B146019557
:10F0D00008EB040609EB02000021B21A00F0FAF96D
:10F0E0000028B4D1002EB2D0039B9B4528BF5B46BD
:10F0F0009C4227D9019D09EB030010F80820E95C28
:10F10000E81891425FD1DD432D1915F0010F024639
:10F1100009EB080113D001339C4213D94078CD5C30
:10F12000013285420BD04EE012F8010FCD5C8542D2
:10F1300049D1013312F8010FCD5C854243D101332F
:10F140009C42F1D8DDF80CE0029ADE4540F2CD8019
:10F15000019B09EB0805995CA85C814240F0C580E1
:10F16000DDF804A0049BDA44CAEB0301C8071AD5F2
:10F17000029FDDF810C0791E685C1CF8017C0CF160
:10F18000FF33874214D10A460DE013F801EC2F5CDF
:10F190004B1EBE450CD1024601382F5C11F8011CF4
:10F1A000B94205D10246501E534503F1FF31ECD15F
:10F1B0000BF1010B934500F29A80079A9044C2EB41
:10F1C000040B324684E7059D05EB080B0BEB0308A7
:10F1D0004FF0000BF5E7804635E7DDF80CA003990A
:10F1E000CAEB0403534538BF5346CAF1010B581C00
:10F1F00006EB0A0205EB0A08CDF808B03B4607907B
:10F200004FF00009019201F1FF3B37468A4609EBB6
:10F210000406F8180021F21A00F05CF900287FF4C7
:10F2200016AF002E3FF413AF544598BF07EB09000B
:10F230002CD9DDF804E098F800001EF80930984257
:10F240004AD16FEA0A021119C9074246534607EB31
:10F25000090018D50AF101039C4217D9424612F859
:10F26000011F10F803C08C450DD036E012F8011FC5
:10F2700010F803E08E4530D1013312F8011F10F869
:10F2800003C08C4529D101339C42EFD8BBF1FF3F2D
:10F290005B463FF4F8AE15F80B1010F80B209142C6
:10F2A00016D11BF0010F0AD00BF1FF33E95CC25CF1
:10F2B000914204D00CE0E95CC25C914208D15A1E34
:10F2C000002B3FF4E0AEA95C825C023B9142F2D09D
:10F2D0000798814433469AE75346DDF808E0F14445
:10F2E0009944F7E70C460126AAE6039A60E74E46E2
:10F2F000C844A8E640F2C853C2F200031A680123CA
:10F300005C3200F001B800BFF0B4002825D00746F9
:10F3100038463E780D46013715F8014B3CB1A64200
:10F32000FAD1002BF4D1176007F8013C11E0C6B107
:10F330003D4600E01BB915F8016B0C46284614F851
:10F34000013B9E42F6D136B1002105F8011C106048
:10F35000781EF0BC70473046F9E710680028D6D117
:10F36000F7E716603046F4E72DE9F00F494C82B01C
:10F37000D4F800C001900F463C4614F8015B0CEB3A
:10F3800005004678274606F00800C6B2002EF3D1E5
:10F390002D2D61D02B2D04BF244614F8015BB346FC
:10F3A000002B41D1302D43D00A239A46BBF1000FE8
:10F3B0000CBF6FF000474FF00047B7FBFAF90AFBAC
:10F3C00019700090002080460CE0303DAB421BDD00
:10F3D000461C05D0C84539D835D00AFB085801204D
:10F3E00014F8015B0CEB0506767806F00407FFB213
:10F3F000002FEAD116F0030606D0012E14BF5726BF
:10F400003726AD1BAB42E3DC431C2AD0BBF1000F17
:10F4100001D0C8F10008002A31D0D0B940461160AF
:10F4200002B0BDE8F00F7047102BBED1302DBCD11B
:10F430002578782D25D0582D23D043BB4FF0080ACE
:10F4400030255346B2E700988542C6DD4FF0FF30C5
:10F45000C6E74046611EE2E714F8015B4FF0010B7E
:10F460009EE7BBF1000F01990CBF6FF000404FF019
:10F47000004022230B60002AD2D0611ECFE7404615
:10F48000CEE74FF0100A6578534602348EE79A466D
:10F4900030258BE79801002070B440F2C854C2F2C6
:10F4A000000406460D462068134631462A4670BCC5
:10F4B000FFF75ABF024B13B1024800F005B870477E
:10F4C000000000005DD90008014600200246034606
:10F4D000FEF7C4B98307F0B4C9B200F09680531E9A
:10F4E000002A00F0948002788A420BD0421CD80790
:10F4F0001AD512F0030F10461CD01478013B0132CC
:10F500008C4211D1F0BC7047002B7CD01278013BAB
:10F510008A42F7D014F0030F204604F1010209D00B
:10F520002478013B8C42EDD012F0030F104602F11B
:10F530000104E9D1032B3FD9046841EA012545EADA
:10F54000054585EA0407A7F1013222EA07021E1FDA
:10F55000041D12F0803FC6F380072DD1032E3346E1
:10F5600029D967B12668204685EA0602A2F101364C
:10F5700026EA0202043412F0803F19D01CE0204633
:10F580002468061D85EA0402A2F1013424EA02027D
:10F5900012F0803F10D13468043B85EA0402A2F1E6
:10F5A000013424EA0202341D12F0803F304603D1B8
:10F5B000043B032BE3D820465D1E23B303788B4224
:10F5C000A0D0431C0022E80714D51C78184601225D
:10F5D00001338C4296D09542184603F1010402F1A2
:10F5E00002020ED01B788B428CD020462478431C1C
:10F5F0008C4287D09542184603F1010402F10202C1
:10F60000F0D100207EE718467CE7134692E71046CB
:10F6100078E700BF032AF0B431D941EA00039C0720
:10F620002ED106680F68151F031D0C1DBE42C5F3C1
:10F63000800C24D1032D2A461FD9BCF1000F08D01D
:10F640001E6825682146184604340433AE4211D0A2
:10F6500015E0214618461C680B68051D0E1D9C42CE
:10F660000DD1314628462E680D68043A031D0C1D45
:10F67000AE4204D1043A032AEBD8214618461AB305
:10F6800003780C78A3420AD1551E0022EB0714D54B
:10F6900010F8013F11F8014F0122A3420DD0181BB1
:10F6A00010E010F8013F11F8014FA342F7D110F814
:10F6B000013F11F8014FA342F1D1AA4202F1020227
:10F6C000EFD10020F0BC70471046FBE71E1E6464BB
:10F6D000646464641048494A4B4C4D44454647FFB6
:10F6E0001048498A8B8C8D84858687FFFCF600083C
:10F6F000D4F600080BF70008E0F6000820212223CA
:10F700002425262748494A4B4C4DFF2021222324FB
:10F7100025262748498A8B8C8DFF0000E1210008AF
:10F720008F210008B32100085D2300085121000843
:10F730004D210008D9270008A52500083B26000810
:10F7400035260008BB2500082F26000800000040D1
:10F750000008014001000000001C002800000040DB
:10F760000008014002000000041C002800000040C6
:10F770000008014004000000081C002800000040B0
:10F7800000080140080000000C1C00280004004094
:10F790000008014040000000001D00280004004057
:10F7A0000008014080000000041D00280004004003
:10F7B000000C014001000000081D0028000400406A
:10F7C000000C0140020000000C1D0028002C01402C
:10F7D0000008014000010000001B0128002C01402E
:10F7E00000080140000800000C1B01280008004030
:10F7F000000C014040000000001E002800080040EE
:10F80000000C014080000000041E00280008004099
:10F81000000C014000010000081E00280008004004
:10F82000000C0140000200000C1E0028002C0140CA
:10F8300000000040000400400008004000000400F8
:10F8400008000C00D00732003200320032003200D3
:10F8500032003200C8006400000041455452313289
:10F86000333400303132333435363738394142435E
:10F870004445464748494A4B4C4D4E4F50515253D0
:10F880005455565758595A00553E0008993E00089D
:10F89000753E0008B13E0008D93E00082D3F000823
:10F8A000613E0008A53F00080000803F0000803F47
:10F8B000000000BF0000803F0000803F000000BF4C
:10F8C000000080BF0000803F0000803F000080BF3C
:10F8D0000000003F0000803F0000803F0000003F2C
:10F8E0000000803F0000803F0000803F0000003F9C
:10F8F000000080BF000080BF0000803F000080BF8C
:10F90000000000BF000080BF0000803F000000BF7B
:10F910000000803F000080BF0000803F0000803F6B
:10F920000000003F000080BF0000803FF704353F2B
:10F93000F70435BF0000803F0000803FF70435BF6B
:10F94000F70435BF0000803F0000803FF70435BF5B
:10F95000F704353F0000803F0000803FF704353F4B
:10F96000F704353F0000803F0000803F00000000AA
:10F97000000080BF000080BF0000803F000080BF0B
:10F9800000000000000080BF0000803F0000000079
:10F990000000803F000080BF0000803F0000803FEB
:10F9A00000000000000080BF0000803F000000BF9A
:10F9B000D0B35D3F0000803F0000803F000000BFEB
:10F9C000D0B35DBF0000803F0000803F0000003FDB
:10F9D000D0B35D3F000080BF0000803F0000003FCB
:10F9E000D0B35DBF000080BF0000803F000080BF3B
:10F9F00000000000000080BF0000803F0000803F4A
:10FA0000000000000000803F0000803F0000000078
:10FA10000000803F0000803F0000803F000080BF6A
:10FA2000000080BF000000000000803F00000000D8
:10FA30000000803F000080BF0000803F0000803F4A
:10FA4000000080BF000000800000803F0000000038
:10FA5000A8AAAA3F000000000000803F000080BF6D
:10FA6000B0AA2ABF000000000000803F0000803FD5
:10FA7000B0AA2ABF000000000000803F0000803FC5
:10FA800000000000000000000000803F000080BF78
:10FA900000000000000000000000803F00000000A7
:10FAA00000000000000080BF0000803F0000000058
:10FAB000000000000000803F000000000000000087
:10FAC0000301000048FA000804000000F0FC0008F0
:10FAD0000400000050FC00080201000078FA000851
:10FAE00000010000000000000600000070FD00089A
:10FAF0000600000090FC000801010000000000006A
:10FB00000400000030FD000806000000A8F900080D
:10FB100008000000D0FB00080800000028F90008D9
:10FB200008000000A8F80008010100000000000023
:10FB300000010000000000000001000000000000C3
:10FB40000400000008FA00080600000070FB00082E
:10FB500000010000000000000201000098FA000807
:10FB60000101000000000000000000000000000093
:10FB70000000803F000080BF0000803F000080BF89
:10FB80000000803F000080BF000080BF0000803F79
:10FB90000000803F0000803F0000803F0000803F69
:10FBA0000000803F0000803F000080BF000080BF59
:10FBB0000000803F00000000000000000000000086
:10FBC0000000803F00000000000000000000000076
:10FBD0000000803F000080BF0000803F000080BF29
:10FBE0000000803F000080BF000080BF0000803F19
:10FBF0000000803F0000803F0000803F0000803F09
:10FC00000000803F0000803F000080BF000080BFF8
:10FC10000000803F000080BF0000803F0000803F68
:10FC20000000803F000080BF000080BF000080BF58
:10FC30000000803F0000803F0000803F000080BF48
:10FC40000000803F0000803F000080BF0000803F38
:10FC50000000803F000080BF0000803F000080BFA8
:10FC60000000803F000080BF000080BF0000803F98
:10FC70000000803F0000803F0000803F0000803F88
:10FC80000000803F0000803F000080BF000080BF78
:10FC90000000803FD0B35DBF0000003F0000803F08
:10FCA0000000803FD0B35DBF000000BF000080BFF8
:10FCB0000000803FD0B35D3F0000003F0000803F68
:10FCC0000000803FD0B35D3F000000BF000080BF58
:10FCD0000000803F00000000000080BF0000803F67
:10FCE0000000803F000000000000803F000080BF57
:10FCF0000000803F000000000000803F000080BF47
:10FD00000000803F000080BF000000000000803F36
:10FD10000000803F0000803F000000000000803FA6
:10FD20000000803F00000000000080BF000080BF96
:10FD30000000803F000000000000803F000080BF06
:10FD40000000803F000080BF000080BF0000000076
:10FD50000000803F000000000000803F0000803F66
:10FD60000000803F0000803F000080BF00000000D6
:10FD70000000803F00000000A8AAAA3F0000803FCA
:10FD80000000803F000080BFB0AA2ABF000080BFF3
:10FD90000000803F0000803FB0AA2ABF000080BF63
:10FDA0000000803F00000000A8AAAA3F000080BF1A
:10FDB0000000803F000080BFB0AA2ABF0000803F43
:10FDC0000000803F0000803FB0AA2ABF0000803FB3
:10FDD00024505542582C34312C312C303030332CB7
:10FDE000303030312C3131353230302C302A314501
:10FDF0000D0A0024504D544B3235312C31313532FF
:10FE000030302A31460D0A0024505542582C3431E6
:10FE10002C312C303030332C303030312C353736DB
:10FE200030302C302A32440D0A0024504D544B32CD
:10FE300035312C35373630302A32430D0A00245004
:10FE40005542582C34312C312C303030332C30305A
:10FE500030312C33383430302C302A32360D0A0011
:10FE600024504D544B3235312C33383430302A3213
:10FE7000370D0A0024505542582C34312C312C3087
:10FE80003030332C303030312C31393230302C306E
:10FE90002A32330D0A0024504D544B3235312C3167
:10FEA000393230302A32320D0A00B56206010300C1
:10FEB000F00500FF19B56206010300F00300FD150F
:10FEC000B56206010300F00100FB11B562060103F3
:10FED00000F00000FA0FB56206010300F00200FC1A
:10FEE00013B56206010300F00400FE17B5620601B7
:10FEF00003000102010E47B5620601030001030180
:10FF00000F49B56206010300010601124FB56206F2
:10FF10000103000112011E67B562061608000307FF
:10FF200003000000000031E5B56206080600C800C5
:10FF300001000100DE6A00000000000000C20100B4
:10FF4000D0FD0008F3FD00080100000000E1000002
:10FF500008FE00082AFE00080200000000960000CB
:10FF60003EFE000860FE000803000000004B000099
:10FF700074FE000896FE00080400000080250000C2
:10FF8000D7060108D70601084145525431323334AF
:10FF900000002710080423022001000000000000D8
:10FFA0008025000000C201000200000001000000E6
:10FFB0008025000000C201000300000002000000D4
:10FFC00080250000004B0000050000000300000039
:10FFD00080250000004B000005000000020010001A
:10FFE0002000010008030400780F01087C0F0108BD
:10FFF000810F0108920F01089B0F0108A60F01084D
:020000040801F1
:10000000B10F0108BC0F01088A0E0108C50F0108D5
:10001000840E0108CE0F0108D80F0108E30F010874
:10002000E90F0108EC0F010800000000CA0E0108EA
:10003000CE0E0108D40E0108DA0E0108DD0E01080B
:10004000E40E0108E70E0108EC0E0108F80E0108A5
:10005000FB0E0108010F0108080F0108120F01082B
:100060001C0F0108250F0108330F01083F0F01087D
:10007000460F01084C0F0108590F0108640F0108D1
:10008000710F010800000000D40C0108D80C010811
:10009000E9960008FF0C0108040D0108B59100085D
:1000A000180D0108210D01089D9100083E0D010861
:1000B000430D01084D970008720D0108D70601088D
:1000C00065910008770D01087F0D010879900008FF
:1000D000930D0108A20D010859900008BC0D0108FC
:1000E000D7060108A98D0008C10D0108C50D01083A
:1000F000B18F0008120D0108E10D010801940008FC
:10010000F40D0108FA0D010841960008150E0108CA
:100110001D0E0108F59500082C0E0108310E01088E
:10012000898F0008B7030108410E0108A194000857
:100130006F0E0108630E0108D58D0008BA0801088A
:10014000D70601089D8D0008D7060108960E010804
:100150009E0E0108A60E0108AE0E0108B50E01089C
:10016000C00E0108C50E0108000000004166726F54
:10017000333220434C492076657273696F6E2032AA
:100180002E32204D61792031302032303134202F11
:100190002031373A30383A3432202D2028636C65CC
:1001A000616E666C696768742900417661696C618B
:1001B000626C6520636F6D6D616E64733A0D0A0049
:1001C00025730925730D0A0053797374656D2055E5
:1001D0007074696D653A202564207365636F6E6481
:1001E000732C20566F6C746167653A202564202A51
:1001F00020302E31562028256453206261747465A6
:100200007279290D0A004350552025644D487A2CF7
:100210002064657465637465642073656E736F72C2
:10022000733A20002573200041434348573A202564
:1002300073002E2563004379636C652054696D65F6
:100240003A2025642C20493243204572726F727324
:100250003A2025642C20636F6E6669672073697A83
:10026000653A2025640D0A00202564202564000DD0
:100270000A5265626F6F74696E672E2E2E0053618D
:1002800076696E672E2E2E004D7573742062652080
:10029000616E79206F72646572206F6620414554EB
:1002A00052313233340D0A0043757272656E742018
:1002B00061737369676E6D656E743A200045727282
:1002C0006F723A20456E61626C6520616E642070C9
:1002D0006C756720696E204750532066697273748D
:1002E0000D0A00456E61626C656420666561747517
:1002F0007265733A2000417661696C61626C6520B9
:1003000066656174757265733A2000496E76616C3A
:1003100069642066656174757265206E616D652E15
:100320002E2E0D0A0044697361626C6564200045DD
:100330006E61626C656420000D0A4C656176696EC1
:100340006720434C49206D6F64652E2E2E0D0A00E8
:10035000526573657474696E6720746F2064656696
:1003600061756C74732E2E2E004E4709004F4B0999
:1003700000437573746F6D206D697865723A200D56
:100380000A4D6F746F720954687209526F6C6C0970
:100390005069746368095961770D0A002325643A2E
:1003A00009002573090053616E69747920636865DB
:1003B000636B3A09007265736574006C6F61640069
:1003C000496E76616C6964206D6978657220747914
:1003D00070652E2E2E0D0A004C6F61646564202519
:1003E00073206D69782E2E2E0D0A0057726F6E677E
:1003F000206E756D626572206F6620617267756D23
:10040000656E74732C206E65656473206964782052
:1004100074687220726F6C6C2070697463682079E4
:1004200061770D0A004D6F746F72206E756D626595
:1004300072206D75737420626520626574776565DE
:100440006E203120616E642025640D0A00437572B0
:1004500072656E74206D697865723A2025730D0A95
:1004600000417661696C61626C65206D69786572C6
:10047000733A20004D697865722073657420746F3B
:100480002025730D0A0043757272656E74207365C2
:100490007474696E67733A200D0A002573207365C2
:1004A0007420746F20004552523A2056616C756575
:1004B0002061737369676E6D656E74206F7574204B
:1004C0006F662072616E67650D0A004552523A20D0
:1004D000556E6B6E6F776E207661726961626C65C6
:1004E000206E616D650D0A0043757272656E742031
:1004F00070726F66696C653A2025640D0A00557349
:100500006167653A0D0A6D6F746F7220696E64657C
:1005100078205B76616C75655D202D2073686F7740
:10052000205B6F72207365745D206D6F746F722035
:1005300076616C75650D0A004E6F207375636820D7
:100540006D6F746F722C207573652061206E756DF0
:10055000626572205B302C2025645D0D0A004D6FB2
:10056000746F722025642069732073657420617430
:100570002025640D0A00496E76616C6964206D6FF8
:10058000746F722076616C75652C20313030302E9E
:100590002E323030300D0A0053657474696E672056
:1005A0006D6F746F7220256420746F2025640D0AAE
:1005B000006175782025752025750D0A00496E7635
:1005C000616C6964204665617475726520696E644A
:1005D00065783A206D757374206265203C2025751E
:1005E0000D0A0043757272656E7420436F6E666902
:1005F000673A20436F70792065766572797468690F
:100600006E672062656C6F7720686572652E2E2E8E
:100610000D0A006D697865722025730D0A00636DFF
:10062000697820256400636D697820256420302076
:1006300030203020300D0A006665617475726520C7
:100640002D25730D0A00666561747572652025732A
:100650000D0A006D61702025730D0A00736574200A
:100660002573203D20000D0A456E746572696E6722
:1006700020434C49204D6F64652C207479706520AF
:1006800027657869742720746F2072657475726E9F
:100690002C206F72202768656C70270D0A000D0AE8
:1006A0002320000D1B5B4B001B5B324A1B5B313B65
:1006B0003148004552523A20556E6B6E6F776E206E
:1006C000636F6D6D616E642C20747279202768658C
:1006D0006C702700082008006C6F6F7074696D657E
:1006E00000656D665F61766F6964616E6365006D5C
:1006F00069647263006D696E636865636B006D6148
:1007000078636865636B006D696E7468726F74748A
:100710006C65006D61787468726F74746C65006DDF
:10072000696E636F6D6D616E6400646561646261C2
:100730006E6433645F6C6F77006465616462616EE0
:100740006433645F68696768006E65757472616CB4
:100750003364006465616462616E6433645F74680D
:10076000726F74746C65006D6F746F725F70776D0B
:100770005F7261746500736572766F5F70776D5F2D
:10078000726174650072657461726465645F617240
:100790006D00666C6170735F737065656400666997
:1007A00078656477696E675F616C74686F6C645FAD
:1007B0006469720073657269616C5F706F72745FF7
:1007C000315F7363656E6172696F00736572696131
:1007D0006C5F706F72745F325F7363656E617269B4
:1007E0006F0073657269616C5F706F72745F335F05
:1007F0007363656E6172696F0073657269616C5FC6
:10080000706F72745F345F7363656E6172696F00DD
:100810007265626F6F745F63686172616374657241
:10082000006D73705F626175647261746500636C02
:10083000695F6261756472617465006770735F708F
:100840006173737468726F7567685F6261756472F3
:10085000617465006770735F70726F76696465724A
:10086000006770735F696E697469616C5F6261755E
:1008700064726174655F696E64657800736572693E
:10088000616C72785F70726F76696465720074650E
:100890006C656D657472795F70726F76696465728C
:1008A0000074656C656D657472795F7377697463E4
:1008B00068006672736B795F696E76657273696FD3
:1008C0006E00766261747363616C65007662617458
:1008D0006D617863656C6C766F6C746167650076CA
:1008E0006261746D696E63656C6C766F6C74616760
:1008F0006500706F7765725F6164635F6368616EE6
:100900006E656C00616C69676E5F6779726F00611C
:100910006C69676E5F61636300616C69676E5F6DD0
:10092000616700616C69676E5F626F6172645F72BC
:100930006F6C6C00616C69676E5F626F6172645F9F
:10094000706974636800616C69676E5F626F617281
:10095000645F796177006D61785F616E676C655F78
:10096000696E636C696E6174696F6E006779726F2E
:100970005F6C7066006D6F726F6E5F746872657326
:10098000686F6C64006779726F5F636D70665F6635
:100990006163746F72006779726F5F636D70666D0B
:1009A0005F666163746F7200616C745F686F6C6422
:1009B0005F7468726F74746C655F6E657574726174
:1009C0006C00616C745F686F6C645F666173745F08
:1009D0006368616E6765007468726F74746C655FDC
:1009E000636F7272656374696F6E5F76616C756553
:1009F000007468726F74746C655F636F72726563A4
:100A000074696F6E5F616E676C65007961776465AC
:100A1000616462616E64007961775F636F6E7472A6
:100A20006F6C5F646972656374696F6E007961777A
:100A30005F646972656374696F6E007472695F7573
:100A40006E61726D65645F736572766F0072635F6D
:100A5000726174650072635F6578706F00746872AC
:100A60005F6D6964007468725F6578706F00726FA3
:100A70006C6C5F70697463685F7261746500796142
:100A8000775F72617465007470615F726174650094
:100A90007470615F627265616B706F696E7400661D
:100AA00061696C736166655F64656C61790066613C
:100AB000696C736166655F6F66665F64656C6179BA
:100AC000006661696C736166655F7468726F7474E7
:100AD0006C65006661696C736166655F6465746509
:100AE00063745F7468726573686F6C6400727373AB
:100AF000695F6175785F6368616E6E656C006769D8
:100B00006D62616C5F666C616773006163635F68EF
:100B100061726477617265006163635F6C70665FC8
:100B2000666163746F720061636378795F646561A5
:100B30006462616E64006163637A5F6465616462CC
:100B4000616E64006163635F756E61726D6564639D
:100B5000616C006163635F7472696D5F7069746377
:100B600068006163635F7472696D5F726F6C6C00C3
:100B70006261726F5F7461625F73697A650062615E
:100B8000726F5F6E6F6973655F6C70660062617231
:100B90006F5F63665F76656C006261726F5F63664C
:100BA0005F616C74006D61675F6465636C696E6141
:100BB00074696F6E006770735F706F735F7000674A
:100BC00070735F706F735F69006770735F706F73CE
:100BD0005F64006770735F706F73725F700067703F
:100BE000735F706F73725F69006770735F706F73AC
:100BF000725F64006770735F6E61765F700067702C
:100C0000735F6E61765F69006770735F6E61765FB8
:100C100064006770735F77705F72616469757300F9
:100C20006E61765F636F6E74726F6C735F6865611F
:100C300064696E67006E61765F73706565645F6D91
:100C4000696E006E61765F73706565645F6D617873
:100C5000006E61765F736C65775F726174650070BA
:100C600069645F636F6E74726F6C6C657200705F45
:100C7000706974636800695F706974636800705FAD
:100C8000726F6C6C00695F726F6C6C00705F796181
:100C90007700695F79617700705F616C7400695FEC
:100CA000616C7400645F616C7400705F6C65766584
:100CB0006C00695F6C6576656C00645F6C65766579
:100CC0006C00705F76656C00695F76656C00645FD0
:100CD00076656C0061757800666561747572655F34
:100CE0006E616D6520617578666C6167206F72203A
:100CF000626C616E6B20666F72206C697374006346
:100D00006D69780064657369676E20637573746FCD
:100D10006D206D697865720064656661756C7473C9
:100D200000726573657420746F2064656661756C0C
:100D3000747320616E64207265626F6F74006475F5
:100D40006D70007072696E7420636F6E666967758E
:100D50007261626C652073657474696E6773206973
:100D60006E2061207061737461626C6520666F72C1
:100D70006D00657869740066656174757265006CF4
:100D8000697374206F72202D76616C206F722076EB
:100D9000616C00677073706173737468726F7567EC
:100DA0006800706173737468726F7567682067702C
:100DB0007320746F2073657269616C0068656C7074
:100DC000006D6170006D617070696E67206F6620E4
:100DD0007263206368616E6E656C206F7264657209
:100DE000006D69786572206E616D65206F72206C90
:100DF000697374006D6F746F72006765742F73652B
:100E000074206D6F746F72206F75747075742076B6
:100E1000616C75650070726F66696C6500696E64FF
:100E2000657820283020746F203229007361766540
:100E3000007361766520616E64207265626F6F7405
:100E4000006E616D653D76616C7565206F72206224
:100E50006C616E6B206F72202A20666F72206C6945
:100E600073740073686F772073797374656D207382
:100E70007461747573004759524F004143430042F7
:100E800041524F00534F4E4152004750530047507C
:100E9000532B4D4147004144584C333435004D509D
:100EA0005536303530004D4D413834357800424D9F
:100EB00041323830004C534D333033444C484300BA
:100EC00046414B45004E6F6E6500545249005155E6
:100ED0004144500051554144580042490047494D52
:100EE00042414C005936004845583600464C594955
:100EF0004E475F57494E47005934004845583658C9
:100F0000004F43544F5838004F43544F464C4154C0
:100F100050004F43544F464C4154580041495250A1
:100F20004C414E450048454C495F3132305F4343A8
:100F3000504D0048454C495F39305F4445470056A5
:100F40005441494C340048455836480050504D5F94
:100F5000544F5F534552564F004455414C434F50F8
:100F60005445520053494E474C45434F5054455207
:100F700000435553544F4D0050504D00564241547C
:100F800000494E464C494748545F4143435F434103
:100F90004C0053455249414C5258004D4F544F520A
:100FA0005F53544F5000534552564F5F54494C5471
:100FB00000534F465453455249414C004C45445F01
:100FC00052494E47004641494C534146450054451D
:100FD0004C454D4554525900504F5745524D45547C
:100FE000455200564152494F00334400504152414E
:100FF0004C4C454C5F50574D00000000760E0108E8
:101000007B0E01087F0E0108920E0108840E010874
:101010008A0E01088E0E010800000000D8060108A3
:1010200002000000541800200000000028230000E7
:10103000E106010800000000561800200000000032
:1010400001000000EF060108020000005A1900200C
:10105000B0040000A4060000F5060108020000002C
:101060005C19002000000000D0070000FE06010807
:10107000020000005E19002000000000D007000000
:1010800007070108020000001819002000000000F6
:10109000D007000013070108020000001A19002001
:1010A00000000000D00700001F0701080200000038
:1010B0001C19002000000000D00700002A070108CA
:1010C000020000001E19002000000000D0070000F0
:1010D000390701080200000020190020000000006C
:1010E000D007000049070108020000002219002073
:1010F00000000000D00700005307010802000000B4
:101100002419002000000000D00700006707010834
:10111000020000002619002032000000007D0000BF
:1011200076070108020000002819002032000000A4
:10113000F20100008507010800000000601900208E
:1011400000000000010000009207010800000000FC
:101150006119002000000000640000009E070108E3
:101160000100000062190020FFFFFFFF01000000E6
:10117000B40701080000000068190020000000000A
:1011800008000000CB0701080000000069190020DA
:101190000000000008000000E20701080000000055
:1011A0006A1900200000000008000000F90701088B
:1011B000000000006B190020000000000800000083
:1011C00010080108000000007C1900203000000019
:1011D0007E00000021080108040000006C190020B6
:1011E000B004000000C201002E0801080400000045
:1011F00070190020B004000000C201003B08010883
:101200000400000074190020B004000000C20100B6
:1012100054080108000000006419002000000000CC
:1012200002000000610801080100000065190020AB
:1012300000000000040000007C080108000000001D
:101240005819002000000000040000008E0801086A
:1012500000000000801900200000000001000000D4
:10126000A108010800000000811900200000000012
:1012700001000000B20801080000000082190020EF
:101280000000000001000000C2080108000000008A
:101290004C1900200A000000C8000000CC0801081A
:1012A000000000004D1900200A000000320000007C
:1012B000DF080108000000004E1900200A000000AD
:1012C00032000000F2080108000000004F19002061
:1012D00000000000090000000409010800000000EF
:1012E0002A19002000000000080000000F09010872
:1012F000000000002B190020000000000800000082
:1013000019090108000000002C190020000000004D
:101310000800000023090108030000002E19002026
:101320004CFFFFFF680100003409010803000000C2
:10133000301900204CFFFFFF68010000460901083A
:1013400003000000321900204CFFFFFF680100007D
:1013500056090108020000003E1900206400000048
:10136000840300006C090108020000003619002007
:1013700000000000000100007509010800000000E5
:101380003C190020000000008000000085090108D1
:10139000020000003819002064000000E80300008B
:1013A00096090108020000003A19002064000000BC
:1013B000E8030000A8090108000000006E1C0020DE
:1013C00001000000FA000000C2090108000000004E
:1013D0006F1C00200000000001000000D709010878
:1013E00000000000721C00200000000096000000B9
:1013F000F109010802000000701C0020010000003B
:10140000840300002D0B0108000000006C1C00206C
:1014100000000000200000000B0A0108000000008E
:101420006D1C00200000000064000000170A010885
:101430000100000034190020FFFFFFFF0100000041
:101440002D0A010801000000BA1C0020FFFFFFFF69
:10145000010000003B0A010801000000BB1C002045
:1014600000000000010000004D0A0108000000001B
:101470001B1C002000000000FA000000550A0108B3
:10148000000000001C1C00200000000064000000A0
:101490005D0A0108000000001D1C00200000000083
:1014A00064000000650A0108000000001E1C002006
:1014B00000000000640000006E0A01080000000047
:1014C0001F1C002000000000640000007E0A0108CC
:1014D00000000000201C002000000000640000004C
:1014E000870A010800000000211C00200000000005
:1014F00064000000900A010802000000221C002085
:10150000E8030000D00700009F0A01080000000067
:10151000B41C002000000000C8000000AE0A010852
:1015200000000000B51C002000000000C800000002
:10153000C10A010802000000B61C0020E8030000F8
:10154000D0070000D30A010802000000B81C0020E8
:1015500064000000D0070000ED0A0108010000004F
:10156000631900200000000004000000FE0A0108CA
:1015700000000000BC1C002000000000FF00000074
:101580000B0B0108000000003519002000000000CE
:1015900005000000180B0108000000002A1C0020B4
:1015A00000000000FA000000270B01080000000006
:1015B0002C1C00200000000064000000360B010815
:1015C000000000002B1C0020000000006400000050
:1015D000440B010800000000401C00200000000037
:1015E00001000000530B010803000000281C00202C
:1015F000D4FEFFFF2C010000620B01080300000075
:10160000261C0020D4FEFFFF2C010000700B0108F7
:1016100000000000301C002000000000300000002E
:101620007E0B010805000000341C002000000000B3
:10163000010000008D0B010805000000381C00208F
:101640000000000001000000990B010805000000E7
:101650003C1C00200000000001000000A50B010858
:1016600003000000241C0020B0B9FFFF504600001A
:10167000B50B010800000000011C00200000000064
:10168000C8000000BF0B0108000000000B1C002078
:1016900000000000C8000000C90B010800000000A5
:1016A000151C002000000000C8000000D30B01083A
:1016B00000000000021C002000000000C800000024
:1016C000DE0B0108000000000C1C002000000000E0
:1016D000C8000000E90B010800000000161C0020F3
:1016E00000000000C8000000F40B0108000000002A
:1016F000031C002000000000C8000000FE0B0108D1
:10170000000000000D1C002000000000C8000000C8
:10171000080C010800000000171C00200000000059
:10172000C8000000120C010802000000BE1C0020CE
:1017300000000000D0070000200C0108000000009D
:10174000C21C00200000000001000000350C010850
:1017500002000000C41C00200A000000D0070000A6
:10176000430C010802000000C61C00200A00000013
:10177000D0070000510C010800000000C11C00202F
:1017800000000000640000005F0C01080000000081
:10179000FC1B002000000000010000006E0C01088E
:1017A00000000000FE1B002000000000C800000038
:1017B000760C010800000000081C0020000000005A
:1017C000C80000003E09010800000000121C0020B3
:1017D00000000000C80000007E0C010800000000AE
:1017E000FD1B002000000000C8000000850C01085F
:1017F00000000000071C002000000000C8000000DE
:101800002D09010800000000111C0020000000004C
:10181000C80000008C0C010800000000FF1B002025
:1018200000000000C8000000920C01080000000049
:10183000091C002000000000C80000005009010839
:1018400000000000131C002000000000C800000081
:10185000980C010800000000001C0020000000009F
:10186000C80000009E0C0108000000000A1C0020B7
:1018700000000000C8000000A40C010800000000E7
:10188000141C002000000000C8000000AA0C010881
:1018900000000000041C002000000000C800000040
:1018A000B20C0108000000000E1C00200000000027
:1018B000C8000000BA0C010800000000181C00203D
:1018C00000000000C8000000C20C01080000000079
:1018D000061C002000000000C8000000C80C010821
:1018E00000000000101C002000000000C8000000E4
:1018F000CE0C0108000000001A1C002000000000AF
:10190000C8000000524F4C4C3B50495443483B598F
:1019100041573B414C543B506F733B506F73523BAC
:101920004E6176523B4C4556454C3B4D41473B56EC
:10193000454C3B0041524D3B00414E474C453B001E
:10194000484F52495A4F4E3B004241524F3B00567E
:101950004152494F3B004D41473B004845414446B9
:101960005245453B004845414441444A3B004341C0
:101970004D535441423B0043414D545249473B0073
:1019800047505320484F4D453B0047505320484F48
:101990004C443B0050415353544852553B00424540
:1019A000455045523B004C45444D41583B004C4549
:1019B000444C4F573B004C4C49474854533B004321
:1019C000414C49423B00474F5645524E4F523B0017
:1019D0004F53442053573B0054454C454D455452BA
:1019E000593B00000000004B000000CB61636F73A7
:1019F0006600000000000000737172746600000051
:101A0000000FC93F000F494000CB9640000FC9406E
:101A10000053FB4000CB164100ED2F41000F494120
:101A20000031624100537B41003A8A4100CB96412C
:101A3000005CA34100EDAF41007EBC41000FC941F5
:101A400000A0D5410031E24100C2EE410053FB410C
:101A500000F20342003A0A420083104200CB1642D1
:101A600000141D42005C234200A5294200ED2F42D4
:101A700000363642007E3C4200C74242000F4942D7
:101A8000A2000000F9000000830000006E000000CA
:101A90004E00000044000000150000002900000076
:101AA000FC0000002700000057000000D1000000EB
:101AB000F500000034000000DD000000C000000060
:101AC000DB000000620000009500000099000000AB
:101AD0003C000000430000009000000041000000B6
:101AE000FE0000005100000063000000AB00000099
:101AF000DE000000BB000000C50000006100000027
:101B0000B7000000240000006E0000003A00000052
:101B1000420000004D000000D2000000E000000084
:101B200006000000490000002E000000EA0000004E
:101B300009000000D1000000920000001C0000001D
:101B4000FE0000001D000000EB0000001C00000073
:101B5000B100000029000000A70000003E000000C6
:101B6000E80000008200000035000000F5000000E1
:101B70002E000000BB0000004400000084000000B4
:101B8000E90000009C00000070000000260000003A
:101B9000B40000005F0000007E0000004100000073
:101BA0003900000091000000D6000000390000005C
:101BB000830000005300000039000000F400000022
:101BC0009C000000840000005F0000008B0000000B
:101BD000BD000000F9000000280000003B000000EC
:101BE0001F000000F800000097000000FF00000048
:101BF000DE00000005000000980000000F0000005B
